:100000000C94220E0C943F0E0C943F0E0C943F0E59
:100010000C943F0E0C9447100C946C120C943F0EF1
:100020000C943F0E0C943F0E0C943F0E0C943F0E1C
:100030000C943F0E0C943F0E0C94B3240C943F0E82
:100040000C94AE150C947D130C9457100C940E1058
:100050000C943F0E0C94EB1F0C943F0E0C943F0E2F
:100060000C943F0E0C943F0E0C943F0E0C943F0EDC
:100070000C943F0E0C945B250C9480120C942E1261
:100080000C943F0E0C94F25E0C943F0E3859045AB7
:1000900073584159185AA558BB58665A665A665A39
:1000A000D958665A665A665A665A5559E459E459F7
:1000B000005A99599959975995599359665A665AB8
:1000C000665A665A665A665A665A2859665A665A6F
:1000D000665A665A665A665A665A665A665A665A20
:1000E000665A665A665A665A665A665A665A665A10
:1000F000665A665A665A665A665A665A665A665A00
:10010000665A665A665A665A665A575A495A375A4A
:100110001C5A45617379436F6E74726F6C00204D89
:100120004300696E636F6D70617469626C6520482D
:100130005700312E342E33005F03AF01D7006B0020
:10014000470035001A0011000102031304050611CF
:10015000070809120A000B0C100F0E0D0101010512
:100160000D1F0C04040E1F04041F0E041F1F1F008C
:100170001F1F1F001F1F1F001F111F001F111F0027
:100180001F1F1F001F111F001F111F00000609174E
:1001900017090600000609121412090603070F1EAC
:1001A0001C18100003050912141810000707070790
:1001B0000707070707050505050505071C1018179C
:1001C000150705071C101817110202021C1018123F
:1001D000140605021C101817140601061C10181529
:1001E000150701011C101816110201061C10181623
:1001F000110204071C10181216020207040A110A41
:100200000A0E00000C17141714170C001C101810FD
:10021000160505051F0A0A0A0A0A1F000E11111FFA
:100220001B1B1F0002060F1F0F060200080C1E1FDB
:100230001E0C08000E0E0E0E1F0E0400040E1F0EE4
:100240000E0E0E0000C030F00CCC3CFC03C333F3A8
:100250000FCF3FFFC303F333CF0FFF3FAAC0803060
:10026000F0B020E0A00CCC8C3CFCBC2CECAC08C862
:100270008838F8B828E8A803C38333F3B323E3A38B
:100280000FCF8F3FFFBF2FEFAF0BCB8B3BFBBB2BBA
:10029000EBAB02C28232F2B222E2A20ECE8E3EFE60
:1002A000BE2EEEAE0ACA8A3AFABA2AEA004060972F
:1002B0007048685878446454744C6C5C7C42625258
:1002C000724A6A5A7A466656764E6E5E7E41615131
:1002D000714969597945659F754D6D5D7D436353DE
:1002E000734B6B5B7B476757774F6F5F7F101814BB
:1002F0001C121A161E1119151D131B171FD0D8D446
:10030000DCD2DAD6DED1D9D5DDD3DBD7DF90989435
:100310009C929A969E9199959D939B5055040605A3
:1003200007C4C6C5C78486858734363537F4F6F5E5
:10033000F7B4B6B5B724262527E4E6E5E7A4A6A5D5
:10034000A701C18131F1B121E1A10DCD8D3DFDBDEF
:100350002DEDAD09C98939F9B929E9A92020202055
:1003600020200000204D4D4920200000204D4D014F
:100370002020000020444343202000002053544FFD
:100380005020000053484F52542100002048414C57
:100390005420000000000000000000002050524FD8
:1003A0004720000052455345542000007E0E0E0E9B
:1003B0000E1B1B1C0E1B1B7E0E0E0E0E232D004152
:1003C00044523A20256C6420202020202020202028
:1003D00020002D2D2D2D202000252D3564002533C6
:1003E0006400202001022020202020202000252D34
:1003F000356400252D31312E313173000002070B99
:100400001014191D22262B3035393F43484C5156C4
:100410005B5F64696D72767B7F0002070C10151AB2
:100420001E23282C31363A3F44484D52565B6064B7
:10043000696E73797F00020C151D263039434C56C6
:100440005F69727F2530386C75005741524E494EB6
:10045000473A20004552524F523A200062616420D0
:10046000706172616D657465722076616C7565008E
:10047000706F776572206973204F666600747572BD
:100480006E6F75742071756575652066756C6C008E
:10049000636F6D6D616E642071756575652066753D
:1004A0006C6C006E6F2064617461006E6F20736C01
:1004B0006F7420617661696C61626C65006C6F6B52
:1004C000206275737900696C6C6567616C20747566
:1004D000726E6F757420616472657373004D432092
:1004E000696E2048414C54004D4320696E2053549E
:1004F0004F50004C207B4C6F6B232C205B5370655E
:1005000065645D2C205B464C5D2C205B4469725D0C
:100510002C205B46315D2C205B46325D2C205B46F7
:10052000335D2C205B46345D7D0054207B54726E1D
:1005300074232C205B436F6C6F725D2C205B5374B3
:10054000617475735D7D0046207B4C6F6B232C209E
:100550005B46315D2C205B46325D2C205B46335D73
:100560002C205B46345D2C205B46355D2C205B46A1
:10057000365D2C205B46375D2C205B46385D7D0068
:10058000484C2048656C7020666F72206C6F6B2041
:10059000636F6D6D616E64730D0048462048656C35
:1005A0007020666F722066756E6374696F6E20636B
:1005B0006F6D6D616E64730D0048542048656C70FA
:1005C00020666F72207475726E6F757420636F6D24
:1005D0006D616E647300507772206F6666004861CB
:1005E0006C7465642100507772206F6E0044434341
:1005F0002070726F6772616D005245534554004818
:10060000616C746564210D5D004C20257520257595
:100610002025632025632025632025632025632072
:10062000256300756E75736564004D6F746F726F2E
:100630006C61204F6C64004D6F746F726F6C612041
:100640004E657700444343004620257520256320EE
:10065000256320256320256320256320256320252D
:1006600063202563004658202575202563202563D7
:100670002025632025632025632025630054202541
:1006800064202563202564004D43205265766973FC
:10069000696F6E2000312E342E33000D5365724E7B
:1006A000722E2025386C75004D5420256420256459
:1006B000005352202564004D6F64756C652023251E
:1006C000642028696E70757420312E2E3820262003
:1006D000392E2E313629203D200053452025640037
:1006E0003537363030002575000D5D002564002556
:1006F000642C2025642C20004D4D31004D4D3200DE
:10070000444343002C2025730D002A454E442A0003
:1007100025732564002A454E442A005A7A41005523
:100720006E6B6E6F776E20636F6D6D616E64000D22
:100730005D003132000032340000343800003936B8
:100740000000313434003139320033383400353769
:1007500036004142434445464748494A4B4C4D4E7A
:100760004F505152535455565758595A30313233CD
:100770003435363738392E2C3A2D2B232F3D3C7CFF
:100780003E20004D4D20492020313420004D4D2089
:10079000492020323761004D4D20492020323762F8
:1007A000004D4D20012020313420004D4D200120EE
:1007B00020323761004D4D20012020323762004445
:1007C0004343202020313420004443432020203262
:1007D000382000444343202031323820004C6F63DE
:1007E0006D656E750000000000000000004443438A
:1007F0002D70726F6772616D6D2E0000004D6F6419
:10080000656C6261616E7369742E000000496E73DD
:1008100074656C6C696E67656E00000000536F66EE
:10082000747761726520557064617465004C43444F
:10083000207665726C69636874696E67004D6173D8
:10084000746572436F6E74726F6C00000045786956
:10085000740000000000000000000000004B69650B
:100860007A656E2000000000000000000044617402
:1008700061666F726D61740000000000004E61617E
:100880006D202020202020000000000000496E760E
:100890006F657220202020000000000000435620D9
:1008A000286279746529000000000000004356208A
:1008B0002862697429000000000000000042617392
:1008C000697361647265730000000000004C616E22
:1008D0006720616472657300000000000052656764
:1008E00069737465720000000000000000506167C9
:1008F000652D4D6F646500000000000000486F6FBB
:10090000666473706F6F7200000000000073383807
:100910002D696E7374656C6C696E67656E436F6E7E
:1009200066696775726174696500000000426F6FE7
:1009300073746572000000000000000000496E74CE
:100940006572666163652042617564000057697372
:1009500073656C000000000000000000004C6F6335
:10096000666F726D6174000000000000004D4D2044
:100970007369676E61616C7061757A650073383890
:100980002D6D6F64756C65000000000000733838D1
:100990002D6D6F64756C657465737400004B6F72B8
:1009A00074736C2E20706F6C2E000000004B6F7201
:1009B00074736C2E206765762E00000000616C6CED
:1009C000652057697373656C0000000000576973F8
:1009D00073656C666F726D6174000000004D696E26
:1009E0002E736368616B656C74696A64004D61782D
:1009F0002E736368616B656C74696A64004D656E23
:100A000075204C6F636F0000000000000050726F93
:100A10006772616D2E2044434300000000457461FD
:100A200074205265736561752E0000000052656781
:100A30006C6167657300000000000000004D414AD2
:100A4000206C6F67696369656C000000004C756D10
:100A5000696E6F736974650000000000004D61737A
:100A6000746572436F6E74726F6C00000045786934
:100A70007400000000000000000000000053656CDE
:100A8000656374696F6E20000000000000466F729D
:100A90006D617420646F6E6E65657300004E6F6DDE
:100AA0002020202020202000000000000053616949
:100AB00073696520202020000000000000435620BC
:100AC0002862797465290000000000000043562068
:100AD000286269742900000000000000004164726F
:100AE000657373652064652062617365004164729B
:100AF00065737365206C6F6E67756500005265677E
:100B000069737465720000000000000000506167A6
:100B1000652D4D6F646500000000000000566F6990
:100B200065207072696E636970616C6500526567FB
:100B30006C616765207338380000000000436F6EF9
:100B400066696775726174696F6E000000426F6F4D
:100B500073746572000000000000000000496E74AC
:100B600065726661636520426175640000436F6E63
:100B7000662E2041696775696C6C612E00466F7244
:100B80006D6174206C6F636F000000000050617530
:100B90007365207369676E616C204D4D004D6F6405
:100BA000756C65732073383800000000005465735D
:100BB00074206D6F64756C652073383800506F6CED
:100BC0002E6372742D636972637569740053656E68
:100BD000732E206372742D636972637400746F7571
:100BE000732041696775696C6C65730000466F72AC
:100BF0006D61742061696775696C6C2E0054707347
:100C0000206D696E2E696D70756C732E0054707353
:100C1000206D61782E696D70756C732E004C6F6B52
:100C2000204D656EFC0000000000000000444343BE
:100C30002D50726F6772616D6D672E0000416E6C92
:100C40006167656E7A757374616E64000045696EE4
:100C50007374656C6C756E67656E000000536F662B
:100C6000747761726520557064617465004C43440B
:100C70002042656C6575636874756E67004D6173BD
:100C8000746572436F6E74726F6C00000045786912
:100C900074000000000000000000000000417573B7
:100CA00077E4686C656E2000000000000044617409
:100CB000656E666F726D617400000000004E616DBC
:100CC0006520202020202000000000000045696EE3
:100CD000747261672020200000000000004356204D
:100CE0002862797465290000000000000043562046
:100CF000286269742900000000000000004261734E
:100D000069732D416472657373650000006C616ED8
:100D10006765204164726573736500000052656702
:100D20006973746572000000000000000050616784
:100D3000652D4D6F6465000000000000004861757E
:100D40007074676C656973000000000000733838C8
:100D50002D45696E7374656C6C756E67004B6F6EB4
:100D600066696775726174696F6E000000426F6F2B
:100D700073746572000000000000000000496E748A
:100D8000657266616365204261756400005765693C
:100D90006368656E0000000000000000004C6F6B8F
:100DA000666F726D6174000000000000004D4D2DF3
:100DB0005369676E616C20506175736500733838D4
:100DC0002D4D6F64756C65000000000000733838AD
:100DD0002D4D6F64756C746573740000004B7572F3
:100DE0007A7363686C2E2D506F6C2E00004B7572F9
:100DF0007A7363686C2E2D456D70662E00616C6C85
:100E000065205765696368656E0000000057656975
:100E10006368656E666F726D61740000006D696E67
:100E20002E20536368616C747A656974006D617813
:100E30002E20536368616C747A656974004C6F632B
:100E40006F6D6F74697665206D656E750044434300
:100E50002070726F6772616D6D696E67004C6179A9
:100E60006F7574207374617475730000005365743A
:100E700074696E67730000000000000000536F6625
:100E8000747761726520557064617465004C4344E9
:100E9000206261636B6C696768740000004D617368
:100EA000746572436F6E74726F6C000000457869F0
:100EB0007400000000000000000000000053656C9A
:100EC00065637420000000000000000000446174AD
:100ED0006120666F726D617400000000004E616DEC
:100EE00065202020202020000000000000456E74B6
:100EF00072792020202020000000000000435620AE
:100F00002862797465290000000000000043562023
:100F10002862697429000000000000000050726916
:100F20006D617279206164647265737300457874D1
:100F3000656E642E20616464726573730052656728
:100F40006973746572000000000000000050616762
:100F5000652D4D6F6465000000000000004D616963
:100F60006E20747261636B000000000000733838FB
:100F70002073657474696E67730000000044656CCB
:100F800065746500000000000000000000426F6F03
:100F900073746572000000000000000000496E7468
:100FA00065726661636520426175640000506F6917
:100FB0006E7473000000000000000000004C6F63BE
:100FC0002E20666F726D617400000000004D4D2090
:100FD0007369676E616C2070617573650073383872
:100FE000206D6F64756C6573000000000073383805
:100FF000206D6F64756C6520746573740053686F41
:10100000727420632E20706F6C2E00000053686F86
:10101000727420632E2073656E732E0000616C6CF9
:1010200020506F696E7473000000000000506F69FB
:101030006E747320666F726D61740000006D696E6E
:101040002E7377697463682E74696D65006D6178BD
:101050002E7377697463682E74696D6500202D2D79
:101060002D2D0025357500536F6674772E205600A0
:10107000312E342E33005365724E722E2025386C7B
:1010800075003A2000253575002533640025346449
:101090003A20002D2D2D0025336400204F4B2020B9
:1010A000202000202020202020200043563A20200D
:1010B0002020204269743A203D200043563A2534CE
:1010C00064204269743A25643D00202D2D2D0025B1
:1010D000346400202D2D2D2D2D0025366400202E6A
:1010E0002E2E2E202020202020202020002533649A
:1010F0002C256473002534646D7300303020426108
:10110000756400446F776E6C6F6164202E2E2E0024
:101110002564206D730020253264004E723A20252C
:10112000326420200073686F72742028312E356D70
:1011300073292000006C6F6E672028342E30323502
:101140006D732900004D6F746F726F6C6100000049
:101150000000000000444343202020202000000025
:1011600000000000004D4D200000000000000000C5
:1011700000000000004443430000000000000000A5
:101180000000000000706F73697469766520284D57
:101190004D290000006E65676174697665202844FA
:1011A0004343290000536176652020202020202021
:1011B0002020202000526573746F7265202020204B
:1011C0002020202000536176652020202020202030
:1011D0002020202000526573746F7265202020202B
:1011E0002020202000206C61796F75742073746159
:1011F0007475732000206C61796F7574207374614D
:1012000074757320004B6F72722028312E356D7308
:1012100029202000004C616E672028342E303235A2
:101220006D732900004D6F746F726F6C6100000068
:101230000000000000444343202020202000000044
:1012400000000000004D4D200000000000000000E4
:1012500000000000004443430000000000000000C4
:101260000000000000506F73697469656620284DA6
:101270004D290000004E6567617469656620284449
:1012800043432900004D6F64656C6261616E736950
:10129000742E2020004D6F64656C6261616E73690D
:1012A000742E2020004865727374656C6C656E2026
:1012B00020202020004F70736C61616E2020202060
:1012C0002020202000206865727374656C6C656E48
:1012D0002020202000206F70736C61616E20202020
:1012E0002020202000436F7572742028312E356D28
:1012F00073292000004C6F6E672028342E30323561
:101300006D732900004D6F746F726F6C6100000087
:101310000000000000444343202020202000000063
:1013200000000000004D4D20000000000000000003
:1013300000000000004443430000000000000000E3
:101340000000000000706F73697469766520284D95
:101350004D290000006E6567617469766520284438
:101360004343290000456E72656769737472656D49
:10137000656E742000526573746175726174696F73
:101380006E20202000456E72656769737472656D0A
:10139000656E742000526573746175726174696F53
:1013A0006E202020002045746174205265736561B1
:1013B000752E20200020457461742052657365618C
:1013C000752E2020004B75727A2028312E356D73D2
:1013D00029202000004C616E672028342E303235E1
:1013E0006D732900004D6F746F726F6C61000000A7
:1013F0000000000000444343202020202000000083
:1014000000000000004D4D20000000000000000022
:101410000000000000444343000000000000000002
:101420000000000000706F736974697620284D4DCC
:1014300029000000006E65676174697620284443C6
:101440004329000000416E6C6167656E7A757374A4
:10145000616E642000416E6C6167656E7A757374AD
:10146000616E6420005769656465726865727374A3
:10147000656C6C6E0053706569636865726E2020E0
:10148000202020200020776965646572686572738A
:10149000742E2020002073706569636865726E2069
:1014A0002020202000696E636F6D7061742E2046CD
:1014B0006F726D617400496E636F6D702E20466FA0
:1014C000726D6174202000466F726D617420696EC8
:1014D000636F6D7061742E00696E6B6F6D706174F7
:1014E0002E20466F726D6174002E2E2E207761695A
:1014F00074696E67202E2E2E2000233D64656C6576
:101500007465000000000000000000286E6F206578
:101510006E74727929000000000000002E2E2E202B
:1015200064656C6574696E67202E2E2E00206661DE
:10153000756C7400000000000000000000002044F2
:101540004343206F6E6C7921000000000000002AE8
:101550003D43616E63656C202020000000000000A8
:101560002070726F6772616D696E67000000000025
:10157000002D73686F727420636972637569742DCE
:1015800020002A7265616420000000000000000055
:101590000000002A777269746500000000000000F6
:1015A000000000002E2E2E2077726974696E67206D
:1015B0002E2E2E20002E2E2E2072656164696E67FD
:1015C000202E2E2E2000212121206661756C742092
:1015D00021212120202000204F4B202020202020CE
:1015E00020202020202020002E2E2E2073617669BE
:1015F0006E67202E2E2E2020002E2E2072657374F2
:101600006F72696E67202E2E2000233D44656C2E7C
:10161000202A3D43616E63656C2000233D5965734C
:10162000202A3D43616E63656C20200020636F6E4D
:1016300066696775726174696F6E2020004F464657
:1016400000000000000000000000000000002A2A46
:101650002A206E6F20547261696E202A2A2A002A7D
:101660002073686F727420636972637569742000F7
:101670002A2A2A2074696D65206F7574202A2A2A07
:1016800000506F696E7420202534642F2534640067
:101690000000436F6E66696775726174696F6E20D2
:1016A00020200020636F6E66696775726174696FD0
:1016B0006E2020002E2E2E207761636874656E20C8
:1016C0002E2E2E2000233D77697373656E00000077
:1016D000000000000000286765656E20696E766F67
:1016E00065722900000000202E2E2E20776973736A
:1016F000656E202E2E2E000020666F75740000008F
:1017000000000000000000000020416C6C65656E68
:10171000204443432100000000002A3D204166622E
:1017200072656B656E0000000000002050726F67EC
:1017300072616D6D6572656E000000002D2D4B6F3E
:101740007274736C756974696E672D2D002A4C650F
:101750007A656E00000000000000000000002A53BF
:101760006368726900000000000000000000002EA5
:101770002E2073636872696A76656E202E2E0000D3
:101780002E2E2E206C657A656E202E2E2E202000A7
:10179000002021212120466F757420212121202045
:1017A0000000204F4B20202020202020202020201F
:1017B0002000002E2E2E204F70736C61616E202E43
:1017C0002E2E00004865727374656C6C656E202067
:1017D0002020200000233D77697373656E202A3D29
:1017E000616662720000233D4A61202A3D416662C3
:1017F00072656B656E20002077697373656E2020BB
:101800002020202020202000554954000000000006
:101810000000000000000000002A2A2A20676565F9
:101820006E204C6F63202A2A2A002A2A6B6F72745A
:10183000736C756974696E672A2A002A2054696A74
:10184000646F766572736368722E2A0057697373CA
:10185000656C732534642F253464000000436F6E7B
:10186000666967202020202020202020200020439F
:101870006F6E6669672020202020202020200050E5
:10188000617469656E74657A0000000000000000F4
:10189000233D7375707072696D6572000000000001
:1018A0000076696465000000000000000000000090
:1018B00000005375707072657373696F6E0000007D
:1018C0000000002045727265757200000000000083
:1018D000000000002044434320756E697175656DFA
:1018E000656E7400002A3D4162616E646F6E202057
:1018F0000000000000002050726F6772616D6D6122
:1019000074696F6E0000002D436F7572742D6369EA
:1019100072637569742D20002A4C6563742E000073
:101920000000000000000000002A45637269740096
:10193000000000000000000000002E2E2E20456355
:10194000726974757265202E2E2E002E2E2E204C5C
:10195000656374757265202E2E2E200021212120B2
:1019600045727265757220212121202000204F4B85
:101970002020202020202020202020202000204562
:101980006E72656769737472656D656E7420002090
:10199000526573746175726174696F6E20202000E6
:1019A000233D5375707072202A3D4162616E642E32
:1019B00000233D4F7569202A3D4162616E646F6E60
:1019C0002000205375707072696D65722020202090
:1019D000202000496E616374696620202020202049
:1019E000202020002A20506173206465206C6F63E2
:1019F0006F202A20002A20436F7572742D6369724C
:101A00006375697420002A2054656D7073206465C5
:101A10007061737365200041696775696C2E2534A8
:101A2000642F253464000000456E72656769737425
:101A300072656D656E7420200052657374617572F5
:101A40006174696F6E20202020002E2E2E20776179
:101A50007274656E202E2E2E202000233D4CF673CE
:101A60006368656E0000000000000000286B656977
:101A70006E2045696E7472616729000000202E2E69
:101A80002E206CF673636865202E2E2E20002046D3
:101A900065686C6572000000000000000000002016
:101AA0006E75722066FC72204443432100000000E2
:101AB0002A203D20416262727563680000000000C8
:101AC000002050726F6772616D6D696572756E6727
:101AD00000002D2D204B75727A7363686C75DF20C2
:101AE0002D2D002A6C6573656E000000000000005B
:101AF000000000002A736368722E000000000000DE
:101B000000000000002E2E20736368726569626514
:101B10006E202E2E00002E2E2E206C6573656E20FA
:101B20002E2E2E20200000212121204665686C6584
:101B30007220212121200000204F4B202020202036
:101B40002020202020202000002E2E207370656988
:101B5000636865726E202E2E000077696564657279
:101B60006865727374656C6C656E00233D4CF6732A
:101B70006368656E202A3D4162627200233D4A61BE
:101B8000202A3D41626272756368000000206CF695
:101B9000736368656E20202020202020200041559E
:101BA0005300000000000000000000000000002AB8
:101BB0002A206B65696E65204C6F6B202A2A2000F5
:101BC0002A2A204B75727A7363686C75DF202A2A83
:101BD000002A205A656974FC626572736368722E0C
:101BE0002A00576569636865202534642F253464AD
:101BF0000000004B6F6E66696775726174696F6E85
:101C000020202000204B6F6E6669677572617469D1
:101C10006F6E2020005B6E6F206D6573736167656A
:101C20005D005B756E6B6E6F776E206572726F72A2
:101C30005D005B756E6B6E6F776E2073746174758B
:101C4000735D000011241FBECFEFD0E1DEBFCDBF1A
:101C500013E0A0E0B1E0E2E8F4EE00E00BBF02C068
:101C600007900D92AE33B107D9F71DE0AEE3B3E0B4
:101C700001C01D92AE38B107E1F70C94AB0E0C9485
:101C8000000081E080933F030895982F80913E03E8
:101C9000891731F0863021F0853029F4963019F01B
:101CA00080E090E0089590933E03892F8250823027
:101CB00058F40E94481F1092310780913E038230F1
:101CC00051F40E94F92907C0943019F40E946B1F47
:101CD00002C00E94571F80913E03863011F40E947B
:101CE000335780913E03813019F482E00E94D86B13
:101CF0004EE353E063E08FEF0E94E8570E94410EED
:101D000081E090E00895089580913E039927089519
:101D100080E00E94AB1A2FEF8F3F920719F0682FD7
:101D200080E009C081E00E94AB1A2FEF8F3F92073D
:101D300021F0682F81E00E94E6400E94FE570E9439
:101D400081690E94552E80913F03882311F40E94DF
:101D50008B19A8950895CFEFD0E1DEBFCDBF0E94CB
:101D6000F4540E948C0F0E9401260E94D1670E94A9
:101D7000991F0E94345521E04EE468E00E94B90F9B
:101D800021E04EE468E087E00E94D2110E947013C7
:101D900078940E945E150E942C55FC0184810E945B
:101DA000F41962E171E082E00E94291A0E947755DD
:101DB000813059F060E081E00E94A11862E271E098
:101DC00082E00E94291AA895FECF6EE171E082E0C0
:101DD0000E94291A60E081E00E94A11866E582E075
:101DE0000E94F91962E371E082E00E94291A0E94C0
:101DF0002C558C0181E00E947617882319F081E030
:101E00000E942F5582E00E947617882319F080E007
:101E10000E942F5583E00E947617882319F082E0F4
:101E20000E942F5584E00E947617882319F083E0E2
:101E30000E942F5580E00E94450E81E00E94D75EEF
:101E400080E00E947617882319F084E10E94C05335
:101E50000E94B86240E050E060E28FEF0E94E857D5
:101E600080E00E94CA4081E00E94CA40809133070E
:101E700090913407A0913507B0913607805D974067
:101E8000A040B04078F40E94880E80913307909172
:101E90003407A0913507B0913607805D9740A04088
:101EA000B04088F3F80181859285892BC9F00E94A2
:101EB000412AEC0146969E012F5E3F4FAC01B901CD
:101EC000F801818592850E947C61BC01892B29F0F3
:101ED000F801818592858C8B9D8B6115710519F4B4
:101EE000F801628173818FEF0E94A35681E011C0D7
:101EF0000E94702E0E943818FFEF8F3F9F07C1F796
:101F00000E94880E80913F038823A1F310923F0323
:101F100080E00E94D52BEECF8FE78ABB1BBA80E111
:101F200087BB18BA80EF84BB8FEF85BB8BEB81BB7F
:101F30008CEC82BB86E082B987EF83B98093610025
:101F400081EF809362008FE18093640089E1809348
:101F500065000E94E95E10926A001ABE8AB78A6024
:101F60008ABF0E94CF16A89588E181BD8CE081BD13
:101F70000895E82F109205078091050780930407C4
:101F80008091040780932707809127078093260775
:101F900091E0909330078C9A119A82B18E7E82B92B
:101FA000199A83B18E7E83B982E08BB99498E83018
:101FB00008F0E92FFF27EE0FFF1FE85CFE4FA59109
:101FC000B491653010F465E003C0693008F068E052
:101FD0004F7D6550660F453411F4606203C04F3485
:101FE00009F46063223008F068608B2F992787FD21
:101FF0009A958F7080939000A9B96093950088EBB3
:102000008AB980E090E00895909126078091270793
:10201000981711F00C9B559A089508951F920F92EE
:102020000FB60F9211248F939F93EF93FF9390918C
:10203000260780912707981761F088B7806188BFCD
:102040000C9B09C089B7806189BF8091300780FFF0
:1020500002C0559813C080912707E82FFF27EC5F37
:10206000F84F84A18CB9809127078F5F8093270751
:1020700080912707883010F010922707FF91EF9189
:102080009F918F910F900FBE0F901F9018951F92E8
:102090000F920FB60F9211248F9389B78F7E89BF4D
:1020A000559A8F910F900FBE0F901F9018951F9209
:1020B0000F920FB60F9211242F933F934F935F937C
:1020C0006F937F938F939F93AF93BF93EF93FF9300
:1020D00080910407282F33278091050799270197BE
:1020E0002817390741F0809104078F3179F48091E6
:1020F0000507882359F4809105078F5F80930507B2
:1021000080910507803210F0109205079BB18091F5
:102110000407E82FFF27EC5FF84F8CB18283228100
:1021200094FD0CC0809104078F5F80930407809119
:1021300004078032A8F01092040712C0222381F411
:102140002093050780910507809304079498822FB8
:102150000E94CA4021E04EE468E0822F0E94B90F3D
:1021600080910407282F332780910507281B310908
:1021700037FF02C0205E3F4F213131050CF0949AA9
:10218000FF91EF91BF91AF919F918F917F916F914F
:102190005F914F913F912F910F900FBE0F901F9025
:1021A000189550E060E070E027E0813D920708F06C
:1021B00051E02FE0813A920708F052E023E28932A1
:1021C000920708F053E026E3813B920708F054E0C1
:1021D00026E48135920708F055E028E8893B92070C
:1021E00008F056E0895D964D08F057E078948BB181
:1021F000992726E0969587952A95E1F79C0121700D
:10220000307080FFB9016F5F7F4FA89587E2603122
:10221000780768F321E04EE468E0852F0E94B90F4B
:10222000089589B1282F3327809190009927982FFE
:102230008827282B392B60E040E050E0FA01E85C69
:10224000FE4F859194918217930729F06F5F4E5F3F
:102250005F4F683098F3862F99278330910509F1F5
:10226000843091054CF481309105A9F082309105BC
:10227000ACF4892B69F024C085309105C1F085301C
:10228000910594F086309105A9F00797B1F018C038
:1022900080EB94E0089580E699E0089580EC92E167
:1022A000089580E895E2089580E498E3089580E039
:1022B0009BE4089580E096E9089580E091EE08950A
:1022C00080E090E008950895482F07C08091270787
:1022D000882391F4559A7894A89580912607282F01
:1022E000332780912707992701972817390791F3FA
:1022F00080912607873051F380912607E82FFF272A
:10230000EC5FF84F44A3809126078F5F80932607E8
:1023100080912607883010F010922607559A80E0A9
:1023200090E0089580910407282F332780910507B6
:10233000281B310937FF02C0205E3F4F2031310595
:102340000CF494989091040780910507981719F45C
:102350008FEF9FEF089580910507E82FFF27EC5F2F
:10236000F84F8281282F3327809105078F5F809354
:10237000050780910507803210F010920507C9010A
:1023800008950895882331F080913007816080930B
:1023900030070895809130078E7F80933007559ADB
:1023A00008950895E82F1092D8068091D80680935A
:1023B000D7068091D7068093FA068091FA0680931B
:1023C000F90691E09093030781B3886281BB8A98F4
:1023D0001598939A92981D9882E080939B00959807
:1023E000E83008F0E92FFF27EE0FFF1FE85CFE4FF3
:1023F000A591B491653010F465E003C0693008F030
:1024000068E04F7D6550660F8B2F992787FD9A9561
:102410008F7080939800A0939900453411F4606206
:1024200003C04F3409F46063223008F068606093A1
:102430009D0088EB80939A0080E090E00895909151
:10244000F9068091FA06981739F00D9905C0809128
:102450009A00806280939A00089508951F920F92C7
:102460000FB60F9211248F939F93EF93FF93909148
:10247000F9068091FA06981761F088B7806288BFE4
:102480000D9B0DC089B7806289BF8091030780FFD3
:1024900006C080919A008F7D80939A0014C080912D
:1024A000FA06E82FFF27E952F94F84A180939C0098
:1024B0008091FA068F5F8093FA068091FA06883041
:1024C00010F01092FA06FF91EF919F918F910F906B
:1024D0000FBE0F901F9018951F920F920FB60F927C
:1024E00011248F9389B78F7D89BF80919A00806274
:1024F00080939A008F910F900FBE0F901F901895A8
:102500001F920F920FB60F9211242F933F934F9368
:102510005F936F937F938F939F93AF93BF93EF934B
:10252000FF938091D706282F33278091D8069927CB
:1025300001972817390741F08091D7068F3179F438
:102540008091D806882359F48091D8068F5F8093B4
:10255000D8068091D806803210F01092D80690915B
:102560009B008091D706E82FFF27E952F94F809111
:102570009C008283828194FD0CC08091D7068F5F7E
:102580008093D7068091D706803278F01092D706D4
:102590000CC0882351F48093D8068091D80680938C
:1025A000D706959881E00E94CA408091D706282FCF
:1025B00033278091D806281B310937FF02C0205EDF
:1025C0003F4F213131050CF0959AFF91EF91BF916A
:1025D000AF919F918F917F916F915F914F913F91BB
:1025E0002F910F900FBE0F901F901895482F0BC082
:1025F0008091FA068823B1F480919A0080628093DA
:102600009A007894A8958091F906282F3327809115
:10261000FA06992701972817390771F38091F9066F
:10262000873031F38091F906E82FFF27E952F94FFF
:1026300044A38091F9068F5F8093F9068091F90693
:10264000883010F01092F90680919A008062809391
:102650009A0080E090E008958091D706282F3327D4
:102660008091D806281B310937FF02C0205E3F4FFA
:10267000203131050CF495989091D7068091D806B9
:10268000981719F48FEF9FEF08958091D806E82FDF
:10269000FF27E952F94F8281282F33278091D806EE
:1026A0008F5F8093D8068091D806803210F0109208
:1026B000D806C90108950895882331F08091030751
:1026C0008160809303070895809103078E7F809334
:1026D000030780919A00806280939A00089508957C
:1026E00087B3876087BBBB9888B3896088BB1DB8F8
:1026F0008EB18FB187E78DB908951F920F920FB6F3
:102700000F9211242F938F939F93EF93FF932FB1E9
:1027100080914003E82FFF27E05CFC4F22838F5F0E
:1027200080934003883110F01092400390915B0336
:10273000E92FFF27E05CFC4F248D27FDC09A809194
:102740005A03981759F0C098892F8F5F80935B03C5
:10275000883110F010925B032FB902C0C09A6F98B5
:10276000FF91EF919F918F912F910F900FBE0F903E
:102770001F90189580915B03282F332780915A036F
:10278000281B3109C90147968831910514F0C90108
:10279000019708950895282F6F9919C0C0988FB197
:1027A0006F9A80915A0390915B03891711F42FB9A6
:1027B0001CC0E92FFF27E05CFC4F848D8FB9892F67
:1027C0008F5F80935B03883110F010925B038091E0
:1027D0005A03E82FFF27E05CFC4F248F8F5F809324
:1027E0005A03883110F010925A0380E090E0089567
:1027F0008091400320914103821719F48FEF9FEFDE
:102800000895E22FFF27E05CFC4F8281482F552777
:10281000822F8F5F80934103883110F01092410323
:10282000CA01907008950895882311F0DD9A0895E3
:10283000DD9808950895CF93382FA0917703B09134
:102840007803109711F4882321F48091740388236E
:1028500061F1809174038F5F8093740399278330B3
:10286000910509F475C0843091053CF481309105DF
:1028700081F0029709F46FC018C08630910569F0A5
:10288000873091051CF4059731F00FC0079749F088
:102890000CC0DC9A60C081E001C080E00E9414148A
:1028A0005AC0DC981092740356C0DE9B4FC033238D
:1028B00009F04CC0CD0153E0969587955A95E1F704
:1028C000209177032770932FCF9991E0482F5527B8
:1028D000622F7727C091CA0A992399F0FA01E45B25
:1028E000F44F20E830E002C0359527956A95E2F76D
:1028F0008081822B8083FA01E45FF44F8081822BF8
:102900000EC0FA01E45BF44F80E890E002C09595B8
:1029100087956A95E2F7982F909580818923808327
:102920009D012F5F3F4F30937803209377038C2FC7
:10293000992744E0880F991F4A95E1F7281739072E
:1029400048F0109278031092770304C0332311F0FB
:10295000DE9A01C0DE98CF910895000000000000CB
:1029600000000895882341F0809165008460809381
:1029700065000E94AD140895809165008B7F80935F
:102980006500089508959B01AC01809133079091F3
:102990003407A0913507B091360782179307A40733
:1029A000B507A0F08091330790913407A0913507C7
:1029B000B0913607821B930BA40BB50B805090414E
:1029C000A040B040A0F080E090E0089580913307EF
:1029D00090913407A0913507B0913607281B390B29
:1029E0004A0B5B0B2050304F4F4F5F4F18F081E088
:1029F00090E0089580E090E008950895EF92FF92AE
:102A00000F931F93AA27BB27E0903307F09034075A
:102A10000091350710913607E80EF91E0A1F1B1F9B
:102A200001C0A895C801B7010E94C3148823C9F347
:102A30001F910F91FF90EF9008950F931F93CF93E5
:102A4000C82F162F042F809165008D7F809365001D
:102A500080E00E94B2148AB38F608ABB8BB3807F00
:102A60009C2F92959F70892B8BBB112321F0809115
:102A70006500816003C0809165008E7F8093650052
:102A800081E00E94B21480E00E94B214002329F079
:102A900088E090E00E94FE140DC08BB3807FCF7061
:102AA0008C2B8BBB0E94AD1481E00E94B214802F4E
:102AB0000E94B214CF911F910F91089588E290E087
:102AC0000E94FE1441E060E080E30E941D1541E099
:102AD00060E080E30E941D1541E060E080E30E9419
:102AE0001D1541E060E080E20E941D1588E20E9411
:102AF000971888E00E94971881E00E94971886E056
:102B00000E9497188CE00E9497186CE372E080E0B6
:102B10000E94D01964E172E081E00E94D0196CE15A
:102B200072E082E00E94D01964E072E083E00E94CB
:102B3000D01964EF71E084E00E94D0196CEE71E06E
:102B400085E00E94D01964EE71E086E00E94D01901
:102B50006CED71E087E00E94D01908951F920F92EA
:102B60000FB60F9211241F932F933F934F935F93B0
:102B70006F937F938F939F93AF93BF93EF93FF9345
:102B8000809175038F5F80937503282F237009F060
:102B9000F4C086958695877099278330910509F44E
:102BA0007CC0843091054CF48130910551F1823024
:102BB0009105DCF5892B89F0E0C08530910509F499
:102BC000A2C0853091050CF49CC08630910509F4B3
:102BD000CEC0079709F4CFC0D0C080913307909141
:102BE0003407A0913507B09136070196A11DB11D9C
:102BF0008093330790933407A0933507B09336073B
:102C000080C08091330790913407A0913507B0912F
:102C1000360781709070A070B070892B19F00E94F7
:102C20008917ABC00E944A17A8C081E00E941B14FC
:102C30000E94840E833009F0A0C00E94A41F20913E
:102C40003107309132078823E9F02E5F3F4F3093F0
:102C50003207209331070E942C55FC01968199235D
:102C600009F48BC08AE0989F90011124809131076C
:102C7000909132078217930708F47FC081E00E9489
:102C8000450E7BC02115310509F477C02150304035
:102C9000309332072093310770C0809176038823E8
:102CA00009F46BC08AB3807F8ABB822F0E94B21462
:102CB00080916500826080936500809165008E7FC1
:102CC000809365000000000081E00E94B21419B3F7
:102CD00080E00E94B2141295107F0E94AD1481E032
:102CE0000E94B21489B38F70182B80E00E94B21436
:102CF000812F992787FD90958827990F881F9927FD
:102D000033C0822F35C0609176036623B1F5909170
:102D1000370780913807981789F010913807E12F0D
:102D2000FF27E95CF84F82811F5F103108F0162FF2
:102D3000803891F480913707811719F480E090E092
:102D400013C0E12FFF27E95CF84F82811F5F10312C
:102D500008F0162F462F02C0462F61E00E941D1575
:102D60001093380781E090E08093760306C081E0FD
:102D70000E941B1402C00E941E18FF91EF91BF9188
:102D8000AF919F918F917F916F915F914F913F9103
:102D90002F911F910F900FBE0F901F9018951092BA
:102DA0007D0017BE11BE89E683BF87B7816087BFEC
:102DB00082EF8FBD3AE13EBD4FEC50E057BD46BDBE
:102DC00085EB90E09BBD8ABD99BD88BD22EC209328
:102DD0008B0030938A005093810040938000909341
:102DE0008700809386000E942C55FC01808580938B
:102DF000CA0A0895EF92FF920F931F93AA27BB2749
:102E0000E0903307F09034070091350710913607B2
:102E1000E80EF91E0A1F1B1F02C00E94880EC8017F
:102E2000B7010E94C3148823C1F31F910F91FF9033
:102E3000EF900895282F220F61112160822F837057
:102E40008150823028F424FF02C02E6001C0217F0F
:102E5000822F9927089590917B03E92FFF27E5584A
:102E6000FC4F8283892F8F5F80937B03883010F023
:102E700010927B0390917C0380917B03981741F41F
:102E8000892F8F5F80937C03883010F010927C0331
:102E9000089508950F931F9311B1812F8074682FA7
:102EA000809179030E941A17082F80937903107874
:102EB000612F80917A030E941A1780937A03007C15
:102EC000807C003829F4882339F0803C61F408C004
:102ED000003449F4803C11F484E103C0882319F4E0
:102EE00085E10E942B171F910F910895843118F0EE
:102EF00080E090E0089520E030E0E82FFF27EB57D6
:102F0000FC4F8081882311F021E030E0C901089551
:102F10000895FF920F931F93CF9380919E03E82F04
:102F2000FF27E756FC4F008113B31083FF248091E5
:102F30009E03E82FFF27EE0FFF1FEE0FFF1FEF0D81
:102F4000F11DE85BFE4FC49110FD42C000FF14C0AC
:102F5000C23129F481E10E947617882331F48C2F45
:102F60000E942B17C43108F054C0EC2FFF27EB57F9
:102F7000FC4F81E080834DC0C43108F04AC0EC2F83
:102F8000FF27DF01AB57BC4F9C919F5F9C93992318
:102F900011F49F5F9C93E131F105DCF1E331F10520
:102FA0006CF07397B1F580919803853690F18CE1C0
:102FB0000E942B1781E0809398032BC08091960389
:102FC000893738F180919703893718F185E01FC060
:102FD000C43128F4EC2FFF27EB57FC4F108200FD83
:102FE00018C08C2F80680E942B170E94840E853099
:102FF00081F4C13121F482E10E94761705C0C2310B
:1030000041F481E10E947617882319F486E00E943A
:10301000450E16950695F39483E08F1508F087CF3B
:1030200080919E038F5F80939E03853010F01092F5
:103030009E03CF911F910F91FF90089590919E0351
:10304000943029F485B3806F85BB97980895979A3B
:1030500085B38F7020E130E002C0220F331F9A95B4
:10306000E2F7922F9095907F892B85BB0895089564
:1030700080917B0320917C03821719F48FEF9FEFDF
:103080000895E22FFF27E558FC4F8281482F5527EE
:10309000822F8F5F80937C03883010F010927C0326
:1030A000CA0108950895CF93C82F1CC08091380796
:1030B000882339F580E00E94AB1A2FEF8F3F9207EB
:1030C00019F0682F80E009C081E00E94AB1A2FEF51
:1030D0008F3F920721F0682F81E00E94E6400E9416
:1030E000FE57A89580913707282F332780913807FE
:1030F0009927019728173907E9F2809137078F3010
:10310000A9F2F89480913707E82FFF27E95CF84F80
:10311000C283809137078F5F80933707809137078D
:10312000803110F0109237077894CF9108951F9353
:10313000182F80E80E945318812F0E9453181F9166
:1031400008958295880F880F807C860F80680E9482
:10315000971808950E94A1188EE00E94971808956C
:103160008CE00E9497180895FF920F931F93CF93BE
:10317000F82E60915A07809159070E94A118C0E06B
:1031800009E417E080915B07C81778F4FF2021F06D
:10319000F80161918F0101C060E282E00E94F9199B
:1031A000CF5F80915B07C81788F3CF911F910F9174
:1031B000FF9008959093640780936307892B89F1AA
:1031C0007093620760936107CB01AA27BB27209108
:1031D0003307309134074091350750913607280F57
:1031E000391F4A1F5B1F20935D0730935E07409392
:1031F0005F075093600780915C078E7F80935C0728
:10320000211531054105510561F42F5F3F4F4F4FA7
:103210005F4F20935D0730935E0740935F075093A5
:10322000600708950895AF92BF92CF92DF92EF9218
:10323000FF920F931F93CF93DF93D82EC62EEA01F0
:1032400089E4E82E87E0F82E109264071092630755
:1032500081E08D1568F1EFE0E61750F14115510559
:1032600039F1FA0101900020E9F731970E2F041B84
:10327000013108F000E16C2D8D2D0E94A11857013D
:10328000002361F0102F8881F50181935F018991FE
:10329000682F82E00E94F9191150A9F7F701D08A2E
:1032A000C18A028B64EF71E084EB98E10E94DA1826
:1032B000DF91CF911F910F91FF90EF90DF90CF9012
:1032C000BF90AF900895CF93DF93CDB7DEB7A097AF
:1032D0000FB6F894DEBF0FBECDBF282FDE011196CA
:1032E00090E0FA014F5F5F4F8491882321F08D9326
:1032F0009F5F9F31B0F31C92AE014F5F5F4F822FF3
:103300000E941319A0960FB6F894DEBF0FBECDBF72
:10331000DF91CF9108958091630790916407892B85
:10332000A9F160915D0770915E0780915F079091B0
:1033300060070E94C314882349F180915C07E091E3
:103340006307F09164078170099580915C0791E0B3
:10335000892780935C0780916107909162079C01A7
:10336000442755278091330790913407A091350762
:10337000B0913607820F931FA41FB51F80935D077E
:1033800090935E07A0935F07B09360070895089538
:10339000109264071092630781E00E9497180895C5
:1033A0000F931F93CF93DF93EB018830C0F49927DD
:1033B00023E0880F991F2A95E1F780640E949718EF
:1033C00007E010E0FE01219684910E9453180150FD
:1033D000104017FFF7CF60E0862F0E94A118DF9101
:1033E000CF911F910F910895813308F080E381BF41
:1033F000089599278130910539F1823091051CF4A7
:10340000892BF1F00895029711F567FF15C0643E0E
:1034100031F0663F41F06C3F51F0643C11F461EED5
:103420000BC0663D11F46FEE07C06C3D11F465EF03
:1034300003C06F3D09F462EE862F0E945318089571
:10344000862F0E9464110895862F0E94F612089517
:1034500008951F93CF93DF93182FEB01FB01649125
:10346000662349F0812F0E94F9192196FE0184916B
:10347000682F8823B9F7DF91CF911F9108951F938B
:10348000CF93DF93182FEB018881882341F0899136
:10349000682F812F0E94F91988818823C1F7DF9155
:1034A000CF911F9108951F93CF93DF93CDB7DEB7D0
:1034B000C055D0400FB6F894DEBF0FBECDBF6796A3
:1034C0001FAD679769968EAD9FAD6997AE01475A5C
:1034D0005F4FBC01CE0101960E94EB70BE016F5F91
:1034E0007F4F812F0E943F1AC05BDF4F0FB6F894C9
:1034F000DEBF0FBECDBFDF91CF911F9108951F9307
:10350000CF93DF93CDB7DEB7C055D0400FB6F89458
:10351000DEBF0FBECDBF67961FAD679769968EADB4
:103520009FAD6997AE01475A5F4FBC01CE0101962E
:103530000E941471BE016F5F7F4F812F0E943F1A5E
:10354000C05BDF4F0FB6F894DEBF0FBECDBFDF917B
:10355000CF911F91089599278130910571F08230A4
:1035600091051CF4892B31F00BC0029749F40E949D
:10357000381808950E94921108950E942C130895FE
:103580008FEF9FEF08950895FC018F3F910519F08B
:1035900010F0E0E0F0E0E45AFD4F8491992708959F
:1035A00090E08F3010F08EE001C081118F5F4423D6
:1035B00011F028E001C0242F77276230710581F0D7
:1035C0006330710524F46130710541F00EC0633041
:1035D000710541F06430710539F007C0236005C002
:1035E000246003C0266001C02760281729F4442303
:1035F00011F02AE001C025E043E050E0990F990F57
:1036000080FD926020FD9160869526954150504046
:1036100057FFF4CF892F99270895982F21E080E054
:1036200067FD282F6F706F3010F061E002C06111EC
:103630006F5F913061F423E030E0880F880F60FD08
:10364000836066952150304037FFF7CF1BC022239F
:1036500031F0683010F045E007C04DE005C068303B
:1036600010F44AE001C042E023E030E0880F880F08
:1036700060FD826040FD8160669546952150304036
:1036800037FFF4CF992708959C01FB018F379105EF
:1036900028F48F77808388E090E00895832F99271E
:1036A000806C8183208380E190E008950895FC017F
:1036B0004081242F332781819927019728173907C3
:1036C00029F04F3031F48181882319F481E090E0B2
:1036D000089580E090E0089508951F9385E697E0AF
:1036E0000E94571B182F87ED97E00E94571B182B3D
:1036F000812F99271F910895AF92BF92CF92DF92A9
:10370000EF920F931F93CF93DF93EC016B015A015C
:10371000122F8091D203882369F40C3059F00D30B8
:1037200049F0CB010E949927992783709070892BCB
:1037300009F48BC08091D2038823A9F5013099F553
:103740008981282F3327888199272817390759F12C
:10375000AC01F901A3E0EE0FFF1FAA95E1F7E21B10
:10376000F30BEC0FFD1F828193818C159D0589F46D
:10377000848195818A159B0561F48681813049F4A5
:103780008085882331F08E1509F45FC0E0861783A9
:103790005CC02F5F3F4F2031310514F020E030E056
:1037A00024173507B1F6CE010E94571B282F882316
:1037B00019F080E090E04BC088819927FC0173E00C
:1037C000EE0FFF1F7A95E1F7E81BF90BEC0FFD1FD9
:1037D000C282D38288819927FC0163E0EE0FFF1F2C
:1037E0006A95E1F7E81BF90BEC0FFD1FA482B58287
:1037F00088819927FC0153E0EE0FFF1F5A95E1F7EE
:10380000E81BF90BEC0FFD1F178388819927FC013A
:1038100043E0EE0FFF1F4A95E1F7E81BF90BEC0FB1
:10382000FD1F068388819927FC0133E0EE0FFF1FFF
:103830003A95E1F7E81BF90BEC0FFD1FE086888154
:103840008F5F8883803108F0288381E090E0DF91EA
:10385000CF911F910F91EF90DF90CF90BF90AF90DD
:1038600008959F92AF92BF92CF92DF92EF92FF9214
:103870000F931F93CF93DF93EC015B016A01922EAC
:10388000F02E1E2D892B31F487ED97E00E94311C1C
:10389000C5E6D7E08091D203882321F087E0C73DB9
:1038A000D807C1F00E94840E8250833098F4F894B7
:1038B000E12E0F2D292DA601B501CE010E947C1B02
:1038C0007894882329F485E090E00E94FE14EACFE2
:1038D0001092D503DF91CF911F910F91FF90EF9040
:1038E000DF90CF90BF90AF909F900895CF92DF92DE
:1038F000EF920F93CF93DF936C01E62E0E9449263F
:10390000EC01892BE9F088859927837090700397E3
:1039100011F423E001C026E001E040E050E0B601F0
:1039200085E697E00E94311C8885833049F4EE24B7
:103930000FE021E040E050E0BA01CA010E94311CD2
:1039400081E090E0DF91CF910F91EF90DF90CF90E9
:103950000895EF920F93CF93DF93EC01E62E0E9430
:103960004926892B49F006E126E040E050E0BE01FF
:1039700085E697E00E94311C81E090E0DF91CF91D5
:103980000F91EF900895EF920F93CF93DF93EC0197
:103990000E944926FC01892BA9F080858370815003
:1039A0009681823028F49078E92E03E02BE004C061
:1039B0009078E92E03E024E040E050E0BE01CA0127
:1039C0000E94311C81E090E0DF91CF910F91EF9048
:1039D0000895EF920F93CF93DF93EC010E94492655
:1039E000FC01892B19F18085282F33272370307033
:1039F00021303105DCF0233031057CF023303105F6
:103A0000A9F40E94382A0E9789F4EE240FE021E0F1
:103A100040E050E0BA01CA0107C0EE2402E027E00E
:103A200040E050E0BE01CA010E94311C81E090E0FC
:103A3000DF91CF910F91EF900895EF920F93CF9375
:103A4000DF93EC010E944926FC01892B79F08085E7
:103A5000992783709070019749F4EE240BE024E0DD
:103A600040E050E0BE01CA010E94311C81E090E0BC
:103A7000DF91CF910F91EF900895AF92BF92CF92C7
:103A8000DF92EF920F93CF93DF935C016B010E9463
:103A90004926EC01892B09F450C088859927837049
:103AA00090708230910569F5D7FE05C06E818881DE
:103AB00099810E94761CC0FE09C0EE8007E024E0D8
:103AC00040E050E0B501CA010E94311CC1FE09C0AE
:103AD000EE8008E024E040E050E0B501CA010E9419
:103AE000311CC2FE09C0EE8009E024E040E050E055
:103AF000B501CA010E94311CC3FE1FC0EE800AE05E
:103B000015C00397D1F4C6018F709078892B49F0C6
:103B1000EE2404E0202F40E050E0B501CA010E94ED
:103B2000311C8C2D807F49F0EE2405E024E040E03C
:103B300050E0B501CA010E94311C81E090E0DF91A4
:103B4000CF910F91EF90DF90CF90BF90AF900895FD
:103B5000EF920F931F93CF93DF93EC01162F0E94E8
:103B6000992783708150823050F4EE2402E0212F97
:103B700040E050E0BE0185E697E00E94311C81E004
:103B800090E0DF91CF911F910F91EF900895EF9208
:103B90000F93E62E662319F0EE240DE001C00CE031
:103BA00023E040E050E0BC01CA010E94311C81E0EA
:103BB00090E00F91EF900895EF920F93262FEE244F
:103BC0000EE040E050E0BC01CA010E94311C81E0DF
:103BD00090E00F91EF900895EF920F93EE240FE095
:103BE000282F40E050E0BA01CA010E94311C81E058
:103BF00090E00F91EF900895EF920F93FC01809168
:103C0000D203882319F480E090E013C06770862FF8
:103C1000806F442311F0862F886FE82E02E121E0A7
:103C200040E050E0BF0185E697E00E94311C81E052
:103C300090E00F91EF900895EF920F93FC01809127
:103C4000D203882319F480E090E013C06770862FB8
:103C5000806E442311F0862F886EE82E02E121E069
:103C600040E050E0BF0185E697E00E94311C81E012
:103C700090E00F91EF900895EF920F93FC01E62EE4
:103C80008091D203882319F480E090E00BC003E117
:103C900021E040E050E0BF0185E697E00E94311C42
:103CA00081E090E00F91EF900895EF920F93FC0167
:103CB000E62E8091D203882319F480E090E00BC0B7
:103CC00004E121E040E050E0BF0185E697E00E947A
:103CD000311C81E090E00F91EF900895EF920F93E7
:103CE000FC01E62E8091D203882319F480E090E055
:103CF0000BC000E121E040E050E0BF0185E697E025
:103D00000E94311C81E090E00F91EF900895EF92B6
:103D10000F93FC01E62E8091D203882319F480E0F2
:103D200090E00BC001E121E040E050E0BF0185E6FA
:103D300097E00E94311C81E090E00F91EF90089590
:103D4000EF920F93FC01E42E05E124E0AB01BF01EB
:103D500080E090E00E94311C81E090E00F91EF90B4
:103D60000895982F882391F0109266078091660736
:103D70008093650781E08093D4038091D40380937E
:103D8000D203BD9A87B7846087BF089587B78B7FBA
:103D900087BF9093D203BD98C59808950895EF9278
:103DA0000F93E090D203EE2069F5882359F1E09259
:103DB0006607809166078093650788E1E2EAF3E091
:103DC00011928A95E9F70FE022E040E050E0BA0155
:103DD00085E697E00E94311C81E08093D4038BE359
:103DE00090E099BD88BD88B599B59BBD8ABD87E730
:103DF00090E097BD86BD1DBC1CBC87B7846087BFA3
:103E0000BE9A05C0BE98C69887B78B7F87BF0F91B3
:103E1000EF900895EF920F93E090D203EE2071F5AA
:103E2000882361F1E092D8078091D8078093D70763
:103E300088E1EAEBF3E011928A95E9F70FE022E0DE
:103E400040E050E0BA0187ED97E00E94311C8BE31F
:103E500090E0909387008093860087E790E09093AE
:103E600081008093800010928900109288008091D8
:103E70007D00846080937D00139A07C013981B987F
:103E800080917D008B7F80937D000F91EF9008954E
:103E900080E00E94B11E81E00E94CF1E81E00E945E
:103EA0000A1F80916200846080936200089580E020
:103EB0000E94B11E809162008B7F8093620080E03F
:103EC0000E94CF1E80E00E940A1F1092D40381E05E
:103ED0000E94D86B089580E00E94CF1E80E00E946F
:103EE0000A1F81E00E94D86B809162008B7F8093D3
:103EF000620088E1E2EAF3E011928A95E9F783E053
:103F00008093B4038FEF8093A2038BE390E099BD7D
:103F100088BD88B599B59BBD8ABD87E790E097BD00
:103F200086BD81E00E94B11E82E090E00E94FA16F8
:103F300008950E942C55FC01808182FF02C0C79A1F
:103F40000895C798089508950E942C55FC0180811A
:103F500082FF07C080E090E0B79907C081E090E061
:103F6000089586B3992780789070089508950E94E7
:103F7000840E833021F00E94840E843021F48091DD
:103F8000D5039927089581E090E0089508958091E0
:103F9000D303992708951092D30308959093EA03C9
:103FA0008093E90308958091E7039091E8030895D1
:103FB00080E1E6EDF3E011928A95E9F71092E603CD
:103FC0001092E8031092E7038FEF9FE79093EA03C4
:103FD0008093E903089578941F920F920FB60F9281
:103FE00011242F933F934F938F939F93EF93FF93BE
:103FF0008091E603883010F01092E6038091E6038A
:10400000E82FFF27EE0FFF1FEA52FC4F24B135B116
:10401000208331838F5F8093E6031092E803109230
:10402000E70320E030E047E0E6EDF3E08191919195
:10403000280F391F415047FFF9CF3093E8032093F1
:10404000E7038091E9039091EA03821793071CF438
:1040500081E08093D303FF91EF919F918F914F91D6
:104060003F912F910F900FBE0F901F9018955F9268
:104070006F927F928F929F92AF92BF92CF92DF9278
:10408000EF92FF920F931F93CF93DF93EC015B01AD
:104090005524675D774011F441E0542EF50190817D
:1040A0008181981709F08AC0552019F481E0809326
:1040B000D5038091D203882339F0EE240EE021E06D
:1040C00040E050E0BA0177C0552019F00E947F27E8
:1040D00002C00E9424276C01009731F4EE2401E015
:1040E00022E0AC01BC0167C0FC0180859927837088
:1040F00090708230910581F0833091051CF4019716
:1041000021F05CC00397D1F159C0F601E68001E0CF
:1041100022E040E050E04DC0F6011681E12E01E0C2
:1041200022E040E050E060817181C5010E947C1B6B
:104130000E9420278370482F55274130510591F068
:104140004230510524F44115510541F037C0423049
:10415000510559F04330510571F030C0E12E07E0B0
:1041600022E026C0E12E08E002C0E12E09E022E0B4
:1041700040E050E01DC0E12E0AE0F9CFF601E680F4
:1041800001E0202F40E050E060817181C5010E9474
:104190007C1B0E9420279927AC014170507080FF42
:1041A00004C0EE2404E021E0E3CFEE2405E021E0AA
:1041B000F60160817181C5010E947C1BF50181813E
:1041C0009927FC0133E0EE0FFF1F3A95E1F7E81B5A
:1041D000F90BEA0DFB1DE280F380F501818199273F
:1041E000FC0123E0EE0FFF1F2A95E1F7E81BF90B16
:1041F000EA0DFB1D64807580F50181819927FC0122
:1042000003E0EE0FFF1F0A95E1F7E81BF90BEA0D3B
:10421000FB1D9680F50181819927FC0113E0EE0FCB
:10422000FF1F1A95E1F7E81BF90BEA0DFB1D8084CF
:10423000F50181819927FC01B3E0EE0FFF1FBA95CC
:10424000E1F7E81BF90BEA0DFB1D278121502783BD
:104250002223B1F4F50181819927FC01A3E0EE0F3F
:10426000FF1FAA95E1F7E81BF90BEA0DFB1D26835A
:10427000F50181818F5F81838181803108F0218305
:10428000892D8C50823038F4C7010E944A6A082F69
:10429000CC24DD2407C01091D203112329F0CC24B3
:1042A000DD2403E010E012C0C7010E9449266C0122
:1042B000009729F0182DFC010085037005C001E06E
:1042C000FFE09F1609F403E051101078802F992722
:1042D000813091050CF427C28330910524F00397B7
:1042E00009F4DEC020C2C7010E94C41A982F82952B
:1042F0008695869583708A83292F220F220F298322
:1043000071E0B72EBA8A82E1888B82E0898BC11472
:10431000D10449F1F6018481958197FF02C02360A1
:104320002983812F99278F779070892BE1F0F601EF
:1043300080850E94382A0F97B4F01F5FF6018085B0
:104340000E940F26892B29F410FF03C089818B2539
:104350008983212F2078812F99278F7190709595CF
:104360008795122F182B892D99278830910509F4EC
:1043700067C0893091059CF48430910544F4823003
:1043800091050CF04BC0019709F443C0CCC18430B7
:10439000910509F43EC0079709F44CC0C4C18B30A5
:1043A000910509F463C08C30910544F4893091057E
:1043B00009F450C00A9709F453C0B5C18E30910575
:1043C0001CF0469731F1AFC1C70153E09695879530
:1043D0005A95E1F7907001960E94C41A982F829521
:1043E0008695869583708A83990F990F9983FCE04F
:1043F0009F1611F418820AC087E0E822FF24E4E542
:10440000F2E0EE0EFF1EF7018491888382E08A8B32
:104410000EC0612F802F0E940D1B40C0F6018681C7
:1044200080788F60682F802F0E940D1B888384E026
:10443000898B79C1F60184818170482F61E005C0C4
:10444000F60184818270482F62E0812F8F770E946D
:10445000D01A24C0F60184818470482F63E0F5CF20
:10446000F60184818870482F64E0EFCFC7010E9475
:10447000C41A982F82958695869583708A83990FA2
:10448000990F9360998382E08A8BF60184819581EC
:104490008F7090708C5B9D4FFC018491888343C129
:1044A00083E08A8B01E0098B88E1888B892D99272D
:1044B0008E309105D4F48C30910574F584309105DB
:1044C00009F4ACC08530910544F48130910509F4BC
:1044D00049C0039709F445C018C18530910509F416
:1044E000B3C0069709F4BDC010C18331910564F4CF
:1044F000803191050CF0CFC08E30910509F4BCC01D
:104500000F9709F4C3C001C1853191050CF4DEC0D9
:10451000459709F4EBC0F9C088E090E0E80EF91E79
:10452000C70143E0969587954A95E1F78F738068B8
:104530008A83C7018095909535E0969587953A9541
:10454000E1F7282F207720688E2D8770282B29836C
:104550009DE0991611F42860298389818027898339
:10456000D4C01F67F601808599278C7090700897DA
:10457000B9F48FE38A83812F99278F779070009702
:1045800031F08F37910511F4117801C01F5F198345
:10459000CE010396BC01C7010E94441B885EB4C0D3
:1045A00017FF02C080E601C080E48983F6018085A0
:1045B0000E94382A212F3327BE016E5F7F4F0F974D
:1045C000B4F0C9018F779070009731F08F37910563
:1045D00011F412E001C01D5F812F86958F709981C3
:1045E000982B998310FF2BC09061998328C0C90133
:1045F0008F779070009731F08F37910511F411E0AB
:1046000001C01F5F1F702981212B2983F60184813E
:10461000958197FF14C02061298311C080E88983A8
:10462000F60124812F70822F80688983848195818F
:1046300097FF02C020692983CE010296BC01C70101
:104640000E94441B805F60C080EA8983F6018481F8
:10465000958124E0969587952A95E1F78F70806B78
:1046600009C080EA8983F60184819581892F992781
:104670008F70806A8983E0CF1982CE010296BC01D7
:10468000C7010E94441B805F888B03C08FEF8A8321
:104690001982098B3AC0F2E19F1611F488E709C02C
:1046A00081E1981611F484E704C090E1991611F4A1
:1046B0008CE78B838F2D9927982F93708B81892B73
:1046C0008B83EA82898280E2888B0DC080E78A83AF
:1046D000E3E19E1611F488E78A838E2D87709A8114
:1046E000982B9A8389828AE0898B0FC0872D99271E
:1046F00083708C6E8B836A828982CE010496BC01A2
:10470000C7010E94441B805E888B20E098899695A3
:1047100096959695915031F0FE01E90FF11D80813B
:104720002827F8CF28838A89833011F01092D40388
:10473000DF91CF911F910F91FF90EF90DF90CF907D
:10474000BF90AF909F908F907F906F905F900895F3
:10475000CF93DF93DC01FC018489882319F4258938
:10476000222361F021E0882321F08150FD01848B18
:1047700021C0FD0185898150858B1CC0FD01828986
:10478000833019F487898823A9F4FD019389892F3F
:10479000869586958695E80FF11D8081282F332711
:1047A000892F99278770907002C0359527958A9533
:1047B000E2F72170FD013289832F9927823091051C
:1047C00031F083309105CCF0039721F016C0CBE691
:1047D000D0E015C0222319F0C7E7D0E002C0CEEC2C
:1047E000D0E0FD018389882351F48689882339F438
:1047F00082E0858B81E0868B2BC0C7EDD0E0FD0188
:104800008389882329F58589882311F5818988235F
:1048100099F48091D4038823D9F48091D20388231A
:10482000B9F481E00E944D55882319F0C35BDF4E37
:104830000FC0CD5ED94F0CC0832F992781309105D1
:1048400029F0029729F4C857DD4F02C0C05FDA4F44
:10485000CE01DF91CF910895DC01FC01848988238A
:1048600019F48589882311F021E02BC0FD013389DB
:10487000932F9150938B8289833069F42789222367
:1048800051F4892F992787709070079721F481E060
:10489000878B338B16C0FD01178A9389892F8695E4
:1048A00086958695E80FF11D8081282F3327892F63
:1048B00099278770907002C0359527958A95E2F701
:1048C0002170FD01828999278230910549F083305A
:1048D00091051CF4019761F01BC0039789F018C083
:1048E000222319F08CE590E0089580E190E008958E
:1048F000222319F08EEB90E008958CE190E008956A
:10490000222319F08BE390E0089587E690E0089564
:104910008BE390E008950895FC018089838B818961
:10492000823010F482E0818B828999278130910551
:10493000B4F0833091051CF0039761F010C081E062
:104940000E944D55882319F08DE490E1089583E18C
:1049500096E0089580E1848B82E390E0089582E3FD
:1049600090E0089508951F920F920FB60F921124B0
:104970001F932F933F934F935F936F937F938F93E7
:104980009F93AF93BF93CF93DF93EF93FF93809168
:10499000D203882331F00E94C71F882311F01092A0
:1049A000B3038091A0038823A1F08091D4038823CE
:1049B00029F08BE390E099BD88BD02C019BC18BCFA
:1049C0008BE390E09BBD8ABD87E790E097BD86BDF5
:1049D0005EC0C2EAD3E0CE010E94A823AC019C01D4
:1049E000255030408CB59DB58217930718F457BDFC
:1049F00046BD0EC08CB59DB5C29697BD86BDCE0195
:104A00000E948C242CB53DB5280F391F37BD26BD1B
:104A10008091B503882381F51091B703112361F5C7
:104A20008091B303882381F481E08093A00386B74B
:104A3000846086BF789465E677E082EA93E00E941E
:104A40003720F8941092A0038091B3038150898B92
:104A50008091B2038B8B8091B403833049F48091B1
:104A6000D203882311F084E101C080E18C8B01C066
:104A70001C8B1D8A1F8A1E8A82EA93E00E942C24C6
:104A800099279BBD8ABD8AB59BB599BD88BDFF910D
:104A9000EF91DF91CF91BF91AF919F918F917F91D6
:104AA0006F915F914F913F912F911F910F900FBE8A
:104AB0000F901F9018951F920F920FB60F9211240E
:104AC0001F932F933F934F935F936F937F938F9396
:104AD0009F93AF93BF93CF93DF93EF93FF93809117
:104AE000A1038823B1F08091D403882339F08BE3AC
:104AF00090E0909387008093860004C01092870016
:104B00001092860087E790E0909381008093800068
:104B100064C0CAEBD3E0CE010E94A823AC019C0183
:104B2000255030408091880090918900821793072A
:104B300028F4509381004093800016C08091880033
:104B400090918900C2969093810080938000CE015D
:104B50000E948C242091880030918900280F391FF1
:104B600030938100209380008091CD03882361F5EC
:104B70001091CF03112341F58091CB03882391F449
:104B800081E08093A10380917C00846080937C000D
:104B9000789467ED77E08AEB93E00E943720F894F1
:104BA0001092A1038091CB038150898B8091CA031D
:104BB0008B8B8091CC03833019F480E18C8B01C006
:104BC0001C8B1D8A1F8A1E8A8AEB93E00E942C246C
:104BD00099279093870080938600FF91EF91DF9152
:104BE000CF91BF91AF919F918F917F916F915F9185
:104BF0004F913F912F911F910F900FBE0F901F90DB
:104C0000189580E892E0E9E4F8E011920197E9F75D
:104C10001092EC031092EB031092C90A08958F7062
:104C200020E030E08550823010F421E030E0C9010E
:104C300008950F931F93CF93DF93CDB7DEB72497DB
:104C40000FB6F894DEBF0FBECDBF8FEF9FEFAFEF73
:104C5000BFEF89839A83AB83BC8300E210E044E01A
:104C600050E0B801CE0101960E945F6C0E94880E50
:104C70000C5F1F4F8FE00C3D180788F324960FB68A
:104C8000F894DEBF0FBECDBFDF91CF911F910F9182
:104C900008959C01009741F408958AE0A89FC001FF
:104CA0001124875B974F0895A0E0B091C90AAB1714
:104CB000A0F440E050E0BA01FA01E60FF71FE75B0D
:104CC000F74F808191818217930739F3AF5F6F5F50
:104CD0007F4F475F5F4FAB1778F380E090E0089518
:104CE0000895BF92CF92DF92EF92FF920F931F939E
:104CF000CF93DF93CDB7DEB723970FB6F894DEBF1F
:104D00000FBECDBF6C01B62E7C010894E108F108FE
:104D10008FEFE81687E2F806A0F5C6010E94492643
:104D20008C01892B09F077C02091C90A203450F4F6
:104D30008AE0289F80011124075B174F2F5F209383
:104D4000C90A22C009E418E0B80120E030E0A90156
:104D5000AFE3F901E40FF51FE75BF74F9185F80129
:104D60008185891708F48B01A1504F5F5F4F275F42
:104D70003F4F665F7F4FA7FFECCFF8018185882307
:104D800019F480E090E048C0F801C082D182FFEFC2
:104D9000EF16F7E2FF06E0F480E2E82EF12CA8958A
:104DA00043E050E0B701CE0101960E94436C298197
:104DB0003A81F8018081918128173907C9F084E090
:104DC00090E0E80EF91E9CEDE9169FE0F90638F335
:104DD000F801808191818F3F910519F010F083E0F7
:104DE0000BC088E00E944D55882321F083E003C06A
:104DF0008B8101C082E0F801808780E8F80186831A
:104E0000148215821282138211861782BB2019F038
:104E1000C6010E948963C80123960FB6F894DEBFCD
:104E20000FBECDBFDF91CF911F910F91FF90EF90FB
:104E3000DF90CF90BF90089561E00E9471260895A1
:104E40008091ED0399270895EF92FF921F93CF93DE
:104E5000DF939091C90A992319F480E090E049C04A
:104E60008091EB038F5F8093EB03891738F080917B
:104E7000ED038F5F8093ED031092EB039091EB03B2
:104E80008AE0989FE0011124C75BD74F8091ED0322
:104E9000992787709070892BA9F41E81E12EFF2439
:104EA000C7018F779070892B69F088850E940F2643
:104EB000892B41F0E0FC06C01F5F612F888199813A
:104EC0000E94A91C8091ED03992787709070049728
:104ED00051F48885992783709070019721F4888117
:104EE00099810E941D1D89858F3F11F08F5F8987F1
:104EF000CE01DF91CF911F91FF90EF900895909197
:104F0000C90A992319F480E090E008958091EC0398
:104F10008F5F8093EC03891710F01092EC0390914F
:104F2000EC038AE0989FC0011124875B974F089596
:104F300008950E944926FC01009709F40895808590
:104F40009927089508950E944926FC01009709F4C5
:104F5000089586819927089508950E944926FC01A5
:104F6000009709F408958481958108950895BF926A
:104F7000CF92DF92EF92FF920F931F93CF93DF9325
:104F8000CDB7DEB723970FB6F894DEBF0FBECDBF07
:104F90007C01B62E0E941C27FC01892BB1F1808573
:104FA0008B1599F1B08611869FEFC92ED92E00E29C
:104FB00010E0A89543E050E0B801CE0101960E94B0
:104FC000436C89819A818E159F0511F468010DC08B
:104FD000D7FE05C028E28030920708F068010C5F18
:104FE0001F4F2FE00C3D120720F38E159F0511F087
:104FF000D7FC0BC0BB82E982FA82A89544E050E05E
:10500000B601CE0101960E945F6C23960FB6F8940C
:10501000DEBF0FBECDBFDF91CF911F910F91FF90EB
:10502000EF90DF90CF90BF900895CF92DF92FF92E4
:105030000F931F93CF93DF93EC01F62E142F892B40
:1050400009F480C088850E94382A482F5885752F1A
:1050500073708F2D99278F779070242F33272817FF
:1050600039071CF420E8F222F42A6E816F1509F446
:1050700069C01986112319F08F8181608F838F2D6C
:10508000992780789070C62EDD24960120783070A4
:105090008217930799F1C6018F779070009711F0EE
:1050A00020E8F2227330D9F4892B29F08881998184
:1050B0000E94C31C1FC0852F99278C709070089781
:1050C000C9F48F2D99278F779070892B99F48F2DA4
:1050D0008160682F888199810E94761C0BC0892B82
:1050E00049F0888199810E94761C888199810E946B
:1050F000C31C04C0888199810E94E91CFE820F2D87
:105100001127C8018F779070892BB9F088850E948C
:105110000F26892B91F000FD03C08F2D8F5F08C0F3
:105120000894C108D1080C151D0539F48F2D815044
:10513000682F888199810E94A91C6F2D888199818F
:105140000E94761CDF91CF911F910F91FF90DF900D
:10515000CF900895FF920F931F93CF93DF93EC01AD
:10516000162FF42E0E94840E833009F01078CE01A1
:105170000E941C27EC010E814F2D612F0E941528E3
:105180008A819B810097C9F060E00E947126EC0142
:10519000892B99F08E81282F332720783070802F2B
:1051A0009927807890702817390711F080E8182720
:1051B0004F2D612FCE010E941528DF91CF911F91B5
:1051C0000F91FF900895EF92FF920F931F93CF934B
:1051D000DF93EC017B01892BE1F10C811D81061726
:1051E0001707B9F11986442319F08F8181608F83E5
:1051F000EC82FD82888599278370907081309105BB
:1052000031F0813091052CF104971CF51BC09801F9
:1052100020703078C701807090782817390729F0FE
:105220006E81888199810E94761C0F7010708FE0CA
:10523000E822FF240E151F0561F0888199810E94E4
:105240001D1D07C00E251F25B801888199810E9468
:105250003D1DDF91CF911F910F91FF90EF90089529
:10526000FF920F931F93CF93DF938B01F42E0E9435
:105270001C27EC01892B49F18A819B81892B01F143
:10528000C8018F709F7B4F2DBC01CE010E94E32887
:105290008A819B810E941C27EC01892BB1F0C801F7
:1052A00080709074880F991F007F107024E016950D
:1052B00007952A95E1F7802B912B4F2DBC0102C059
:1052C0004F2DB801CE010E94E328DF91CF911F91AD
:1052D0000F91FF900895EF92FF920F931F93CF933A
:1052E000DF938C017B0160E00E947126EC01892B29
:1052F00081F060E0C7010E947126FC01892B49F012
:10530000EA82FB821986028313831186C8010E94F8
:105310000364DF91CF911F910F91FF90EF9008955B
:10532000CF93DF93EC010E94BD64209769F0CE011A
:105330000E941C27FC01892B39F0C281D381128283
:1053400013821186209799F7DF91CF9108951F93CB
:10535000CF93DF93C9E4D8E01FE38A819B81892B37
:1053600021F0888199810E94902911502A9617FF77
:10537000F4CFDF91CF911F910895EF92FF920F9399
:105380001F93CF93DF93CDB7DEB726970FB6F89470
:10539000DEBF0FBECDBF7C010E9449268C01892B48
:1053A000D9F0B701CE0101960E946557F8014481FA
:1053B00055816681CE0101960E944857AE014F5F2C
:1053C0005F4F6AE08FEF0E94E857F80144815581F2
:1053D0006681C7010E94A92A26960FB6F894DEBFFF
:1053E0000FBECDBFDF91CF911F910F91FF90EF9036
:1053F00008951F93CF93DF9310E0C9E4D8E0909114
:10540000C90A1917F0F48985899FC00111248035D4
:10541000910534F08E8199278F779070892B59F000
:105420008E8180788E83888199810E94C31C8881B7
:1054300099810E94BD291F5F2A969091C90A191768
:1054400010F3DF91CF911F9108950F931F938C015B
:10545000C8010E94A01E84E00E94EC1D61E0C8010A
:105460000E94DC1D8AE00E94EC1D1F910F9108959F
:10547000E82FFF27EF70F070E455FC4F84919927D7
:1054800008958EEE93E008958091FE0382FF05C09B
:105490008091F0039091F10308958091EE03909133
:1054A000EF03089508958091FE0382608093FE03C8
:1054B00008950F931F93CF93DF93CEEED3E08091A7
:1054C000FE0399278C010170107080FF03C080E0FB
:1054D00090E021C06091F6037091F7038091F8038A
:1054E0009091F903611571058105910531F00E94D4
:1054F000C314882311F4C8010EC01A821B821C8AAF
:105500001D8A1092EF031092EE03188A1E8A0E94E1
:10551000410E81E090E0DF91CF911F910F910895AE
:105520009C018091F0039091F103892B11F4C90142
:1055300008952F703F7B77FD3064CB018F709070A2
:1055400044E0880F991F4A95E1F7822B932B089529
:105550000895FC018091EE039091EF032091F003F8
:105560003091F103E817F907F9F460930004232B55
:10557000B1F08091F4039091F503F4E0969587954E
:10558000FA95E1F7BC016F707070892F99278695A5
:10559000869580FD7068CA010E94902A0FC05093C2
:1055A000F5034093F4030EC0E217F30769F4BA0160
:1055B0008091F4039091F5030E94902A9093F50353
:1055C0008093F4030E94410E089508959C01892B55
:1055D00069F41092FE031092F6031092F7031092F2
:1055E000F8031092F9030E94592A08956093000469
:1055F0005093F5034093F40380913307909134075F
:10560000A0913507B091360788519C4FAF4FBF4FDF
:1056100081608093F6039093F703A093F803B0930F
:10562000F9038091FE0382FF10C081608B7F80931D
:10563000FE033093F1032093F003B9018091EE0350
:105640009091EF030E946B2907C08E7F8093FE0329
:105650003093EF032093EE030E94410E08950895C6
:105660002091FE032B7F21602093FE039093F10392
:105670008093F0038091F4039091F5030E94902AA7
:105680009093F5038093F4030E94410E0895CF9305
:10569000DF93EB018093FF030E94382A809301047B
:1056A000209759F044E054E060E070E0CE010E94A1
:1056B0007C61D0930304C09302040E94410EDF91E9
:1056C000CF910895CF93C82F882319F064ED71E02E
:1056D00002C064EF71E084E00E94D019CC2319F07D
:1056E0006CEC71E002C06CEE71E085E00E94D019B4
:1056F000CC2319F064EC71E002C064EE71E086E046
:105700000E94D019CC2319F06CEB71E002C06CED53
:1057100071E087E00E94D019CF910895CF93DF9375
:10572000C82FDD27C4FF02C083E001C085EA0E94C4
:105730005318C0FF02C084E001C085EA0E945318DC
:10574000C1FF02C085E001C085EA0E945318C2FF74
:1057500002C086E001C085EA0E945318C3FF02C060
:1057600087E001C085EA0E945318DF91CF91089528
:10577000809310040E94410E0895882319F06CE96B
:1057800071E002C064EA71E082E00E94D0190895DD
:105790000895882319F06CEA71E002C064EB71E0AF
:1057A00081E00E94D019089508950F931F93CF931D
:1057B0000EEE13E0C0911004CC2399F060E081E07C
:1057C0000E94A1188C2F81500E944F54BC0182E08E
:1057D0000E94291A1092100488EE93E00E94FA1693
:1057E00002C0882319F00E94C81903C0682F0E94C4
:1057F000A1188091EE039091EF03892BF9F00E949C
:105800002C55FC01828193814091EE035091EF036E
:105810008417950749F4218532858091020490917F
:1058200003042817390751F04283538380910204FF
:1058300090910304818792870E94B3542091EE03D4
:105840003091EF032115310529F4F80126833783C0
:10585000128A118A8091FE0382FD0DC08091FA03A5
:105860009091FB03A091FC03B091FD030097A1056B
:10587000B10519F105C06CEB73E082E00E94291AB2
:105880008091FA039091FB03A091FC03B091FD037A
:10589000BF93AF939F938F938FEB93E09F938F93DF
:1058A00082E08F930E947F1A8DB79EB707960FB63E
:1058B000F8949EBF0FBE8DBF43C02115310531F452
:1058C00062ED73E082E00E94291A18C03F932F9383
:1058D00089ED93E09F938F93C2E0CF930E947F1A4C
:1058E0008091FE030F900F900F900F900F9080FF0C
:1058F00002C08C2F01C080E20E945318C091FF03A8
:105900000E94840E853010F085E00EC0833061F473
:105910008C2F99278370907023E0880F991F2A9508
:10592000E1F7845A9C4F08C0992703E0880F991F1C
:105930000A95E1F784589C4FBC0182E00E94291A25
:105940006CE080E00E94A1188091000499278F7775
:1059500090709F938F938EED93E09F938F9382E04F
:105960008F930E947F1A8091FF0399278370907014
:105970000F900F900F900F900F90019779F483E1A3
:105980000E947617882331F080E00E94531864E665
:1059900071E010C080E20E9453180FC080E00E94A6
:1059A00053188091000487FF03C06CE372E002C0CB
:1059B00064E372E080E00E94D0190E94840EC82F38
:1059C000813049F488E00E941A54AC0160E08C2FC9
:1059D0000E946319E0C040E050E060E0862F0E9422
:1059E0001319C0E08AE00E947617882371F0809135
:1059F000F0039091F103892B39F48091FF039927EB
:105A000083709070039709F4C1E060E081E00E9428
:105A1000A1188091FA039091FB03A091FC03B0912F
:105A2000FD030097A105B10509F442C08DE00E9475
:105A30007617882329F48EE00E947617882381F157
:105A400082EE93E09F938F93C2E0CF930E947F1AE0
:105A50008DE00E9476170F900F900F90882379F0B9
:105A60006CEA71E081E00E94D01964EA71E08C2F49
:105A70000E94D0196CE271E089EC9BE20EC064EBED
:105A800071E081E00E94D0196CE971E08C2F0E94D6
:105A9000D0196CE271E08DEB9BE20E94DA187BC0BA
:105AA00086E00E941A54BC0182E00E94291A44C078
:105AB0008091F0039091F103009769F19F938F9388
:105AC0008EEE93E09F938F9382E08F930E947F1AD4
:105AD0008091F4039091F50314E0969587951A95BB
:105AE000E1F7282F2F70892F9927869586950F909B
:105AF0000F900F900F900F9080FD2061822F0E94D9
:105B00008E2BCC2321F08CE30E94531815C080E229
:105B10000E9453182CC084E094E09F938F9383EFEE
:105B200093E09F938F9382E08F930E947F1A0F9050
:105B30000F900F900F900F90CC23C9F08091F0033D
:105B40009091F103892B99F48091F4039091F503DE
:105B5000A4E096958795AA95E1F78F7080610E94E1
:105B60008E2B81E00E94622B6CEF71E011C02091BE
:105B7000F4032F708091F4039091F50397FD206159
:105B8000822F0E948E2B80E00E94622B64E072E0E4
:105B900083E00E94D019CF911F910F910895CF9368
:105BA000DF93EC012C853D854E855F856A817B8185
:105BB000211531054105510509F46BC061157105C9
:105BC000E1F0E881F981CF01AA27BB27821793076B
:105BD000A407B50741F0CB01AA27BB27821793077B
:105BE000A407B50751F488898E7F888BCF010E9466
:105BF00090291A821B8218821982888199819C01BE
:105C0000442755278C859D85AE85BF8568892817D3
:105C100039074A075B0729F481E068276B7F688BA7
:105C20003DC06C7F688B1C8A1D8A1E8A6E8981E04C
:105C30000E94A11880E00E941A54BC0182E00E94D8
:105C4000291A8889992796958795969587959C0115
:105C50002170307080FD13C088819981009711F008
:105C60008C839D832A833B832E833F8328833983C0
:105C7000198A6C857D858FEF0E94A35607C04C85DD
:105C80005D85688179818FEF0E94BF5688898B7FFF
:105C900004C0672B19F488898460888B1C861D8654
:105CA0001E861F86DF91CF9108956091F603709153
:105CB000F7038091F8039091F9036115710581054F
:105CC000910561F00E94C314882341F01092F603FD
:105CD0001092F7031092F8031092F90308950895B3
:105CE000EF92FF921F93CF93DF93EC01EEEEEE2E37
:105CF000E3E0FE2E81319105CCF48F3091050CF05C
:105D0000D0C08A30910509F473C18B30910534F409
:105D1000009709F40BC197FD7AC135C18C3091050C
:105D200009F462C00D970CF07EC05DC1853191050C
:105D3000D9F18631910574F48231910509F4D1C00D
:105D4000823191050CF4E4C083319105D1F144977F
:105D5000B1F05DC18F3891056CF48D3891050CF070
:105D600062C08C31910509F4B4C08A38910509F4F8
:105D70004CC14DC18339910509F447C148C1809197
:105D8000000499278F7790702091010433278217A0
:105D900093070CF03CC10E94840E833009F037C198
:105DA000809100048F5F1DC020910004822F9927ED
:105DB0008F779070892B09F42AC121502093000419
:105DC00024C18091FF03992783709070019729F473
:105DD00064E671E080E00E94D01980910004809513
:105DE00080788093000411C18AE00E94761788238E
:105DF00099F08091F0039091F103892B69F08091E3
:105E0000F4039091F50320E030E4822793279093E8
:105E1000F5038093F403F9C08091F4039091F503A6
:105E200020E030E850C08091FA039091FB03A091EC
:105E3000FC03B091FD030097A105B10581F120910C
:105E4000FA033091FB0321503040220F331FCE0163
:105E50008F7790700E9709F42160C7FF1AC041E058
:105E600060E0C9010E94ED6860E070E0CB010E9433
:105E7000DA1864E172E081E00E94D0196CE172E00E
:105E800082E00E94D019F7011486158616861786BF
:105E9000BCC041E0642FC9010E94ED68B6C0C7FDD7
:105EA000B4C01C2F1D508AE00E94761781111C5F20
:105EB00021E030E002C0220F331F1A95E2F78091F3
:105EC000F4039091F50382279327F7018683978344
:105ED0009CC06CE38091EE039091EF030E94A81D9B
:105EE00094C0F89483E00E94450E882319F084E062
:105EF0000E94D86B83E10E947617882339F06BE407
:105F00008091EE039091EF030E94A81D78947DC0CC
:105F10008AE00E947617811182E00E94450E882354
:105F200009F473C084E00E94D86B6FC08AE00E94BD
:105F300076178823A9F08091F2039091F3030097DC
:105F400009F465C0AA27BB278093FA039093FB034B
:105F5000A093FC03B093FD03C7010E94CF2D57C04F
:105F60008091FA039091FB03A091FC03B091FD0393
:105F70000097A105B10539F48FEF0E94C05381E06D
:105F80000E94D52B44C08091FA039091FB03A0910D
:105F9000FC03B091FD039C01AD0163E0220F331FB0
:105FA000441F551F6A95D1F7280F391F4A1F5B1FE1
:105FB000280F391F4A1F5B1FCE01AA2797FDA09506
:105FC000BA2F280F391F4A1F5B1F2030F8E23F0706
:105FD000F0E04F07F0E05F07D4F4F701248735873E
:105FE0004687578712C08EEE93E00E94CF2D0DC0DA
:105FF0001092FA031092FB031092FC031092FD031F
:106000008091FE038B7F8093FE030E94410EDF91FF
:10601000CF911F91FF90EF900895FC01EC5BFF4F33
:106020008081E454F040882319F480E090E00895E2
:10603000E95BFF4F8081E754F040882329F4848195
:10604000883511F0883719F481E090E0089580E0F8
:1060500090E008950895CF93DF93EC010E940D30F6
:10606000882319F480E090E01FC0FE01E95BFF4F38
:106070008081882351F4CC5BDF4F8881C454D040A9
:10608000823018F481E090E00FC08081882311F005
:106090008C8101C08D81992787FD90958095909581
:1060A0008827990F881F9927DF91CF910895CF9363
:1060B000C82FCF7719F480E090E029C0862F0E9486
:1060C000382A282F33272B31310589F02C3131051F
:1060D00024F42E30310529F017C02C31310569F038
:1060E00013C0EC2FFF27EB5CFB4F84910BC0EC2F10
:1060F000FF27E75EFB4F849105C0EC2FFF27E4509C
:10610000FC4F8491992703C0CF5F8C2F9927CF91A3
:106110000895CF93C82FCF7719F480E090E02EC078
:10612000C150862F0E94382A282F33272B31310562
:1061300079F02C31310524F42E30310529F01CC0C2
:106140002C31310569F018C08C2F992708960DC0A5
:1061500083E0C89FC00111240B966EE070E007C079
:106160008C2F9927880F991F079669E070E00E948D
:10617000A671CB01992702C08C2F9927CF91089542
:10618000019791F40E942C55FC018181882311F420
:1061900084E608C0843011F485E604C08150843060
:1061A00008F08150992708958FEF9FEF0895089583
:1061B0001F93CF93C82FFB01142F8181282F3327E2
:1061C00082819927982F8827282B392BC90101977D
:1061D0008F5F974210F062E010C0112321F0C901D7
:1061E0000E941C2703C0C9010E944926009751F450
:1061F000112311F06BE001C06AE08C2F0E94F919A5
:1062000080E090E0CF911F910895EF92FF920F935D
:106210001F93CF93DF93EB01E42E41E00E94D8302F
:106220008C01892B19F48FEF90E064C00E946D1BE4
:10623000882319F088E090E05DC0FB80EE2051F0EB
:1062400021E0F21639F4F82EF801808191810E9444
:10625000C31C08C0EE2031F0F80160858B810E94DC
:106260008930F82E6C81862F992785FF02C0F0E8CF
:10627000FF2AF801C481D581DF7784FDD06867FFEC
:1062800005C0C07F8F709070C82BD92B2F2D33275E
:1062900020783070F8016681862F99278078907079
:1062A0002817390731F0607840E0808191810E94A1
:1062B000AA2840E06F2DF801808191810E94AA28D0
:1062C00040E0BE01F801808191810E943029F801EF
:1062D000808191810E94BD290E94840E833019F42F
:1062E00080E090E007C0823019F481E490E002C0C1
:1062F00082E490E0DF91CF911F910F91FF90EF909A
:10630000089541E00E9405319927089540E00E94D8
:106310000531992708951F93CF93DF93182F40E0FD
:10632000812F0E94D830EC01892BF1F060E0812FA1
:106330000E94F91968858E810E945730682F812F3D
:106340000E94F9196C816F708C819D8197FD60614D
:106350008E8187FD6062812F0E94F9198E818F776F
:10636000682F812F0E94F9198FEF90E0DF91CF9174
:106370001F9108951F93CF93DF93182F40E0812F33
:106380000E94D830EC01892BC9F060E0812F0E9477
:10639000F91988858370682F812F0E94F9198885E3
:1063A0000E94382A682F812F0E94F9196FEF812FE0
:1063B0000E94F9196FEF812F0E94F9198FEF90E079
:1063C000DF91CF911F9108950F931F93CF93DF9388
:1063D0008B0141E00E94D830EC01892B19F48FEF3A
:1063E00090E014C08C819D818070F8012381332757
:1063F000822B932B40E0BC01888199810E94302937
:10640000888199810E94BD2980E090E0DF91CF9141
:106410001F910F9108950F931F93CF93DF938B01DB
:1064200041E00E94D830EC01892B19F48FEF90E005
:1064300018C02C813D81307CF801838199278F73AE
:106440009070982F8827282B392B40E0B90188813C
:1064500099810E943029888199810E94BD2980E01C
:1064600090E0DF91CF911F910F9108951F93CF93EB
:10647000DF93182F40E0812F0E94D830EC01892B48
:1064800041F060E0812F0E94F9196C81812F0E94F8
:10649000F9198FEF90E0DF91CF911F9108951F932D
:1064A000CF93DF93182F40E0812F0E94D830EC016A
:1064B000892B69F060E0812F0E94F9198C819D8100
:1064C000892F99278F73682F812F0E94F9198FEFD9
:1064D00090E0DF91CF911F910895DF92EF92FF92AC
:1064E0000F931F93CF93DF93982F8B01823008F087
:1064F00059C088E4989F7001112481E194E0E80E6E
:10650000F91EFB018181C82FDD27828199278770C1
:106510009070982F8827C82BD92B2197F7E0C83F78
:10652000DF0718F082E090E03FC00E94840E8330C5
:1065300039F00E94840E823019F086E090E034C079
:10654000CC0FDD1FF801628167FFC160862F99279C
:10655000E6E096958795EA95E1F771E0D72ED82287
:1065600087010B5B1F4FF80180819181FFEF8F3F07
:106570009F0749F040E0642F0E94ED688FEF9FEF86
:10658000F8018083918340E06D2DCE010E94ED687B
:10659000882319F489E090E007C0DD2019F0F801A4
:1065A000C083D18380E090E0DF91CF911F910F9164
:1065B000FF90EF90DF900895FF920F931F93CF937A
:1065C000F82EFB018181082F11278281992787707E
:1065D0009070982F8827082B192B87E0083F180701
:1065E00018F082E090E01CC0C8010E94DD67873689
:1065F00011F0873411F4C4E001C0C0E0C801880F75
:10660000991F0E944A6A039709F4C16060E08F2DC8
:106610000E94F9196C2F8F2D0E94F9198FEF90E0CD
:10662000CF911F910F91FF9008951F93CF93182F33
:10663000FB01C181CC2319F482E090E00FC060E03F
:106640000E94F919EC2FFF27E557F44F80818095C0
:10665000682F812F0E94F9198FEF90E0CF911F9141
:1066600008951F93CF93182FFB01C181C150C032F1
:1066700018F082E090E015C060E00E94F91960E037
:106680008C2F0E94C75E682F812F0E94F91961E04C
:106690008C2F0E94C75E682F812F0E94F9198FEFFF
:1066A00090E0CF911F9108950E94E25E80E090E01B
:1066B00008951F93CF93182FFB018181992700978D
:1066C00019F0039729F008C0C091CA0ACC0F07C07F
:1066D000C091CB0AC17003C082E090E00AC060E0C4
:1066E000812F0E94F9196C2F812F0E94F9198FEFC9
:1066F00090E0CF911F910895FB0181819281282F15
:1067000033272115310521F02330310559F014C00C
:10671000913490F4892F99270196959587958093C8
:10672000CA0A0DC08091CB0A992311F0816001C083
:106730008E7F8093CB0A03C082E090E0089580E0D2
:1067400090E008950895EF92FF920F931F93CF93D7
:10675000DF93CDB7DEB760970FB6F894DEBF0FBEFC
:10676000CDBFF82E63E00E94F91961E08F2D0E94E1
:10677000F91964E08F2D0E94F91963E08F2D0E94B2
:10678000F91964E08F2D0E94F9190E946955DC0106
:10679000CB01BF93AF939F938F9384E494E09F9337
:1067A0008F938E010F5F1F4F1F930F930E947B6C7F
:1067B0008DB79EB708960FB6F8949EBF0FBE8DBFDB
:1067C00033E0E32EF80191919295907F81918F01B2
:1067D0008053982B692F8F2D0E94F919EA94E7FEB8
:1067E000F1CF80E090E060960FB6F894DEBF0FBE68
:1067F000CDBFDF91CF911F910F91FF90EF90089542
:106800001F93CF93182FC0E00E94840E982F8250C0
:10681000823008F4C8E0923009F4C0616C2F812FF7
:106820000E94F9198FEF90E0CF911F9108951F9367
:10683000CF93DF93182FFB018181282F332782818B
:106840009927982F8827822B932B0E94C030EC0128
:1068500097FF03C082E090E00AC060E0812F0E94B1
:10686000F9196C2F812F0E94F9198FEF90E0DF91B9
:10687000CF911F91089560E00E94F91982E00E9473
:10688000450E8FEF90E0089580E00E94450E80E075
:1068900090E0089583E00E94450E80E090E0089526
:1068A00080E090E008951F93CF93DF93182F0E940C
:1068B000736BEC0160E084E0989F812D992711248F
:1068C00080FD61E0CE01892F99278295869587709A
:1068D00080FD6460C0FD6860D7FD6062CE7FDF71BF
:1068E000209709F06068812F0E94F919209791F094
:1068F00060E0C1FD61E0C2FD6064C97F209709F0DE
:106900006068812F0E94F919CD2B21F060E0812F62
:106910000E94F9198FEF90E0DF91CF911F910895B8
:106920000F931F93CF93DF93182FC9E4D8E000E0B3
:106930008091C90A081778F58F8180FF29C0688582
:106940008E810E945730682F812F0E94F9196C8127
:10695000812F0E94F9196881812F0E94F91988817D
:106960009981892F9927682F6F738C819D8197FD5D
:1069700060648E8187FD6068812F0E94F9198E8185
:106980008F77682F812F0E94F9198F818E7F8F83D7
:106990000F5F2A96CDCF80E890E0DF91CF911F91D5
:1069A0000F9108956F927F928F929F92AF92BF92B4
:1069B000CF92DF92EF92FF920F931F93CF93DF93CB
:1069C000CDB7DEB7C254D0400FB6F894DEBF0FBECD
:1069D000CDBF882E01E010E0AA249A2CB1E0BB2E96
:1069E0007E01E00EF11E3701C92CDD24F601E457CB
:1069F000F34FE081EE2319F4095F1F4F2CC0EB2108
:106A000041F1F70101937F01812F992787708083DE
:106A1000C80101970E94DD67982F873411F08736EF
:106A200021F4F701808180688083973411F09235DA
:106A300021F4F7018081806480830894E11CF11CBB
:106A4000A394F601E457F34F9B2D90958081892301
:106A50008083BB0C19F49394F1E0BF2E0F5F1F4F9E
:106A6000F7E0093F1F0720F48FE18A1508F0BCCF3B
:106A70006A2D882D0E94F919DD2473010A2D112732
:106A80000115110581F0F70181917F01682F882D93
:106A90000E94F919D3942D2D3327C801800F911F1F
:106AA0002817390784F38FEF90E0CE5BDF4F0FB6E6
:106AB000F894DEBF0FBECDBFDF91CF911F910F9134
:106AC000FF90EF90DF90CF90BF90AF909F908F900E
:106AD0007F906F900895CF92DF92EF92FF920F9385
:106AE0001F93CF93DF93D82ECC248091CA0A88239A
:106AF00009F454C0F8948C2D992787FD9095880F40
:106B0000991F9C01245B344F8C01045F144FEC01EE
:106B1000C453D54F4881942F9095D8018C918923E7
:106B2000F901E080E82A5981952F9095F80181813B
:106B30008923F901F180F82A2E2D332727FD30957E
:106B4000842F99272817390749F42F2D332727FD3C
:106B50003095852F99272817390799F08C2D8F5F4D
:106B6000682F8D2D0E94F9196E2D8D2D0E94F91917
:106B70006F2D8D2D0E94F919E882F982F80111829A
:106B800010827894C3942C2D332727FD3095809163
:106B9000CA0A9927281739070CF4ACCF60E08D2D6D
:106BA0000E94F9198FEF90E0DF91CF911F910F9123
:106BB000FF90EF90DF90CF9008951F93CF93C82F51
:106BC000162F603418F06AE474E002C064E574E0E3
:106BD0008C2F0E94291A812F99278A30910589F1DB
:106BE0008B3091057CF48630910511F18730910549
:106BF0001CF40297D1F039C088309105F9F009975B
:106C0000D1F033C08E30910529F18F30910534F4E5
:106C10008B309105C9F00D97D1F027C081349105D3
:106C2000E1F082349105E1F020C06CE574E01AC017
:106C300060E774E017C06DE774E014C060E974E0C9
:106C400011C063EA74E00EC06BEA74E00BC06DEB38
:106C500074E008C066EC74E005C06DED74E002C03D
:106C600068EE74E08C2F0E94291A103420F06DE039
:106C70008C2F0E94F91981E090E0CF911F91089527
:106C80000F931F93D8018A30C0F48617B0F4992768
:106C9000FC0114E0EE0FFF1F1A95E1F7E81BF90B5A
:106CA000EF55FB4F8685882341F000811181041741
:106CB000150718F02017310708F48D01C8011F913E
:106CC0000F91089563EF74E00E94291A81E090E02B
:106CD00008956AE275E00E94291A81E090E0089523
:106CE00067E475E00E94291A81E090E008951F93FF
:106CF000182F60E875E00E94291A6AE975E0812F73
:106D00000E94291A69EB75E0812F0E94291A81E0FF
:106D100090E01F910895CF93C82F0E94840E992769
:106D200083309105A1F0843091052CF4009749F04F
:106D3000029751F017C08430910561F0079794F4E1
:106D40000CC066ED75E00BC06EED75E008C066EE38
:106D500075E005C06DEE75E002C069EF75E08C2F3F
:106D60000E94291A81E090E0CF910895EF92FF925E
:106D70000F931F93182F7B01042F80E00E94450E74
:106D8000402FB701812F0E948B3699271F910F91B9
:106D9000FF90EF900895EF92FF920F931F93182F9B
:106DA0007B01042F83E00E94450E402FB701812F05
:106DB0000E948B3699271F910F91FF90EF900895B5
:106DC0006FEF75E00E94291A82E00E94450E80E074
:106DD00090E008950F931F93CF93C82F762F642FC1
:106DE00000E010E0A801872F0E9440368C01892B1B
:106DF00021F462E08C2F0E94DD35C801CF911F91F4
:106E00000F9108957F928F929F92AF92BF92CF92EF
:106E1000DF92EF92FF920F931F93CF93DF93882E11
:106E2000942E2FEF37E260E00E94EA365C01009773
:106E300019F481E090E062C10E9449266C01892B1F
:106E400069F421E0291510F06AE012C0C5010E9422
:106E50001C276C01892B11F46BE00AC031E0391555
:106E600008F0D6C00E946D1B782E882331F068E0B0
:106E7000882D0E94DD35992741C1F601C481D58155
:106E800050EFE52E5FE7F52EEC22FD228D2F99279E
:106E900087FD90958827990F881F99278C0121E0FD
:106EA00030E040E050E0692D82E00E944036892BBE
:106EB00021F020E030E8E22AF32ACE0181709070C0
:106EC0008C0121E030E040E050E0692D84E00E9438
:106ED0004036892B21F081E090E0E82AF92ACE01A2
:106EE00096958795817090708C0121E030E040E0AC
:106EF00050E0692D85E00E944036892B21F0E2E0C8
:106F0000F0E0EE2AFF2ACE01969587959695879513
:106F1000817090708C0121E030E040E050E0692DFC
:106F200086E00E944036892B21F024E030E0E22AFE
:106F3000F32A83E0D695C7958A95E1F7C170D070A2
:106F40008E0121E030E040E050E0692D87E00E94B2
:106F50004036892B21F088E090E0E82AF92A472D75
:106F6000B701C5010E943029F601608586810E9423
:106F7000573099278C012FE730E040E050E0692D31
:106F800081E00E944036C82F8091D004863411F4ED
:106F900011E015C0823511F4172D11C000E010E08A
:106FA000F601868187FF02C001E010E021E030E0B9
:106FB00040E050E0692D83E00E944036182FC13038
:106FC00029F4C0E0C5010E94C31C06C0F60160851B
:106FD0008C2F0E948930C82F1111C0682C2F3327A5
:106FE00020783070F6016681862F9927807890701E
:106FF0002817390729F0607840E0C5010E94AA28C7
:1070000040E06C2FC5010E94AA28C5010E94BD293D
:107010000E94840E823011F461E405C00E94840E47
:10702000833021F062E4882D0E94DD35F6018481F1
:10703000958183FF03C081E390E002C080E390E08C
:107040009F938F93F6018481958182FF03C081E332
:1070500090E002C080E390E09F938F93F6018481DB
:10706000958181FF03C081E390E002C080E390E05E
:107070009F938F93F6018481958180FF03C081E304
:1070800090E002C080E390E09F938F93F6018681A9
:1070900087FF03C086E690E002C082E790E09F93FE
:1070A0008F93F6018581282F332727FD3095209572
:1070B00030952227330F221F332781E390E0821B74
:1070C000930B9F938F93608586810E9457309927F9
:1070D0009F938F93BF92AF9289E096E09F938F9397
:1070E0008F920E947F1A81E090E02DB73EB72D5E0F
:1070F0003F4F0FB6F8943EBF0FBE2DBFDF91CF912B
:107100001F910F91FF90EF90DF90CF90BF90AF90C5
:107110009F908F907F900895CF93C82F2FEF37E2E5
:1071200060E08C2F0E94EA36009719F10E944926F0
:10713000FC01892B19F463E276E018C08085992759
:10714000837090708230910561F0833091051CF45A
:10715000019721F00EC0039739F00BC06AE276E088
:1071600005C067E376E002C064E476E08C2F0E94FD
:10717000291A81E090E0CF9108957F928F929F929B
:10718000AF92BF92CF92DF92EF92FF920F931F9335
:10719000CF93DF93A82EB42E2FEF37E260E00E944A
:1071A000EA364C01009719F481E090E021C10E9479
:1071B00049266C01892B69F421E02B1510F06AE057
:1071C00012C0C4010E941C276C01892B11F46BE0D2
:1071D0000AC031E03B1508F08FC00E946D1B782E6D
:1071E000882331F068E08A2D0E94DD35992700C19F
:1071F000F601E480F580E701C070C70181709070EE
:107200008C0121E030E040E050E06B2D81E00E94F5
:107210004036892B09F0C160C7019695879581702A
:1072200090708C0121E030E040E050E06B2D82E076
:107230000E944036892B09F0C260C7019695879558
:1072400096958795817090708C0121E030E040E048
:1072500050E06B2D83E00E944036892B09F0C4601A
:1072600063E0F694E7946A95E1F7F1E0EF22FF24FA
:10727000870121E030E040E050E06B2D84E00E9487
:107280004036892B09F0C860870121E030E040E0FA
:1072900050E06B2D85E00E944036892B09F0C061DB
:1072A000870121E030E040E050E06B2D86E00E9455
:1072B0004036892B09F0C062870121E030E040E0D0
:1072C00050E06B2D87E00E944036892B09F0C064A6
:1072D000870121E030E040E050E06B2D88E00E9423
:1072E0004036892B09F0C068472DBE01C4010E94B9
:1072F0003029C4010E94BD290E94840E882321F4F4
:1073000062E48A2D0E94DD35F6018481958187FF34
:1073100003C081E390E002C080E390E09F938F93ED
:10732000F6018481958186FF03C081E390E002C06D
:1073300080E390E09F938F93F6018481958185FF90
:1073400003C081E390E002C080E390E09F938F93BD
:10735000F6018481958184FF03C081E390E002C03F
:1073600080E390E09F938F93F6018481958183FF62
:1073700003C081E390E002C080E390E09F938F938D
:10738000F6018481958182FF03C081E390E002C011
:1073900080E390E09F938F93F6018481958181FF34
:1073A00003C081E390E002C080E390E09F938F935D
:1073B000F6018481958180FF03C081E390E002C0E3
:1073C00080E390E09F938F939F928F9288E496E062
:1073D0009F938F93AF920E947F1A81E090E02DB728
:1073E0003EB72B5E3F4F0FB6F8943EBF0FBE2DBF8A
:1073F000DF91CF911F910F91FF90EF90DF90CF9091
:10740000BF90AF909F908F907F9008957F928F92C2
:107410009F92AF92BF92CF92DF92EF92FF920F9323
:107420001F93CF93DF93A82EB42E2FEF37E260E0A7
:107430000E94EA364C01009719F481E090E02EC1D9
:107440000E9449266C01892B69F421E02B1510F06C
:107450006AE012C0C4010E941C276C01892B11F440
:107460006BE00AC031E03B1508F09DC00E946D1B27
:10747000782E882331F068E08A2D0E94DD35992727
:107480000DC1F601C481D5817FEFE72E70ECF72E98
:10749000EC22FD228D2F9927817090708C0121E0C4
:1074A00030E040E050E06B2D81E00E944036892BB7
:1074B00021F020E031E0E22AF32ACE01892F99273A
:1074C0008695817090708C0121E030E040E050E0C2
:1074D0006B2D82E00E944036892B21F080E092E003
:1074E000E82AF92ACE01892F9927869586958170F9
:1074F00090708C0121E030E040E050E06B2D83E0A3
:107500000E944036892B21F0E0E0F4E0EE2AFF2AC9
:10751000CE01892F992786958695869581709070E2
:107520008C0121E030E040E050E06B2D84E00E94CF
:107530004036892B21F020E038E0E22AF32ACE0100
:10754000892F992782958F70817090708C0121E02E
:1075500030E040E050E06B2D85E00E944036892B02
:1075600021F080E090E1E82AF92ACD2FDD27C295AD
:10757000C695C770C170D0708E0121E030E040E048
:1075800050E06B2D86E00E944036892B21F0E0E030
:10759000F0E2EE2AFF2A472DB701C4010E943029EC
:1075A000C4010E94BD290E94840E882321F462E454
:1075B0008A2D0E94DD35F60184819581892F9927D6
:1075C00082958695877080FF03C081E390E002C0BA
:1075D00080E390E09F938F93F60184819581892FBA
:1075E000992782958F7080FF03C081E390E002C0ED
:1075F00080E390E09F938F93F60184819581892F9A
:10760000992786958695869580FF03C081E390E053
:1076100002C080E390E09F938F93F601848195816F
:10762000892F99278695869580FF03C081E390E096
:1076300002C080E390E09F938F93F601848195814F
:10764000892F9927869580FF03C081E390E002C0CF
:1076500080E390E09F938F93F60184819581892F39
:10766000992780FF03C081E390E002C080E390E0AF
:107670009F938F939F928F9285E696E09F938F932F
:10768000AF920E947F1A81E090E02DB73EB72F5E47
:107690003F4F0FB6F8943EBF0FBE2DBFDF91CF9185
:1076A0001F910F91FF90EF90DF90CF90BF90AF9020
:1076B0009F908F907F900895AF92BF92CF92DF926C
:1076C000EF92FF920F931F93CF93DF93A82EC42FB7
:1076D0000E94840E882311F466E05DC028EF37E035
:1076E0004C2F60E08A2D0E94EA366C01892B19F03C
:1076F00021E02A1518F481E090E083C088E4A89E78
:10770000C00111248F5E9B4FC23008F44EC0A5E427
:10771000EA2EF12CE80EF91EF70180819181FFEF2E
:107720008F3F9F0749F040E0642F0E94ED688FEF84
:107730009FEFF701808391838091B204873411F425
:10774000BB2410C0823519F4F1E0BF2E0BC002E05B
:1077500010E021E030E040E050E06C2F81E00E943A
:107760004036B82E00E010E021E030E0A8016C2F98
:1077700082E00E944036EC01860101501040000F6B
:10778000111F0B0D111D40E0682FC8010E94ED680C
:10779000882331F469E08A2D0E94DD35992731C0B4
:1077A000CC2319F0F70100831183C60101970E94D1
:1077B000DD67C0E0D0E0082F112707FD1095C80154
:1077C0000E94CD71892B11F0C1E0D0E0DF93CF93FF
:1077D000C8010E94E0719F938F93DF92CF928DE753
:1077E00096E09F938F93AF920E947F1A81E090E082
:1077F0002DB73EB7275F3F4F0FB6F8943EBF0FBE81
:107800002DBFDF91CF911F910F91FF90EF90DF90EF
:10781000CF90BF90AF9008951F93182F68E876E03F
:107820000E94291A65E976E0812F0E94291A0E9498
:107830006955DC01CB01BF93AF939F938F938BE985
:1078400096E09F938F931F930E947F1A8DB79EB7E8
:1078500007960FB6F8949EBF0FBE8DBF81E090E0F3
:107860001F910895EF92FF920F931F93CF93DF9391
:10787000E82EF42E0E942C55EC01FF20E1F08B85C0
:1078800099278C0124E130E040E050E06F2D80E04A
:107890000E9440368B878C859927880F991F8C0111
:1078A0002EEF31E042E050E06F2D81E00E94403643
:1078B000969587958C878C859927880F991F9F931C
:1078C0008F938B8599279F938F9388EA96E09F9358
:1078D0008F93EF920E947F1A8DB79EB707960FB6CF
:1078E000F8949EBF0FBE8DBF81E090E0DF91CF91F5
:1078F0001F910F91FF90EF9008950F931F93CF93D7
:10790000C82F642F442379F08091CB0A9927817086
:1079100090708C0121E030E040E050E080E00E9477
:1079200040360E94D75E8091CB0A99278170907073
:107930009F938F9381EB96E09F938F93CF930E94B9
:107940007F1A0F900F900F900F900F9081E090E0B2
:10795000CF911F910F910895DF92EF92FF920F93B5
:107960001F93CF93E82E842F00E010E020E230E058
:1079700041E050E0682F80E00E944036C82F882305
:1079800009F447C099279F938F9387EB96E09F93C5
:107990008F93EF920E947F1ADC2EDA9460E08D2D97
:1079A0000E94C75E082F112781E0F82E0F900F90DC
:1079B0000F900F900F90C7E08F2D99278023912370
:1079C000892B11F061E301C060E38E2D0E94F9194B
:1079D000C150FF0CC7FFF0CF60E28E2D0E94F91955
:1079E00061E08D2D0E94C75E082F1127C1E0FC2E9B
:1079F000C7E08F2D992780239123892B11F061E314
:107A000001C060E38E2D0E94F919C150FF0CC7FF21
:107A1000F0CF81E090E0CF911F910F91FF90EF9018
:107A2000DF900895FF920F931F93F82E642F80919B
:107A3000CA0A9927880F991F8C0120E430E040E0A2
:107A400050E080E00E9440368F5F86958093CA0A9E
:107A50009927880F991F9F938F938AED96E09F93A4
:107A60008F93FF920E947F1A0F900F900F900F90AC
:107A70000F9081E090E01F910F91FF900895CF93B8
:107A8000C82F4423C9F4C13031F460EE76E08C2F66
:107A90000E94291A13C00E9411119F938F9386EEA2
:107AA00096E09F938F93CF930E947F1A0F900F9031
:107AB0000F900F900F9002C0C13019F481E090E058
:107AC0000DC069EE76E08C2F0E94291A8091A104E6
:107AD0009091A2040E94D11080E090E0CF9108958F
:107AE0000F931F93CF93C82F842F0FEF1FEF27EE15
:107AF00033E040E050E0682F80E00E9440360E9472
:107B0000C03097FF06C062E08C2F0E94DD359927B8
:107B100011C090709F938F938CEE96E09F938F93FC
:107B2000CF930E947F1A81E090E00F900F900F900A
:107B30000F900F90CF911F910F910895EF92FF92A8
:107B40000F931F93982F642F4423C9F088E4989FC4
:107B50007001112481E194E0E80EF91E00E010E0CC
:107B600021E030E0A80180E00E944036F701E95BA7
:107B7000FF4F892B19F081E0808301C0108281E0E2
:107B800090E01F910F91FF90EF900895AF92BF92F8
:107B9000DF92EF92FF920F931F93CF93DF93CDB7B6
:107BA000DEB72D970FB6F894DEBF0FBECDBFD82E2F
:107BB00080E090E00E94FF617C015C01C7010197B9
:107BC0008F5F934008F056C0AE014F5F5F4FBE011C
:107BD000635F7F4FC7010E947C618C01892B09F490
:107BE00049C08D850E94382A9F938F931F930F93CE
:107BF0008FEE96E09F938F93DF920E947F1A8DB74E
:107C00009EB707960FB6F8949EBF0FBE8DBF8D85A9
:107C10009927837090708230910561F083309105CF
:107C20001CF4019721F00EC0039739F00BC068EFE8
:107C300076E005C06CEF76E002C060E077E08D2D65
:107C40000E94291ACE0101969F938F9384E097E0BA
:107C50009F938F93DF920E947F1AC7010E94FF615A
:107C60007C010F900F900F900F900F908A159B053D
:107C700009F0A4CF6AE077E08D2D0E94291A81E0F7
:107C800090E02D960FB6F894DEBF0FBECDBFDF910A
:107C9000CF911F910F91FF90EF90DF90BF90AF9029
:107CA0000895CF92DF92FF920F931F93CF93F82EF8
:107CB000C42F00E010E02FEF37E241E050E06C2FDE
:107CC00080E00E9440366C01892B09F464C000E01A
:107CD00010E02FE730E04EE050E06C2F81E00E9492
:107CE0004036C82F8091CD04882309F454C0809178
:107CF000DC04882309F44FC06AE672E081EC94E06A
:107D00000E94AC6C892B41F06EE672E081EC94E04D
:107D10000E94AC6C892B11F461E023C062E772E031
:107D200081EC94E00E94AC6C892B41F066E772E034
:107D300081EC94E00E94AC6C892B11F462E011C0DC
:107D40006AE772E081EC94E00E94AC6C892B41F010
:107D50006EE772E081EC94E00E94AC6C892BD9F460
:107D600063E0862F99278370907081309105CCF065
:107D7000833091051CF0039721F013C0CB3119F02B
:107D800008C0CC3111F464600CC0CE3711F46860C7
:107D900008C0CE3031F062E08F2D0E94DD3599278A
:107DA00007C040ED54E0C6010E94746181E090E09C
:107DB000CF911F910F91FF90DF90CF90089502C057
:107DC0000E94D96080E090E00E94FF610097C1F7B7
:107DD00081E090E00895EF92FF920F931F93CF936D
:107DE000DF93CDB7DEB766970FB6F894DEBF0FBE50
:107DF000CDBFE82ECE0101960E94E65FED81FE81A7
:107E0000CF0101978F5F934008F041C020E0AE01A1
:107E1000495F5F4F60E1CF0174E0880F991F7A9549
:107E2000E1F70E94C25FFF2400E010E0F801EC0FD0
:107E3000FD1F21853285C90101978F5F974200F5AB
:107E40003F932F93FF2019F082E892E002C085E86B
:107E500092E09F938F9380E197E09F938F93EF92AF
:107E60000E947F1A8DB79EB707960FB6F8949EBFF3
:107E70000FBE8DBFF3940E5F1F4F96E09F15B0F6B7
:107E80006DE08E2D0E94F919EF81F885B9CF65E17B
:107E900077E08E2D0E94291A81E090E066960FB659
:107EA000F894DEBF0FBECDBFDF91CF911F910F9130
:107EB000FF90EF900895CF92DF92FF920F931F9360
:107EC000CF93C42F00E010E02FEF37E241E050E005
:107ED0006C2F80E00E9440366C01892BA1F0E1E01C
:107EE000FE2EFC1680F400E010E02FEF37E241E0B8
:107EF00050E06C2F8F2D0E944036BC01C6010E94BD
:107F00006B29F394EECF81E090E0CF911F910F9118
:107F1000FF90DF90CF9008950E94A72981E090E024
:107F20000895DF92EF92FF920F931F93CF93DF9309
:107F3000082FEB01D42E823008F00EC188E4089F90
:107F4000900111242F5E3B4F4881142F1F71642F25
:107F50007727CB01807E90708034910509F4A3C00F
:107F60008134910534F40097A9F0809709F463C037
:107F7000F3C08038910509F4BFC0813891052CF415
:107F80008036910509F4B0C0E7C0803C910509F442
:107F9000CCC0E2C021E02D1508F0E0C08981C82FD7
:107FA000DD27CE010E941C27FC01892B09F4D4C0D7
:107FB000E480F58014FF05C080E090E8E82AF92A03
:107FC00004C08FEF9FE7E822F9221F700681007836
:107FD0001F3019F460E8602729C080851F7011F0F8
:107FE0001F3019F460E070E020C00E94382A282F6A
:107FF00033272C31310571F02D31310524F42B312B
:10800000310529F010C02E37310531F00CC0110FA9
:10801000115009C0110F07C089E0189F802D11244D
:10802000682F772702C0612F7727602B40E0CE01B1
:108030000E94AA2850C0437F488315E4E12EF12C0A
:10804000E20EF31EF70180819181FFEF8F3F9F07C2
:1080500049F040E0642F0E94ED688FEF9FEFF70139
:10806000808391832881203209F476C0233209F479
:1080700073C0F1E0FD15D0F46981213231F4C62FCF
:10808000DD272197CC0FDD1F05C0C62FDD27CC0FC4
:10809000DD1F219740E061E0CE010E94ED68F7010D
:1080A000C083D18359C0F1E0FD1518F080E090E065
:1080B00055C08981C82FDD27CE010E94AD27F0EF82
:1080C000EF2EFFEFFF2EE822F922812F99278F70E4
:1080D0009070E82AF92A40E0B701CE010E943029C9
:1080E000CE010E94BD2938C060FF02C080E001C0FF
:1080F00083E00E94450E30C0112311F4812F18C077
:10810000C0E0C11748F560E08C2F0E94B65E682F72
:10811000802F0E94F91961E08C2F0E94B65E682FB3
:10812000802F0E94F919CF5FECCF112321F481E059
:108130000E94D75E11C0115060E0812F0E94B65E90
:10814000682F802F0E94F91961E0812F0E94B65E8E
:10815000682F802F0E94F91981E090E0DF91CF9184
:108160001F910F91FF90EF90DF9008959B012F5F7B
:108170003F4F42E0B9010E94913F8FEF90E0089598
:108180009B012F5F3F4F41E0B9010E94913F8FEF6C
:1081900090E008958230C0F4282F332788E490E0DF
:1081A000289FF001299FF00D389FF00D1124EF5EFC
:1081B000FB4FEC5BFF4F1082339610828FEF9FEFE7
:1081C000929382930E94076C089508952F923F9294
:1081D0004F925F926F927F928F929F92AF92BF92D7
:1081E000CF92DF92EF92FF920F931F93CF93DF9383
:1081F000CDB7DEB726970FB6F894DEBF0FBECDBF62
:108200008B83E62E823008F003C288E49B81989F1E
:10821000800111240F5E1B4F34E4C32ED12CC00EFD
:10822000D11ED6018C918823B1F0F8018081918113
:10823000A281B38188539F4FAF4FBF4FBC01CD0187
:108240000E94C314882339F0C8010E940D3088238E
:1082500011F4D6018C938091330790913407A0914B
:108260003507B0913607F80180839183A283B383E9
:10827000D6018C91803408F01C92C8010E942B30EA
:10828000882391F0B8E0EB1641F4F6018081882351
:1082900009F4BEC181508083BBC1EE2009F4B8C18E
:1082A000FDE0EF1609F4EE24D601FC90F801EF0D85
:1082B000F11DE482F394FC92C8010E940D30B82EA7
:1082C000882309F49AC1C8010E942B30882309F43D
:1082D00060C1EE2009F09CC1F601E08286E791E0E2
:1082E0008C839D8324E0422E512C400E511E095B4D
:1082F0001F4FD8018C9107541040882329F495E032
:10830000492E512C400E511EF2018081882309F420
:108310003AC143E050E06BE177E0C2010E94CB6CD0
:10832000892B39F4C201039605C0FE814F2F5527D2
:10833000FBC0C2010E94296E49825A821E8286E9D0
:10834000E1EAF4E011928A95E9F705C00894211C4E
:10835000311C29823A8229803A80D1019C9199234B
:1083600091F09C3281F0943271F0953261F0892F56
:1083700080538A3040F0892F992787FD90950E947D
:10838000D771892B19F3F1018081882309F4C7C0C3
:1083900004C00F5F1F4F09831A8309811A81D80116
:1083A000DC908D2D992787FD90950E94D771892BA0
:1083B00081F7DD2009F4B9CFBCE2DB1641F40F5F91
:1083C0001F4F09831A83EE81EF5FEE839FC08FE01A
:1083D000FE81F89F7001112481EA94E0E80EF91EF5
:1083E00082E0682E712C6E0C7F1CCC2497E2D9168B
:1083F00019F0A2E2DA1629F40F5F1F4F09831A83DE
:10840000CD2CA980BA80450183010E191F090250A5
:10841000104008C00894811C911CF301D1923F01C7
:108420000F5F1F4F0B301105ACF4D401DC90DD2041
:1084300089F0CC2011F0DC1469F7CC2059F4BCE2AF
:10844000DB1641F08D2D992787FD90950E94D771FD
:10845000892B01F3F3011082D5018C91843239F418
:10846000C501019689839A8340E150E008C08532B6
:1084700051F4C501019689839A8342E050E0BE0120
:108480006F5F7F4F06C04AE050E0BE016F5F7F4FD5
:10849000C5010E94D96CDC01CB01F7018083918377
:1084A00081E0F701868704C00F5F1F4F09831A839D
:1084B00009811A81D801FC90FF2081F08F2D992726
:1084C00087FD90950E94D771892B41F4BCE2FB1681
:1084D00059F704C00F5F1F4F09831A8309811A815E
:1084E000F801F080FF2041F08F2D992787FD9095AE
:1084F0000E94D771892B71F7FCE2FF1621F40F5F00
:108500001F4F09831A838E818F5F8E83E981FA81E1
:108510008081882321F09E819A3008F43ECFD101DA
:108520001C92BE814B2F5527142F8091760190917C
:108530007701892BD1F0EC81FD8160817181C201CD
:108540000E94AC6C892B41F4EC81FD812281338146
:108550002115310581F417C08C819D8104968C838F
:108560009D83DC018D919C91E4CF6FE177E08B815D
:108570000E94291A08C0412FB2018B81F901099587
:10858000882309F445C06FE277E08B810E94291AA5
:108590003FC0E6EFF1E0A8014C5F5F4F2F2D095B74
:1085A0001F4FD8018C9107541040882321F4A80153
:1085B0004B5F5F4F21508091F601882349F19081F4
:1085C000DA018C919817A1F48181281708F10280B3
:1085D000F381E02D309749F0BA018B810995682F1E
:1085E0008F3F19F08B810E94F919F601108210C09B
:1085F00034968081882319F70BC00C5F1F4F4F2DD5
:10860000B8018B810E94913F882311F0D601BC9262
:1086100026960FB6F894DEBF0FBECDBFDF91CF9187
:108620001F910F91FF90EF90DF90CF90BF90AF9090
:108630009F908F907F906F905F904F903F902F9082
:108640000895FB0121E057FF04C020E050954195BB
:108650005F4F8330910549F18430910534F48130C6
:10866000910591F0029729F12AC08430910519F003
:10867000059761F024C081818F5F818399278417DA
:108680009507ECF0222359F0118219C081818150A5
:10869000818399278417950794F0222321F0842F52
:1086A000815081830CC021830AC012821382168AF2
:1086B00006C090E08281882309F491E0928380E0F3
:1086C00090E008950F931F93CF93DF938C010E9446
:1086D000442AEC01009731F46DE570E182E00E94DC
:1086E000291A0FC09F938F9383E690E19F938F93F6
:1086F00082E08F930E947F1A0F900F900F900F903F
:108700000F900115110521F0B80182E00E94291A8D
:10871000CE01DF91CF911F910F9108950F931F9379
:10872000CF93DF93EC018B01009731F097FD35C0BB
:108730000297029790F52BC060E081E00E94A1189B
:10874000F8018281882359F467E670E182E00E9493
:10875000291A60E770E182E00E94291A18C00E947D
:108760006955DC01CB01BF93AF939F938F9386E74D
:1087700090E19F938F9382E08F930E947F1A8DB731
:108780009EB707960FB6F8949EBF0FBE8DBF40E010
:1087900050E0B801CE010E94214380E090E0DF91DB
:1087A000CF911F910F9108958230910541F0833050
:1087B000910541F440E050E00E94214303C08FEF57
:1087C0009FEF089580E090E008950895AF92BF92E2
:1087D000CF92DF92EF92FF920F931F93CF93DF938D
:1087E000EC017B010E94412A8C01C230D10509F4C1
:1087F00053C0C330D1052CF42097D1F0219731F02C
:1088000092C0C630D1050CF08EC02AC0FC0161892F
:10881000262F269526952370637009F461E083E086
:10882000689FC0011124280F2350F70121837BC0CA
:1088300060E081E00E94A11882E890E10E9462431A
:10884000892B09F470C0F70191818AE0989FC001DB
:1088500011248D57984FBC0182E00E94291A63C0F1
:1088600049E050E0B701CE010E942143F801808128
:1088700091818F3F910509F008F455C0F70181817E
:10888000882311F486E08183F7018181863008F026
:108890004AC088E0818347C0FC01A280B380A11454
:1088A000B10409F040C0F70182818823A1F1F801E9
:1088B000C081D1812097B9F1F7013181832F63E025
:1088C0000E949A71282F2F5F832F0E949A71892FFF
:1088D0009927880F991F880F991F282BF801C488A2
:1088E000D588622FCE010E94B727CE010E9499271A
:1088F000B5010E94472BC114D10469F0C801469606
:108900009C01F801418960817181C6010E94DC608F
:10891000F801848B958B90E0F7018281882309F41C
:1089200091E0F701928380E090E0DF91CF911F9179
:108930000F91FF90EF90DF90CF90BF90AF90089590
:10894000482F30E0832F992787FD9095FC01EE5A40
:10895000F84F2491241729F03F5F222399F78FEFD6
:108960009FEF08950895EF92FF920F931F93CF9377
:10897000DF93EB018230910509F486C083309105C5
:1089800034F4009709F43EC0019769F0BAC084300E
:10899000910509F443C0843091050CF470C005972B
:1089A00009F456C0AEC00E94412A8C01FC018081AE
:1089B0009181892B09F4A5C046E1E42EF12CE00E4B
:1089C000F11E8E01065F1F4F65960C171D07B8F448
:1089D000F7018081882339F00E94A04487FD03C0FD
:1089E000F701808101C080E2F80181938F01F701D6
:1089F0008081882351F30894E11CF11CE6CFF80133
:108A000010827FC00E94624360E081E00E94A11852
:108A10002A96BE0182E00E943F1A73C08981FB0141
:108A2000E80FF11DEF012A9682850E94A0448F5F16
:108A3000E82FFF27E7FDF095EE5AF84F8491882341
:108A400019F4E2E5F7E08491992787FD909515C028
:108A50008981FB01E80FF11DEF012A9682850E94B2
:108A6000A044181614F08FE201C08150E82FFF27B0
:108A7000E7FDF095EE5AF84F8491888342C049E0B3
:108A800050E00E9421433DC00E94412A8C01FC011C
:108A900082819381892BA9F59A81992349F489E0F0
:108AA0008B8381E0888F99839F8B8A838E8B29C0EB
:108AB00089818F5F89838F8B8B3018F11B821A829B
:108AC0001E8A8CE098012A5E3F4FD901FE013A963A
:108AD00001900D928A95E1F7F801848995890097B4
:108AE00031F04189608171810E94DC6007C0A90179
:108AF000F8016189808191810E947461F801848B01
:108B0000958B80E090E0DF91CF911F910F91FF90C6
:108B1000EF900895AF92BF92CF92DF92EF92FF92C3
:108B20000F931F93CF93DF93CDB7DEB721970FB687
:108B3000F894DEBF0FBECDBF9C018B018230910542
:108B400009F455C0833091052CF40097C1F00197CA
:108B500059F0A5C084309105D9F1843091050CF409
:108B600041C00597C9F19BC04BE050E060E270E066
:108B7000C8010A960E94746CF801158A90C0FB0126
:108B80008281882309F48BC08181882309F487C0FE
:108B9000065F1F4FA801B90199270E947C619F932E
:108BA0008F9385E890E19F938F9362E0F62EFF927A
:108BB0000E947F1A60E081E00E94A118B8018F2D09
:108BC0000E943F1A0F900F900F900F900F9067C068
:108BD000FB018181992721C0FB01818199270E9496
:108BE00034621DC049E050E00E94214358C090E02B
:108BF000FB018281882309F491E0F80192830E94AD
:108C0000412A7C01F8018281882361F0F70184897F
:108C10009589009711F0848902C00E94FF61F801D4
:108C200081833DC05AE0A52EB12CA00EB11EF801E3
:108C30008181A501BE016F5F7F4F99270E947C61F2
:108C40006C01F7011282138210821182BC018FEF36
:108C50000E94A356F70180819181892B69F0698177
:108C6000C6010E94B727C6010E94992760E070E004
:108C70000E94472B0E94532AF70180819181892B02
:108C800059F0B501C70146960E94B66CF801818182
:108C90009927F701848B958B8FEF9FEF02C080E0BF
:108CA00090E021960FB6F894DEBF0FBECDBFDF91E6
:108CB000CF911F910F91FF90EF90DF90CF90BF90D9
:108CC000AF9008950F931F93CF93DF93EC010E9411
:108CD000412A8C01209719F02297C9F03DC0CE019E
:108CE0000E946243892BC1F160E081E00E94A118DB
:108CF000F80184899589892B11F081E001C082E017
:108D00000E941A54BC0182E00E94291A25C0FC016D
:108D1000C281D381209701F580819181892BE1F077
:108D200084899589892BC1F060E081E00E94A118B7
:108D300083E00E941A54BC0182E00E94291A84EF49
:108D400091E00E94FA16F801848995890E94D96001
:108D5000F801C48BD58B168A80E090E0DF91CF912B
:108D60001F910F9108951F93CF93DF93EB018230F2
:108D7000910509F440C0833091052CF4009789F0E7
:108D8000019731F04CC0863091050CF048C02EC0E0
:108D90000E942C55FC01848163E00E949A718983B2
:108DA0003EC060E081E00E94A118898113E0819FAC
:108DB000802D11240E94F41982E090E00E94FA169E
:108DC00081B7612F0E949A71898399279F938F930E
:108DD00089E890E19F938F9382E08F930E947F1A9E
:108DE0000F900F900F900F900F9019C04FEE5FEF04
:108DF0000E94214314C08A81882359F00E942C5577
:108E0000398123E0329F90011124FC0124830E94C8
:108E1000B35490E08A81882309F491E09A8380E03A
:108E200090E0DF91CF911F9108951F93CF93DF932F
:108E3000EC018A81882309F45CC060E081E00E9433
:108E4000A1188C819D819F938F938DE890E19F93D2
:108E50008F9312E01F930E947F1A8B810F900F90C7
:108E60000F900F900F90843059F483E990E19F9315
:108E70008F931F930E947F1A0F900F900F9010C036
:108E8000888599279F938F9387E990E19F938F938C
:108E90001F930E947F1A0F900F900F900F900F90CA
:108EA000898D9A8D97FD03C06BE970E10AC08E5FD2
:108EB0009F4F19F463EA70E104C084E00E941A54E1
:108EC000BC0182E00E94291A81E0888F8E8B8B8101
:108ED00099278130910564F08330910524F004973F
:108EE000029730F402C083E001C088E08F8B01C09C
:108EF0001E8ADF91CF911F9108950F931F93CF93F7
:108F0000DF938C01FC018281882311F581E083834A
:108F1000643019F488E090E003C080E094E0F80148
:108F200086839783F8012481358186819781821712
:108F3000930724F481E090E08483958381E0F80135
:108F40008283683009F410C180E00E94450E0CC194
:108F5000F801848195819093410580934005C62F47
:108F6000DD27C430D10561F1C530D10594F4C1309D
:108F7000D10509F4C2C0C230D1051CF4209701F11B
:108F8000F3C0C230D10509F4BAC0239709F4E9C08F
:108F9000EBC0C730D10509F4B0C0C830D10544F4E6
:108FA000C530D10509F4A9C0C630D10549F0DCC0EF
:108FB000C830D10509F47EC0299709F49EC0D4C0F9
:108FC000F801838181508230E0F58EEF9FEF818F31
:108FD000928FC8010E9415476AE081E00E94A118A3
:108FE00089E00E941A54BC0182E00E94291AC43010
:108FF000D10581F0C530D1051CF4CD2B21F019C06D
:10900000269771F016C0F8018481958101970E941E
:10901000775E0CC0F801848181500E94975E06C083
:10902000F8018481958101970E94AC5EF801818FDF
:10903000928FF801818D928D97FD5DC0818D808723
:109040005AC06AE081E00E94A1188AE00E941A5486
:10905000BC0182E00E94291AC430D10589F0C530D4
:10906000D1051CF4CD2B21F046C02697C1F043C09A
:10907000F80184819581608501970E946D5E16C01C
:10908000F8018481958109971CF08FEF9FEF0FC045
:10909000F8018481608581500E948C5E07C0F801D0
:1090A00084819581608501970E94A25EF801818F7D
:1090B000928F21C00E94412AFC012081318121151B
:1090C0003105C9F08189992783709070039799F4CD
:1090D000F801648175816115710569F083818150A2
:1090E000823048F0615070404085C9010E94252AB5
:1090F000F801138239C081E035C084E033C0F80143
:1091000083818150823010F481E02DC06AE081E0DB
:109110000E94A118F8018381863079F489E00E94C9
:109120001A54BC0182E00E94291AF80184819581B9
:10913000618501970E94635E0FC08AE00E941A5405
:10914000BC0182E00E94291AF80184819581418D39
:10915000618501970E94595EF801818F928F86E0A8
:1091600001C087E0F8018383DF91CF911F910F91B8
:1091700008959C01FB018130910561F082309105D9
:109180001CF4892BD1F024C083309105E9F00597B8
:10919000C1F01EC08EEF9FEF818F928F40914005EE
:1091A00050914105CA0101978050944018F44483BE
:1091B00055830EC0248335830BC0CB010E94154715
:1091C00007C081E0838304C040E050E00E94214357
:1091D00080E090E008950F931F93CF93DF938C016D
:1091E000EB010E94412AFC0180819181892B31F0A1
:1091F0008189992783709070039761F060E081E026
:109200000E94A11885E00E941A54BC0182E00E94CD
:10921000291A1BC00230110541F00430110589F4F0
:1092200069E0CE010E947D4710C068E0CE010E9437
:109230007D478B81882349F40E94B0188FEF9FEF00
:1092400006C0BE01C8010E94B94880E090E0DF91ED
:10925000CF911F910F910895CF93DF93EB0182304F
:10926000910509F481C08330910534F40097A1F091
:109270008130910569F07CC08430910509F462C0A9
:10928000843091050CF46BC0059709F460C070C080
:109290000E94B94819866CC08A81882309F468C085
:1092A00060E081E00E94A1188B81882331F46BEA91
:1092B00070E182E00E94291A18C0898599279F933E
:1092C0008F938C819D819F938F938BEB90E19F93E4
:1092D0008F9382E08F930E947F1A8DB79EB7079677
:1092E0000FB6F8949EBF0FBE8DBF898D9A8D97FDE6
:1092F0000BC0823091051CF0029721F005C0898DCA
:10930000805D03C08FE301C085E40E94531881E0B3
:10931000888F8E8B8B8199278630910561F08730FD
:10932000910524F40197029758F403C0079729F098
:1093300007C086E003C08CE001C08EE08F8B18C0B0
:109340001E8A16C08B81863039F463E00EC08B8193
:10935000863011F481E001C086E08B8309C040E0D3
:1093600050E00E94214304C062E0CE010E947D478C
:1093700080E090E0DF91CF9108959B0182309105CC
:1093800029F08430910539F461E001C060E0C90141
:109390000E947D4702C00E94B94880E090E0089595
:1093A0009B018230910529F08430910539F465E004
:1093B00001C064E0C9010E947D4702C00E94B94813
:1093C00080E090E008959B018230910529F084307F
:1093D000910539F467E001C066E0C9010E947D474C
:1093E00002C00E94B94880E090E008951F93182FB2
:1093F00060E081E00E94A118812F992781309105BA
:1094000071F0823091051CF4892B39F013C0823041
:10941000910539F0039739F00DC08BE005C08CE061
:1094200003C08DE001C08EE00E941A54BC0182E0AE
:109430000E94291A1F910895CF93C82F1816B4F4CB
:1094400080E00E94F6496C2F80E090E00E946D5E03
:10945000892B39F440E065E08CE190E00E94595E90
:1094600007C08C2F0E94815E892B11F082E001C021
:1094700083E00E94F64984EF91E00E94FA16CF91B2
:109480000895CF93DF93EB0182309105E1F18330B2
:1094900091051CF4892B29F04EC08330910571F1A0
:1094A0004AC08A81882309F446C060E081E00E94B6
:1094B000A1188C819D8197FF0CC08AEC90E19F934D
:1094C0008F9382E08F930E947F1A0F900F900F90DE
:1094D0000FC09F938F938FEC90E19F938F9382E0C7
:1094E0008F930E947F1A0F900F900F900F900F9004
:1094F00083E08F8B81E0888F8E8B1DC040E050E031
:109500000E94214318C08A81882321F08C810E9407
:109510001C4A05C081E00E94F64981E08A8380E010
:1095200090E00E94775E8C839D8381E08B838FE740
:1095300090E08E839F8380E090E0DF91CF9108954B
:109540000F931F93CF93DF938B018130910571F0BF
:10955000823091051CF4892B79F0B4C082309105DA
:1095600009F43FC083309105B9F1ACC08FEF9FEF94
:10957000FB0184839583A6C0FB018281882309F4C3
:10958000A1C060E081E00E94A118F801848195816A
:1095900097FF0CC083ED90E19F938F9382E08F93B0
:1095A0000E947F1A0F900F900F900FC09F938F9380
:1095B0008AED90E19F938F9382E08F930E947F1AB0
:1095C0000F900F900F900F900F9085E0F801878B10
:1095D00081E0808F868B76C040E050E00E9421437E
:1095E00071C0FB018281882389F1C481D581C03893
:1095F000D10520F48C2F0E941C4A2EC0F8E2C03006
:10960000DF07A0F480E00E94F6498D2F9927806C37
:10961000682F80E190E00E946D5E009729F46C2F26
:1096200081E190E00E946D5E892B11F082E007C01D
:1096300041E065E08CE190E00E94595E83E00E9489
:10964000F64984EF91E00E94FA1606C081E00E947C
:10965000F64981E0F8018283F801848195810197C0
:109660008F37910540F480E090E00E94775EF8012A
:109670008483958315C080E190E00E94775E982FE7
:109680008827F8018483958381E190E00E94775ECA
:10969000F80124813581282B392B3F7324833583AE
:1096A000F80184819581805098422CF08FEF9FEFD4
:1096B000F8018483958381E0F80183838FEF97E23B
:1096C0008683978380E090E0DF91CF911F910F9187
:1096D00008951F93CF93DF93EB01122F82309105F2
:1096E00019F1833091052CF4009761F0019729F06E
:1096F0002EC0863091055CF512C0842F0E944D5516
:10970000898325C060E081E00E94A1188981810FD2
:109710000E947254BC0182E00E94291A18C042E0E3
:1097200050E00E94214313C08A81882351F089812F
:10973000882321F0842F0E94575503C0842F0E9454
:109740005F5590E08A81882309F491E09A8380E054
:1097500090E0DF91CF911F91089522E048E00E94B0
:10976000694B089520E041E00E94694B08950F93F2
:109770001F93CF93DF938C01EB0126E044E00E941E
:10978000694B0230110529F48A81882311F40E9463
:10979000991F80E090E0DF91CF911F910F91089584
:1097A0001F93CF93DF93EB018230910541F183301A
:1097B00091052CF4009789F0019729F03CC0863080
:1097C0009105CCF517C010E080E090E00E944A6A55
:1097D000039709F411E019832EC060E081E00E9434
:1097E000A11889818E5F0E947254BC0182E00E94A0
:1097F000291A21C042E050E00E9421431CC08A8106
:10980000882399F060E081E00E94A1186EED70E17C
:1098100082E00E94291A8981882319F083E090E070
:1098200002C081E090E00E947A6A90E08A818823F9
:1098300009F491E09A8380E090E0DF91CF911F914D
:1098400008950F931F93CF93DF939C01EB01823018
:10985000910509F46BC0833091052CF4009739F120
:10986000019731F097C0863091050CF093C059C034
:109870008C819D8101978C5F934010F02C833D83F8
:109880008CEF93E08E839F8311E01B831E8B83E01C
:109890008F8B188F00E08C819D81880F991F029714
:1098A0000E944A6A039709F4012F098373C060E09C
:1098B00081E00E94A1188B812C813D81813009F5C6
:1098C0002D5F3F4F3F932F938C819D819F938F936B
:1098D00080E393E09F938F9312E01F930E94531AAB
:1098E00089818C5F0E947254BC01812F0E94291AC9
:1098F0008DB79EB707960FB6F8949EBF0FBE8DBF6B
:1099000049C03F932F938AE393E09F938F9382E024
:109910008F930E94531A0F900F900F900F900F90FB
:1099200039C042E050E00E94214334C02A81222302
:10993000A1F089812C813D81882329F0220F331FDA
:1099400063E070E004C0220F331F61E070E0C901E2
:1099500002970E94926A1A821DC08B81813019F48D
:109960008A832E8B17C08C819D8101978C7F0196F5
:109970008C839D83122F880F991F02970E944A6A39
:10998000039709F411E0198391E09B839E8B83E098
:109990008F8B988F80E090E0DF91CF911F910F9196
:1099A0000895FF920F931F93CF93DF93EC018B01E8
:1099B000F42E0E942C55FC01C230D10509F471C06F
:1099C000C330D1052CF42097C9F0219771F07DC0E8
:1099D000C430D10509F44DC0C430D1050CF44DC0DC
:1099E000C530D10509F449C070C0FF2019F0848545
:1099F000E80155C08385F801818367C060E081E09C
:109A00000E94A118E8019981FF20F9F0892F6AE0EE
:109A10000E949A71892F99279F938F9389810E9421
:109A20009A7199279F938F938DEE90E19F938F93D7
:109A300082E08F930E947F1AEDB7FEB737960FB67C
:109A4000F894FEBF0FBEEDBF40C082E3989FC001F7
:109A500011249F938F9385EF90E19F938F9382E0E2
:109A60008F930E947F1A0F900F900F900F900F907E
:109A70002CC0F80181818F3F41F1FF2019F040E0B7
:109A80005FEF02C04BEE5FEFB801CE010E942143B1
:109A9000FF20D9F0E80189818823B9F481E0898326
:109AA00014C0E8018A81882341F09981FF2011F0D8
:109AB000948701C093870E94B35490E0F80182819B
:109AC000882309F491E0E8019A8380E090E0DF9137
:109AD000CF911F910F91FF90089540E00E94D14CCB
:109AE000089541E00E94D14C0895CF93DF93EB019C
:109AF0008230910559F1833091052CF4009759F08B
:109B0000019729F02FC08630910564F51AC00E9494
:109B10003455898327C060E081E00E94A1188981C3
:109B20009927880F991F880F991F8E5C984FBC0149
:109B300082E00E94291A6BEF70E182E00E94291AEC
:109B400011C048E050E00E9421430CC08A81882364
:109B500019F089810E94385590E08A81882309F4A0
:109B600091E09A8380E090E0DF91CF910895CF93C8
:109B7000DF93EB0182309105C1F18330910534F41C
:109B8000009749F08130910551F157C08630910519
:109B90000CF053C024C08A81882309F44EC061E0D0
:109BA00080E00E94A1188981885F0E947254BC01E4
:109BB00082E00E94291A60E081E00E94A118698178
:109BC000623020F082E10E941A5404C0862F845F24
:109BD0000E947254BC0182E00E94291A2EC042E009
:109BE00050E0BE010E94214328C08A81882319F1D8
:109BF0008981823018F48E5F89831FC060E081E024
:109C00000E94A1188981833051F48FE00E941A5478
:109C1000BC0182E00E94291A0E94926509C080E17D
:109C20000E941A54BC0182E00E94291A0E945A66BE
:109C30008FEF9FEF04C081E08A8380E090E0DF91A6
:109C4000CF910895CF9380913705803178F01092AD
:109C500037051092380561E0862F0E94A118CEE0EA
:109C600085EA0E945318C150C7FFFACF60913705AB
:109C700081E00E94A11880913805992781309105D3
:109C800059F0823091051CF4892B21F014C0029701
:109C900039F011C085E001C084E00E9453180BC068
:109CA00080E20E94531885E00E9453188091370586
:109CB0008F5F80933705809138058F5F80933805DB
:109CC000833010F010923805CF910895CF93DF9331
:109CD000EB018230910559F1833091051CF4892BF9
:109CE00031F053C0863091050CF04FC01BC08A8103
:109CF000882309F44AC061E080E00E94A11889E14C
:109D00000E941A54BC0182E00E94291A60E081E09E
:109D10000E94A11881E10E941A54BC0182E00E94B5
:109D2000291A33C040E050E00E9421432EC08A81AE
:109D3000882329F10E94571F64E971E084E00E94A2
:109D4000D0196CE871E085E00E94D01968EC70E0F1
:109D500082E29EE40E94DA1860E0862F0E94A11839
:109D600083E00E941A54BC0182E00E94291A0E94DA
:109D700019260E945D620E94D5540E94335790E0DC
:109D80008A81882309F491E09A8380E090E0DF9152
:109D9000CF910895CF92DF92EF92FF920F931F938E
:109DA000CF93DF93029709F0CEC060E0862F0E9428
:109DB000A11880E20E94531860E081E00E94A1187F
:109DC00080E00E94450E63E071E182E00E94291A62
:109DD00021E04EE468E086E00E94B90F6D9880E0D3
:109DE0000E94C21180E00E945C13CC24DD248EEF1F
:109DF0000E94CB1380E00E94AB1A8F5F9F4FD1F778
:109E000081E00E94AB1A8F5F9F4FD1F7A8950E9407
:109E100038188331910509F488C08B30910509F415
:109E200084C00A9701F581C0CF3FD10551F020973A
:109E300041F06C2F80E00E94F9196C2F81E00E94A4
:109E4000F919CF33D10519F0CB32D10519F4B4E8A3
:109E5000CB2ED12CC332D10511F0AA9721F4A6E064
:109E6000CA2EA1E0DA2E0E94F813EC018F5F9F4FFB
:109E7000D9F6C114D10409F4BACFE0903307F090B9
:109E80003407009135071091360788EC90E0A0E088
:109E9000B0E0E80EF91E0A1F1B1F3BC0A8950E94E8
:109EA000AB1AEC019FEFCF3FD90721F481E00E946C
:109EB000AB1AEC01AFEFCF3FDA0721F18C2F0E94F4
:109EC000CB130894C108D108E0903307F090340711
:109ED000009135071091360788EC90E0A0E0B0E0E3
:109EE000E80EF91E0A1F1B1F0DC0CF3FD10551F010
:109EF000209741F06C2F80E00E94F9196C2F81E0CF
:109F00000E94F9190E94F813EC019FEFCF3FD90787
:109F100061F7C114D10409F468CFC801B7010E94E8
:109F2000C314882309F4BACF60CF81E00E94C21124
:109F300081E00E945C136D9A0E94345521E04EE44A
:109F400068E00E94B90F80E090E0DF91CF911F910F
:109F50000F91FF90EF90DF90CF900895CF93DF9314
:109F6000EB018230910509F440C0833091052CF457
:109F7000009771F0019731F048C0863091050CF0E0
:109F800044C02EC00E942C55FC01868189833DC0AF
:109F900060E081E00E94A1186981662369F484E190
:109FA0000E941A549F938F9382E08F930E947F1A8E
:109FB0000F900F900F9029C085E0689FC001112479
:109FC0009F938F9380E191E19F938F9382E08F9392
:109FD0000E947F1A0F900F900F900F900F9015C056
:109FE00049EC50E00E94214310C08A81882339F057
:109FF0000E942C552981FC0126830E94B35490E0D5
:10A000008A81882309F491E09A8380E090E0DF91CF
:10A01000CF910895CF93DF93EB018130910569F0E3
:10A02000823091051CF4892B81F049C08230910562
:10A0300039F183309105F9F042C00E942C55FC01A2
:10A04000808599278C839D833AC060E081E00E94DF
:10A05000A1188C819D819F938F9386E191E19F93BD
:10A060008F9382E08F930E947F1A0F900F900F9032
:10A070000F900F9024C040E050E00E9421431FC089
:10A080008A81882361F483E08B8380E290E08E8371
:10A090009F8391E0988F82E08F8B9E8B0AC01E8AEF
:10A0A0000E942C552C81FC0120872093CA0A0E9413
:10A0B000B35490E08A81882309F491E09A8380E088
:10A0C00090E0DF91CF910895EF92FF920F931F934D
:10A0D000CF93DF938C01EB010E942C557C01023061
:10A0E000110509F463C00330110544F4011511058D
:10A0F00071F00130110509F446C072C0033011053A
:10A1000009F43DC0063011050CF06AC03CC08A81DC
:10A11000882309F465C0F7018085882309F460C0AD
:10A1200060E081E00E94A1188C819D819F938F93B4
:10A130008BE191E19F938F9382E08F930E947F1A2E
:10A1400060E089810E94B65E082F61E089810E94EB
:10A15000B65E182FC0E80F900F900F900F900F90E1
:10A1600094E0802F8C2309F096E0812F8C2309F056
:10A170009F5F892F0E945318C69591F731C01E8AA0
:10A1800081E00E94D75EF70180859927AC01BE016E
:10A19000C8010E9421438981992701968C839D8360
:10A1A0008B818230E9F488E08B831AC02A812223D4
:10A1B00091F481E090E08C839D83F701808599275D
:10A1C0008E839F8311E01A83822F0E94D75E188F9F
:10A1D00085E08F8B1E8B88E08B838C8181508983F7
:10A1E00080E090E0DF91CF911F910F91FF90EF9071
:10A1F0000895CF92DF92EF92FF920F931F93CF9328
:10A20000DF937C01C62F0E94C8190E942C556C0157
:10A21000C33208F06FC085E0C89F800111240A573F
:10A220001D4FF7018281882311F080E001C082E098
:10A230000E945318F6018581992781309105B1F06C
:10A24000823091051CF4892B39F031C082309105A0
:10A25000B9F00397F9F02BC08C2F992744E0880FB1
:10A26000991F4A95E1F7835C914F1DC08C2F992768
:10A2700034E0880F991F3A95E1F7835E934F13C03E
:10A280008C2F992724E0880F991F2A95E1F7835096
:10A29000964F09C08C2F9927C4E0880F991FCA9543
:10A2A000E1F78352984FBC0182E00E94291AE8012D
:10A2B0008C8187FD0BC060E081E00E94A1188C8139
:10A2C0000E941A54BC0182E00E94291AE801EA8126
:10A2D000FB81309721F0B70180E090E00995F7010C
:10A2E0008689882329F06789808D0E94AA1802C078
:10A2F0000E94B018DF91CF911F910F91FF90EF90C6
:10A30000DF90CF90089560E0E6E8F2E0482F55270F
:10A3100047FD509520E030E080819927841795070C
:10A3200011F4C90108956F5F2F5F3F4F3596623278
:10A3300098F38FEF9FEF08950895BF92CF92DF9229
:10A34000EF92FF920F931F93CF93DF93CDB7DEB7BA
:10A350006B970FB6F894DEBF0FBECDBFB82E21E2CB
:10A36000281718F480E090E0FBC16E010894C11C2E
:10A37000D11C8BE1F60111928A95E9F7A89585E049
:10A38000B89EF0011124EA57FD4F0280F381E02DC1
:10A39000309721F0B60181E090E009956B2DC60160
:10A3A0000E94F9500E94880E85E0B89E7001112429
:10A3B00086E892E0E80EF91E0E943818AC018A3057
:10A3C000910509F4E9C08B30910564F4009709F414
:10A3D0000AC1181619060CF41EC14F5F5F4F09F42D
:10A3E000AEC1E0CF8331910509F48EC0843191056F
:10A3F00044F48B30910509F487C0419709F49BC15F
:10A40000D1CF8431910519F0459751F1CBCFF601A9
:10A410008281882381F0F701228133812115310562
:10A4200031F0BE016F5F7F4F84E090E081C1F601A3
:10A4300081818F5F28C0F601868BF7019081F0E261
:10A44000FB1534F0F7018581891711F4B39431C0FD
:10A45000892F0E948351682F772767FD709540C030
:10A46000F6018281882389F0F70122813381211549
:10A47000310531F0BE016F5F7F4F85E090E058C13C
:10A48000F60181818150818367C1F601868B6B2D36
:10A49000F7019081BB2091F02BEF3FEFE20EF31E0E
:10A4A000F701808125E030E0E20EF31E891731F4D8
:10A4B000BA946B2D772767FD709512C030E23B157B
:10A4C00064F0D7011596F7018581891731F46F5F24
:10A4D00061321CF415968C91F8CF772767FD709543
:10A4E000B62E85E0689FF0011124EA57FD4F0280E7
:10A4F000F381E02D309709F42FC1BE016F5F7F4FCC
:10A5000081E090E0099528C1F7019181992361F1DB
:10A51000092F1127075C1A4FF801808118162CF0BB
:10A52000892F0E948351F8018083F7018181E82FF0
:10A53000FF27E75CFA4F80810E949D51282F332727
:10A5400027FD3095F7018181E82FFF27E75CFA4F5F
:10A55000C90137FF04C088279927821B930B80838A
:10A5600037FFFAC0B1943AC0F70122813381211537
:10A57000310551F0BE016F5F7F4F82E090E0F9013D
:10A58000099599237CF319C0F6018281882309F487
:10A5900091E0F6019283E0C0F60182818823F1F018
:10A5A000F7012281338121153105A9F0BE016F5FCA
:10A5B0007F4F83E090E0F9010995F60182818823BD
:10A5C00009F0CAC0F70122813381BE016F5F7F4F5E
:10A5D00081E090E0ADC0F6011282BEC08B2D9927BC
:10A5E00087FD9095BDC0F6018381813009F4DACEF4
:10A5F000883089F481E00E94D75E60E0F6018181B5
:10A600000E94B65E61E0F60181810E94B65E80E044
:10A610000E94D75EA1C0F6018381992785309105FC
:10A6200009F454C08630910584F48230910581F19B
:10A63000833091051CF40197B9F08EC083309105E9
:10A6400099F0049709F43EC087C08730910509F45A
:10A6500056C0873091050CF44CC08830910521F02C
:10A66000099709F453C078C0F60186819781892B38
:10A6700021F48FEF9FE786839783F6018681978188
:10A68000841795070CF468C01482158282E08383D6
:10A69000F601848195819C0163E0220F331F6A9546
:10A6A000E1F7280F391F280F391F240F351F37FDF9
:10A6B00053C086819781821793070CF44DC0248381
:10A6C00035834AC0F601108685E08383F6019085C4
:10A6D0008AE0989F90011124240F351F2F3F3105E8
:10A6E00009F008F420878EEF9FEFF601818F928F9B
:10A6F00033C04830510584F5F60141872DC0423002
:10A70000510554F5F601418F528F26C0F601818123
:10A71000E80FF11D842F805D8287F701228133814C
:10A7200021153105C9F0BE016F5F7F4F82E090E0D7
:10A73000F901099511C080E00E94450E0DC0F60197
:10A740008381883009F02ECEBE016F5F7F4F80E09D
:10A7500090E00E94645026CE6B2DCE01019620CE53
:10A760006B960FB6F894DEBF0FBECDBFDF91CF91D1
:10A770001F910F91FF90EF90DF90CF90BF900895C1
:10A78000CF93C82F6CE571E080E00E94D01964E699
:10A7900071E082E00E94D01964E871E084E00E94D8
:10A7A000D0196CE771E085E00E94D01964E771E090
:10A7B00086E00E94D0196CE671E087E00E94D01913
:10A7C00080913905823210F010923905C7FD04C01E
:10A7D0008C2F0E949D510EC0809139050E949D5181
:10A7E000992787FD909597FF03C0909581959F4F7E
:10A7F000809339056CE372E080E00E94D0196CE12F
:10A8000072E082E00E94D01964EF71E084E00E945F
:10A81000D0196CEE71E085E00E94D01964EE71E011
:10A8200086E00E94D0196CED71E087E00E94D0199B
:10A83000CF910895CF93C82F8B3118F085E19CE11B
:10A840002CC00E942C55FC018581992782309105EE
:10A8500081F0833091051CF4019721F018C0039713
:10A8600079F015C081E1C89FC0011124865B954E27
:10A8700014C081E1C89FC00111248158974E0DC0BA
:10A8800081E1C89FC00111248C54994E06C081E11A
:10A89000C89FC001112487519B4ECF9108958823F2
:10A8A00019F082E29CE108950E942C55FC018581FB
:10A8B00099278230910561F0833091051CF401974E
:10A8C00021F00CC0039739F009C088ED94E1089598
:10A8D00087EC94E1089586EB94E1089585EA94E18C
:10A8E00008950895CF93C82F8E3018F082E39CE12D
:10A8F00038C00E942C55FC01858199278230910532
:10A9000099F0833091051CF4019721F021C0039741
:10A91000A9F01EC08C2F992754E0880F991F5A95D3
:10A92000E1F78B539C4E1DC08C2F992744E0880F74
:10A93000991F4A95E1F78B519D4E13C08C2F992793
:10A9400034E0880F991F3A95E1F78B5F9D4E09C05F
:10A950008C2F992724E0880F991F2A95E1F78B5DAA
:10A960009E4ECF910895EF92FF921F93CF93DF9366
:10A9700082E4E82E85E0F82EC0E0D0E01FE1CE01B1
:10A980000E943B6CF70161917F01861719F0CE019F
:10A990000E94546CA8951150219617FFF0CFDF91BB
:10A9A000CF911F91FF90EF900895909147059430BB
:10A9B00008F091E08FE0E2E4F5E011928A95E9F782
:10A9C00088E1809346059093470581E08093430595
:10A9D00084E18093480582E080934D0582E3809373
:10A9E0004E050E94B354089540E250E060E070E0EC
:10A9F00082E495E00E94436C809144059091450566
:10AA00008F5F9F4F11F40E94D55480914305883089
:10AA100018F081E08093430580914F059091500597
:10AA2000885F974020F01092500510924F0580915A
:10AA30004705843010F0109247058AEF9FEFA1E0A0
:10AA4000B0E0ABBFFC0187918F3F21F0882311F06C
:10AA500080936F000895089582E495E008958093AF
:10AA600047050E94B354089580914305992708959E
:10AA7000CF93C82F883008F0C7E080914305C817EE
:10AA800051F0C09343050E94B35421E04EE468E0C6
:10AA90008C2F0E94B90FCF91089520E030E0909163
:10AAA0004205982311F021E030E0C901089590910A
:10AAB0004205982B909342050E94B3540895982F15
:10AAC0009095809142058923809342050E94B3545A
:10AAD00008958CEF9FEFA1E0B0E0ABBFFC01879140
:10AAE0009791A791B691B070BC01CD0108958FEFF9
:10AAF0009FEFA1E0B0E0ABBFFC01879199270895DB
:10AB00000E944926FC01892BB9F0A2E6B5E043E09A
:10AB10002D913C911197808191812817390729F057
:10AB2000828193812817390719F41D921C9211977D
:10AB30004150139647FFECCF089508959F92AF922E
:10AB4000BF92CF92DF92EF92FF920F931F93CF931A
:10AB5000DF93CDB7DEB726970FB6F894DEBF0FBEF2
:10AB6000CDBFC82E7B01942ECE0101960E94655761
:10AB7000DD2492E6A92E95E0B92EF5018081918120
:10AB80008E159F0509F096C082818F5F8283843085
:10AB900008F4C5C0C7010E941C278C01009709F466
:10ABA000C0C0FFEFCF1639F5992029F0FC01648170
:10ABB0007581C7011BC0FC01448155816681C701B5
:10ABC0000E94E62AC7010E94BC61BC01F801808591
:10ABD0000E94472BF80182819381009749F00E94DF
:10ABE0001C27FC0164817581808191810E94302B3A
:10ABF0000E94532A59C0992049F0FC014481558193
:10AC000060E0CE0101960E94485741C0FC0144819A
:10AC100055816681CE0101960E944857AE014F5F73
:10AC20005F4F67E08C2D0E94E857F80180858F7791
:10AC30008B83C7010E94BC61BC01CE0104960E94B7
:10AC400065570E94FE578823E1F3AE014F5F5F4FC7
:10AC500069E08C2D0E94E857F801828193810E945F
:10AC600049268C010097D1F0FC0160817181CE01F1
:10AC700001960E946557F8014481558160E0CE013C
:10AC800001960E9448570E94FE578823E1F3AE01C7
:10AC90004F5F5F4F68E08C2D0E94E85740E050E026
:10ACA0006DE08C2D0E94E857F5011082118281E041
:10ACB00090E037C0D39483E090E0A80EB91E93E0F3
:10ACC0009D1508F05ACFDD2402E615E0F8018081D9
:10ACD0009181892BA1F40E94442A8E159F0519F4B5
:10ACE0000E94592A07C0AE014F5F5F4F65E08FEFAA
:10ACF0000E94E857F801E082F182128206C0D394E4
:10AD00000D5F1F4FF3E0FD1508F783E08D1538F454
:10AD1000AE014F5F5F4F66E08FEF0E94E85780E023
:10AD200090E026960FB6F894DEBF0FBECDBFDF9140
:10AD3000CF911F910F91FF90EF90DF90CF90BF9038
:10AD4000AF909F9008950F931F93CF93DF93082F99
:10AD5000EB01672B79F010E040E0BE01802F0E94EC
:10AD60009E55882339F40E94FE578823E1F31F5F24
:10AD7000143190F3DF91CF911F910F9108958F922D
:10AD80009F92BF92CF92DF92EF92FF920F931F9309
:10AD9000CF93DF93CDB7DEB726970FB6F894DEBF1B
:10ADA0000FBECDBFB82E4B016A01CB010E941C27FC
:10ADB0008C01892B09F445C0C6010E941C277C0127
:10ADC000892B09F43EC0F80180850E94382A8C0145
:10ADD000F70180850E94382A081B190BC80117FF4C
:10ADE00003C0909581959F4F0297E4F0FFEFBF1647
:10ADF00021F481E00E94B82B24C086E0FE01319648
:10AE000011928A95E9F781E08983AE014F5F5F4F28
:10AE100061E28B2D0E94E85714C0B601C4010E9464
:10AE20006B290FC010E041E0B6018B2D0E949E55AA
:10AE3000882399F70E94FE578823E1F31F5F14319E
:10AE400090F326960FB6F894DEBF0FBECDBFDF910C
:10AE5000CF911F910F91FF90EF90DF90CF90BF9017
:10AE60009F908F9008950E94571FF894FFCF6827F6
:10AE700090E027E0862F86959F5F60FF03C0682FD4
:10AE8000622701C0682F9830A8F3862F992708956C
:10AE9000FC01262F862F8F77828326952074CA0186
:10AEA000892F9927869586958F73822B8383CA0174
:10AEB00023E0969587952A95E1F78F778483842FF1
:10AEC0008295807F8F7785830895FC01CB01262FA3
:10AED0002F772083880F892F881F990B91958F7763
:10AEE00081830895803480F4E82FFF27662329F0BA
:10AEF000EB55FA4F8AE080830895EB55FA4F808135
:10AF0000882311F08150808308950895EF92FF9275
:10AF10000F931F93CF93DF93782FC62F7A01A895B5
:10AF200080919205282F33278091930599270197C7
:10AF30002817390741F080919205833039F48091C8
:10AF40009305882319F480E090E03BC0909192052E
:10AF500089E0989F8001112402591A4F872F806839
:10AF6000F8018083682F80E00E943757F801C18381
:10AF70006C2F0E943757982FE801229605E0E114C4
:10AF8000F10431F0F70181917F018F77888301C04F
:10AF900018826991892F0E943757982F015007FF17
:10AFA000EECF87FD90959883809192058F5F809377
:10AFB000920580919205843010F01092920581E004
:10AFC00090E0DF91CF911F910F91FF90EF90089546
:10AFD0000F931F93CF93DF93082F162FEA0102C020
:10AFE0000E94880EAE01612F802F0E948657882311
:10AFF000B9F3DF91CF911F910F9108959F92AF9276
:10B00000BF92CF92DF92EF92FF920F931F93CF9355
:10B01000DF93CDB7DEB76C970FB6F894DEBF0FBEE7
:10B02000CDBF992458C227FF05C010929B058FEF12
:10B0300080939D0580919B05893040F4E82FFF2780
:10B04000E456FA4F20838F5F80939B0580919B0588
:10B05000893009F040C280919C0587FF3CC24CE9D1
:10B06000E42E45E0F42E90E017E0F70181917F0196
:10B07000682F892F0E943757982F115017FFF5CF4F
:10B0800087FD90958091A405981709F01FC2FF24B1
:10B0900080919C0588230CF019C23FE7B32EB8229B
:10B0A00030919E05C32EDD2440919F05842F992762
:10B0B0009695982F882797958795C82AD92A209101
:10B0C0009D05822F9927AA27BB27FC013197E334DE
:10B0D000F10508F0FBC1EA5BFF4FEE0FFF1F059083
:10B0E000F491E02D09941091A0058091A105282FDD
:10B0F000332726FD1068322F2227330F330F80911C
:10B10000A20599278F77907003E0880F991F0A9501
:10B11000E1F7282B392B8091A30599278077907030
:10B12000B4E095958795BA95E1F7282B392B41E046
:10B13000B901C6010E94302941E0612FC6010E9479
:10B14000AA28C6010E948055BDC18091A0059927FB
:10B1500090E4899F902D88271124C82AD92A6091CC
:10B16000A105662319F041E0642F01C041E0C6014A
:10B170000E94ED68A7C18091A005682F7727809174
:10B18000A105282F3327C901877090709695982FB5
:10B19000882797958795682B792B20743070220F1C
:10B1A000331F8091A205822B482FC6010E94252AB9
:10B1B00089C18091A005E82EFF24002711278091E6
:10B1C000A10599279695982F882797958795AA275F
:10B1D00097FDA095BA2FE82AF92A0A2B1B2B8091FC
:10B1E000A205992790E4899F902D88271124AA27EA
:10B1F00097FDA095BA2FE82AF92A0A2B1B2B20913C
:10B20000A305822F9927AA27BB2787709070A0706B
:10B21000B07035E1880F991FAA1FBB1F3A95D1F76F
:10B22000E82AF92A0A2B1B2B269526952695D80164
:10B23000C7010197A109B1098F5F9F4FAF4FB04080
:10B2400008F040C1A601C801B7010E943C653AC19F
:10B250000E94840E843009F435C180919E050E94BD
:10B26000450E882309F42EC184E00E94D86B2AC1C0
:10B27000C114D10409F426C1B6018B2D0E94A35636
:10B2800021C16091A005C6010E94B72780919E054B
:10B290008A8780919F058B87C6010E9499278C879A
:10B2A000AE01465F5F4F69E0A7C01AE0E12EF12CC6
:10B2B000EC0EFD1EAE01405F5F4FBE01645F7F4F2D
:10B2C000C6010E947C616C018F778A87CC0CCD2CE3
:10B2D000CC1CDD08D1948C2D8F778B8788898D8746
:10B2E00089898E871F86A70161E18B2D0E94E8570F
:10B2F0008E010F5F1F4FF80194E081898187915083
:10B30000319697FFFACFA70162E18B2D0E94E85793
:10B31000F80193E0868981879150319697FFFACFA3
:10B32000A70163E169C0A3E0FA2E33E0F30E83E0E6
:10B33000F80E8601243199F48091A005C82EDD24F1
:10B340008091A10599279695982F8827979587959D
:10B35000C82AD92A8091A2058C8F188A23C0AE01F1
:10B36000405F5F4FBE01645E7F4FC6010E947C61FB
:10B370006C0194E0EAE0EF1588F0DE01AF0DB11D3D
:10B380005096E92FFF27E456FA4F80818D939F5FF7
:10B39000F394973018F4FAE0FF1598F7FE01EF0DDB
:10B3A000F11D108A9E01205F3F4F4C8DB601C801F0
:10B3B0000E94DC608C018F778A87000F012F001FAD
:10B3C000110B1195802F12C0213121F4C6010E946A
:10B3D000FF6103C0C6010E9434626C018F778A87C7
:10B3E000CC0CCD2CCC1CDD08D1948C2D8F778B8789
:10B3F000AE01465F5F4F60E18B2D0E94E85762C04F
:10B40000C6010E94D9605EC08091A005282F332715
:10B410008091A10599279695982F882797958795CC
:10B42000282B392BA901B6018B2D0E94BF564AC08B
:10B43000C6010E94902946C0BB24E5EAF5E081914F
:10B44000882369F44EE955E064E08B2D0E94E857AB
:10B45000809195058B1538F4B092950504C0B3948E
:10B460003FE33B1560F782E0809396052BC0809107
:10B470009605833038F583E08093960530939705E1
:10B48000409398058091A0058093990510929A05A4
:10B4900019C0809196058230A8F482E080939605C9
:10B4A0003093970540939805109299050BC09091A1
:10B4B0009605992339F481E080939605309397059A
:10B4C0009093980561E08B2D0E94725710929B0516
:10B4D0008FEF80939D050E94F8139C018FEF2F3F03
:10B4E000380709F0A0CD0E94BA130A970CF421C1C5
:10B4F0009091920580919305981711F19091930581
:10B5000089E0989F70011124EEE6F5E0EE0EFF1E33
:10B5100008E010E0F70181917F010E94CB130150F8
:10B52000104017FFF7CF809193058F5F80939305AD
:10B5300080919305843008F4FCC010929305F9C003
:10B540007E010894E11CF11C570180919405803420
:10B5500029F060919605662309F475C08FEF898301
:10B560000894E11CF11C8091960599278130910582
:10B57000C9F0823091051CF4892B39F059C0823012
:10B58000910519F10397C1F153C080E4F70181934C
:10B5900080919705982F97708F5F8093970591936F
:10B5A0007F0148C081E4F7018193809197058770FE
:10B5B000819380919805982F9F778F5F809398054E
:10B5C00091937F018091980531C082E4F7018193C6
:10B5D0008091970587708193809198058F778193EB
:10B5E00080919905982F9F778F5F8093990591930C
:10B5F0007F01809199051AC083E4F70181938091BE
:10B60000970587708193809198058F7781938091BA
:10B6100099058F77819380919A05982F9F778F5FF7
:10B6200080939A0591937F0180919A0587FF02C0CC
:10B630001092960580919605882309F059C0809153
:10B6400094058F5F53C08134A1F58FEF89830894EF
:10B65000E11CF11C83E0F70181937F018F010894C5
:10B66000E11CF11C0E94840E8F77F8018083809189
:10B6700094058F5F809394050E94412A8C01FC0100
:10B68000808981FF13C0808191810E94805541E0B3
:10B69000F8016289808191810E94AA2841E0F80125
:10B6A00066817781808191810E94302951E0952EB9
:10B6B0001FC0803410F060939405809194058068D9
:10B6C00089830894E11CF11C82E0F70181937F01DA
:10B6D000809194050E947257809194058F5F8093AA
:10B6E000940590919505981718F480E4809394053B
:10B6F000CE010996E816F90620F4F70111927F01B0
:10B70000F9CFDD24750107E010E0F70160818D2D90
:10B710000E943757D82EF70181917F010E94CB13E9
:10B720000150104017FFF1CFD7FCD0948D2D0E940F
:10B73000CB13A895892D99276C960FB6F894DEBF88
:10B740000FBECDBFDF91CF911F910F91FF90EF9072
:10B75000DF90CF90BF90AF909F900895CF93DF93ED
:10B76000CDB7DEB726970FB6F894DEBF0FBECDBFBC
:10B7700036E0FE01319611923A95E9F74983AE0120
:10B780004F5F5F4F0E94E85726960FB6F894DEBFD2
:10B790000FBECDBFDF91CF9108951F93CF93DF935D
:10B7A000EC0110E001C0A8950E94B71F8823D9F3CF
:10B7B00010C0A89504C081E090E00E94FA160E9493
:10B7C000B71F8823C1F361E080E090E00E94DC1D98
:10B7D00021970E94C71F882311F4209751F70E94D8
:10B7E000C71F811111E0C5E00EC063E080E090E06A
:10B7F0000E94DC1D0E94CB1F01C0A8950E94B71FAC
:10B800008823D9F3C1500E94C71F882311F0CC238D
:10B8100061F7CC2309F41C2F812F9927DF91CF9159
:10B820001F910895EF92FF921F93CF93DF937C01B6
:10B83000CFEFDFEF10E0612FC7010E94551E80E0BF
:10B8400090E00E94CD5B882311F0C12FDD271F3FC0
:10B8500049F483E090E00E94CD5B882331F0CFEF84
:10B86000D0E005C01F5FD7FDE6CFD7FD14C01C2F69
:10B87000CFEFDFEF612FC7010E94551E83E090E0FC
:10B880000E94CD5B882311F0C12FDD27112319F011
:10B890001150D7FDEFCFCE01DF91CF911F91FF90D7
:10B8A000EF9008954F925F926F927F928F929F9246
:10B8B000AF92BF92CF92DF92EF92FF920F931F93BE
:10B8C000CF93DF93CDB7DEB726970FB6F894DEBFE0
:10B8D0000FBECDBF782E5B01C42E522E402E80911C
:10B8E000620082608093620080E00E94F41986E02A
:10B8F000FE01319611928A95E9F7AE014F5F5F4FD5
:10B9000062E28FEF0E94E8570E94D81F83EC87B94C
:10B910008FEE86B96FEF862E962E662480E00E9409
:10B92000450E82E390E00E94FA1684E00E94450EE4
:10B9300084E690E00E94FA16E0903307F090340716
:10B94000009135071091360780ED97E0A0E0B0E058
:10B95000E80EF91E0A1F1B1FDD241092E605109247
:10B96000E5052BC00E94D31FAC012091E505309165
:10B97000E605C901885A9D4F8417950734F0C9011F
:10B98000885592404817590744F45093E605409370
:10B99000E505DD2059F0DA9409C0240F351F3595EF
:10B9A00027953093E6052093E505D39494E09D1503
:10B9B00050F08AE090E00E94FA16C801B7010E9498
:10B9C000C314882379F28091E5059091E6054497A8
:10B9D0005CF584E393E00E94CE1F83E090E00E9438
:10B9E000CD5B10E0412F612F80E090E00E941C1E93
:10B9F00083E090E00E94CD5B811111E041E060E0C6
:10BA000080E090E00E941C1E83E090E00E94CD5BED
:10BA100081111F5F113041F484E190E09093E605BD
:10BA20008093E50545E0D42E8091E5059091E605EB
:10BA30004497855A9B4028F4B4E0BD1510F144208A
:10BA400001F560E081E00E94A1188091E5059091E8
:10BA5000E6058431910514F485E106C0895B9B40BD
:10BA600014F086E101C087E10E941A54BC0182E013
:10BA70000E94291A80E00E94450E88EE93E00E9401
:10BA8000FA168091E5059091E605805E9C4F0E9434
:10BA9000CE1F86E990E00E94FA160E94840E843040
:10BAA00009F0D8C0072D11270330110509F447C04C
:10BAB000043011054CF40130110539F10230110543
:10BAC000FCF4012B71F0ACC0053011050CF4A8C0DA
:10BAD000073011050CF453C0093011050CF0A0C05B
:10BAE0006FC0452D6C2DC5010E94FC1D8FE090E0BC
:10BAF0000E94CD5B882309F497C0852C992494C0BB
:10BB00006C2DC5010E946E1E4CC040E06C2DC5011D
:10BB10000E941C1E83E090E00E94CD5B882309F008
:10BB200046C041E06C2DC5010E941C1E83E090E0E0
:10BB30000E94CD5B882309F477C0480177C010E0EC
:10BB4000012F169540E0602FC5010E941C1E83E066
:10BB500090E00E94CD5B882309F410680F5F0830E5
:10BB600080F3612FC5010E94871E83E090E00E9450
:10BB7000CD5B882309F458C0812E992455C061E01B
:10BB800085E090E00E943C1E8FE090E00E94CD5B3B
:10BB9000C50187709070F5E07F1661F46C2D0E94EE
:10BBA0003C1E8FE090E00E94CD5B8823E9F1882461
:10BBB00099243CC00E94125C4C0133E0632E34C0D7
:10BBC000C5019695879596958795682F6F5F85E057
:10BBD00090E00E943C1E8FE090E00E94CD5BC5018A
:10BBE0008370907027E0721661F46C2D0E943C1EE9
:10BBF0008FE090E00E94CD5B882341F08824992457
:10BC000005C00E94125C4C0193E0692E61E085E062
:10BC100090E00E943C1E8FE090E00E94CD5B04C04B
:10BC20008FEF882E982E08C097FC06C0442021F084
:10BC30008CE291E00E94FA1680E00E94450E97FE89
:10BC400009C08CE291E00E94FA16639482E08615A6
:10BC500008F064CE16B886B187B90E942C55FC0155
:10BC600084810E94F41981E08983AE014F5F5F4FA8
:10BC700062E28FEF0E94E857809162008D7F80938F
:10BC80006200C40126960FB6F894DEBF0FBECDBF8A
:10BC9000DF91CF911F910F91FF90EF90DF90CF90A8
:10BCA000BF90AF909F908F907F906F905F904F90DC
:10BCB00008950F93242F01E0462FBC0180E00E94DD
:10BCC000525C0F9108950F9300E0202F462FBC0186
:10BCD00081E00E94525C0F9108950F9301E020E0F3
:10BCE000462FBC0182E00E94525C0F9108950F9391
:10BCF00000E0202F402FBC0183E00E94525C0F9196
:10BD000008950F9301E020E0482F60E070E085E0A7
:10BD10000E94525C0F9108950F93992701E020E053
:10BD2000462FBC0185E00E94525C0F9108950F934D
:10BD3000992700E0202F402FBC0186E00E94525C32
:10BD40000F9108950F9301E020E0462FBC0187E09A
:10BD50000E94525C0F9108950F9300E0202F402F16
:10BD6000BC0188E00E94525C0F910895880F611118
:10BD70008F5FF894E82FFF27E45FF44F9081809164
:10BD8000CB0A80FD10827894892F99270895880F17
:10BD900061118F5FF894E82FFF27DF01A45BB44F98
:10BDA0008C91E453F54F808378949927089590916E
:10BDB000CB0A882311F0916001C09E7F9093CB0A3B
:10BDC0000895089580E4ECECFAE011928A95E9F781
:10BDD000089584E0809374001092710082E2809351
:10BDE000700008951F920F920FB60F9211248F9337
:10BDF0009F93EF93FF93809171009927887F9070B4
:10BE00008032910509F487C0813291056CF480314C
:10BE10009105D9F0813191051CF40897D1F07DC0CE
:10BE2000489709F43FC079C080349105A9F1813465
:10BE3000910524F4889709F441C06FC080359105BD
:10BE4000D9F08835910561F068C08091E70587FFDA
:10BE500002C080EA01C081EA8093730085E861C076
:10BE6000E091ED05F091EE05809173008193F093E0
:10BE7000EE05E093ED0548C0E091ED05F091EE058B
:10BE8000809173008193F093EE05E093ED0580912E
:10BE9000E80581508093E8058091E8058230F4F24E
:10BEA00085EC3FC08091EB059091EC05892F992797
:10BEB000809373008FEF8093E705D0CF8091E705E3
:10BEC00087FF09C08091EB059091EC05809373008A
:10BED0001092E705C3CF8091E9058823E1F08091B6
:10BEE000E805882389F0E091ED05F091EE05819158
:10BEF000F093EE05E093ED05809373008091E805E3
:10BF000081508093E805AACF84E98093740081E092
:10BF10008093EA0508C085EA04C08FEF8093EA05A4
:10BF200084E980937400FF91EF919F918F910F901E
:10BF30000FBE0F901F9018958091740099278770FD
:10BF40009070009711F081E090E00895089560935B
:10BF5000E8059093EC058093EB052093E905509359
:10BF6000EE054093ED058EEF8093E7051092EA050C
:10BF700085EA8093740008958091EA05992787FDEA
:10BF8000909508950E94A75F01C0A8950E94BC5F8C
:10BF9000892BD9F38091EA05992787FD909508951B
:10BFA000AB0120E060E134E0880F991F3A95E1F79A
:10BFB0000E94C25F0895AB0121E060E174E0880F48
:10BFC000991F7A95E1F70E94C25F089520E0AC01C5
:10BFD00066E080E090E00E94C25F089521E0AC013D
:10BFE00066E080E090E00E94C25F0895EF92FF92C9
:10BFF0000F931F93CF93DF93CDB7DEB722970FB682
:10C00000F894DEBF0FBECDBF7C0119821A82098170
:10C010001A8120E0AE014F5F5F4F62E0C801E4E0AB
:10C02000880F991FEA95E1F70E94C25FA895898160
:10C030009A81009719F08E159F0549F7C80122963D
:10C040000FB6F894DEBF0FBECDBFDF91CF911F9129
:10C050000F91FF90EF9008950F931F93CF93DF936D
:10C06000CDB7DEB722970FB6F894DEBF0FBECDBFB7
:10C070008C0101978F5F934000F520E0AE014F5F88
:10C080005F4F62E0C801A4E0880F991FAA95E1F70D
:10C090000E94C25FC8010E94F65F24E080309207D0
:10C0A00060F421E0AE014F5F5F4F62E0F4E0880F83
:10C0B000991FFA95E1F70E94C25F22960FB6F89495
:10C0C000DEBF0FBECDBFDF91CF911F910F910895BD
:10C0D000EF92FF920F931F93CF93DF93CDB7DEB70D
:10C0E00066970FB6F894DEBF0FBECDBF7C010197F7
:10C0F0008F5F9340F8F4C7010E942C60CE01019637
:10C100000E94E65F8E01095F1F4F40E150E06FEF34
:10C1100070E0C8010E94746C8B819C818F8398872A
:10C12000B801C7010E94DB5FEB82FC82CE01019661
:10C130000E94EE5F66960FB6F894DEBF0FBECDBFCD
:10C14000DF91CF911F910F91FF90EF9008950F9382
:10C150001F93CF93DF93CDB7DEB726970FB6F89432
:10C16000DEBF0FBECDBFCE0101960E94E65F0B8100
:10C170001C810115110589F020E0AE014D5F5F4F74
:10C1800062E0C801B4E0880F991FBA95E1F70E94F8
:10C19000C25FCE0101960E94EE5FC80126960FB6DF
:10C1A000F894DEBF0FBECDBFDF91CF911F910F91ED
:10C1B00008950E94686008959F92AF92BF92CF92B7
:10C1C000DF92EF92FF920F931F93CF93DF93CDB740
:10C1D000DEB7A8970FB6F894DEBF0FBECDBF8C01B7
:10C1E0006B01942E7901232B99F0672B89F084E061
:10C1F0000030180768F40115110521F0C8010E94EC
:10C200002C6003C00E94A7608C010115110511F478
:10C21000C80158C05E010894A11CB11CF701CB8273
:10C22000DC829D82DE0116962081222351F0CE0110
:10C230004196A817B90728F431962D93208122231F
:10C24000C1F7C5014096A817B90708F41C920FA3BF
:10C2500018A7CE0141960E94E65FEE24FF240989CB
:10C260001A8901151105B1F0A895BE01695E7F4FCD
:10C27000C8010E94D05FC50105964BE050E0BC01AB
:10C28000CE014C960E94BD6C992324F478010F894D
:10C29000188DE7CFF50100831183A895B5018FA113
:10C2A00098A50E94DB5F21E0AE01495D5F4F62E02F
:10C2B000C70114E0880F991F1A95E1F70E94C25F29
:10C2C0008FA198A5A8960FB6F894DEBF0FBECDBF7C
:10C2D000DF91CF911F910F91FF90EF90DF90CF9062
:10C2E000BF90AF909F9008959A01462FBC0180E0C7
:10C2F00090E00E94DC600895EF92FF920F931F93ED
:10C30000CF93DF93CDB7DEB760970FB6F894DEBF5B
:10C310000FBECDBF9C017B018A0101978F5F9340C7
:10C3200018F080E090E01BC0BE016F5F7F4FC90135
:10C330000E94D05FE114F10419F08D81F701808330
:10C340000115110551F08BE0F801DE0116960D90F4
:10C3500001928A95E1F7F80113868B819C816096A2
:10C360000FB6F894DEBF0FBECDBFDF91CF911F9106
:10C370000F91FF90EF900895EF92FF920F931F930C
:10C38000CF93DF93CDB7DEB766970FB6F894DEBFD5
:10C390000FBECDBF7C01CE0101960E94E65F0981F0
:10C3A0001A811BC08FEF0F3F1807D1F020E0AE01BC
:10C3B000495F5F4F64E0C801062E02C0880F991FD5
:10C3C0000A94E2F70E94C25F89859A858E159F05BF
:10C3D00011F4C80107C00F8118850115110511F767
:10C3E00080E090E066960FB6F894DEBF0FBECDBF3A
:10C3F000DF91CF911F910F91FF90EF9008950F93D0
:10C400001F93CF93DF93CDB7DEB766970FB6F8943F
:10C41000DEBF0FBECDBF8C018150944018F080E08C
:10C4200090E017C0CE0101960E94E65F011511054C
:10C4300071F0BE01695F7F4FC8010E94D05F8F819C
:10C440009885009721F02FEF8F3F920711F4898193
:10C450009A8166960FB6F894DEBF0FBECDBFDF910E
:10C46000CF911F910F910895CF93DF93CDB7DEB792
:10C4700026970FB6F894DEBF0FBECDBF24E0813003
:10C48000920718F080E090E00FC0009739F4CE01D9
:10C4900001960E94E65F89819A8106C00E94F65F3C
:10C4A000009711F40E94F65F26960FB6F894DEBF4F
:10C4B0000FBECDBFDF91CF910895CF92DF92EF9263
:10C4C000FF920F931F93CF93DF93CDB7DEB766979D
:10C4D0000FB6F894DEBF0FBECDBF1D821E8219823B
:10C4E0001A8201E010E00B831C83A895CE01800F17
:10C4F000911F0E94EE5F97E0C92ED12CCC0EDD1E5D
:10C5000040E150E06FEF70E0C6010E94746C80E182
:10C51000E82EF12C83E00F3F18073CF40F5F1F4F0C
:10C520000F8318870150104002C01F8218860E9496
:10C53000880E21E0A60160E1C7010E94C25F0F5F83
:10C540001F4F80E190E0E80EF91E94E000301907DB
:10C550000CF366960FB6F894DEBF0FBECDBFDF9129
:10C56000CF911F910F91FF90EF90DF90CF900895A2
:10C57000EF92FF920F931F93CF93DF93CDB7DEB768
:10C5800066970FB6F894DEBF0FBECDBFCE01019601
:10C590000E94E65F89E00E947617882329F08EE0EA
:10C5A0000E947617882351F48B819C818F5F9F4F67
:10C5B00021F589819A818F5F9F4FF9F464E971E0D9
:10C5C00084E00E94D0196CE871E085E00E94D019E7
:10C5D00068EC70E082E29EE40E94DA1860E0862F48
:10C5E0000E94A11883E00E941A54BC0182E00E94BC
:10C5F000291A0E945D620E94335709811A81C8017D
:10C6000001978F5F9340A0F4BE01695F7F4FC8011F
:10C610000E94D05FEF80F88489859A8501978F5FAB
:10C62000974218F0C8010E9468608701A895E7CF7B
:10C630008D819E818F5F9F4F51F4CE0101960E94A4
:10C64000E65F1D821E82CE0101960E94EE5F669615
:10C650000FB6F894DEBF0FBECDBFDF91CF911F9113
:10C660000F91FF90EF900895CF92DF92EF92FF929B
:10C670000F931F93CF93DF93CDB7DEB726970FB6F7
:10C68000F894DEBF0FBECDBF6C017B01CE010196D9
:10C690000E94E65F0D811E8124E00030120718F031
:10C6A00027C0C80127C0C80101978F5F934000F5DC
:10C6B000A89520E0A70160E1C80134E0880F991F28
:10C6C0003A95E1F70E94C25F20E0F701329681912E
:10C6D00091919F778C159D0521F32F5F2730B8F33B
:10C6E000F70100811181C80101978F5F934000F32A
:10C6F00080E090E026960FB6F894DEBF0FBECDBF67
:10C70000DF91CF911F910F91FF90EF90DF90CF902D
:10C7100008959F92AF92BF92CF92DF92EF92FF92D5
:10C720000F931F93CF93DF93CDB7DEB760970FB60C
:10C73000F894DEBF0FBECDBF0091EF05002319F0C6
:10C7400080E090E04EC0BE016F5F7F4F0E94346377
:10C75000009709F446C011E01093EF05AB80BC8050
:10C7600045E0C42ED12CCC0EDD1EC5010E941C2735
:10C77000FC01892B91F1902E868187FD912EE12E6F
:10C78000F601808191818C011F77F92EFF1CFF2417
:10C79000FF1CC80101978E5F9742B8F4C8010E9440
:10C7A0001C27FC01892BC9F0FF2021F086819920EC
:10C7B00031F403C08681992011F0806801C08F7721
:10C7C0008683B801C5010E946B29E39482E090E062
:10C7D000C80ED91E96E09E1598F61092EF0581E0DE
:10C7E00090E060960FB6F894DEBF0FBECDBFDF912C
:10C7F000CF911F910F91FF90EF90DF90CF90BF905E
:10C80000AF909F9008956F927F928F929F92AF9278
:10C81000BF92CF92DF92EF92FF920F931F93CF932D
:10C82000DF93CDB7DEB766970FB6F894DEBF0FBEC5
:10C83000CDBF6C01F090EF05FF2019F080E090E093
:10C8400087C00E9449268C01009709F481C0FC0131
:10C8500082819381009709F47BC08F2CF801868137
:10C8600087FF02C0B1E08B2EA7E06A2E712C6C0E00
:10C870007D1EB301C6010E9434637C015C01892BDB
:10C88000C9F40E94A7607C01892B09F460C0CE0125
:10C8900001960E94E65F8D819E818F8398878050EC
:10C8A000944010F0AF82B886ED82FE82CE010196F0
:10C8B0000E94EE5F8EE0FE01399611928A95E9F7AB
:10C8C000C986DA86F1E09F2EF801828193818C156A
:10C8D0009D0591F1E2E0AE2EB12C0E9449268C011B
:10C8E000009751F1BE016F5F7F4F6A0D7B1DDC0128
:10C8F0002D913C91FB012087318740E050E0FC0105
:10C90000868187FF02C041E050E0882D99274817B3
:10C91000590721F03068FB0120873187939482E02A
:10C9200090E0A80EB91EF801828193818C159D05B7
:10C9300019F0F6E0F91588F621E0A30160E1C701DE
:10C9400074E0880F991F7A95E1F70E94C25FC701D2
:10C9500066960FB6F894DEBF0FBECDBFDF91CF91C4
:10C960001F910F91FF90EF90DF90CF90BF90AF900D
:10C970009F908F907F906F900895EF92FF920F930A
:10C980001F93CF93DF93CDB7DEB7A0970FB6F89480
:10C99000DEBF0FBECDBFBE01695F7F4F0E94346313
:10C9A0007C01892B09F45BC0CE0147960E94E65FAB
:10C9B0000B8D1C8D0E151F0519F400E010E01AC038
:10C9C00001151105A9F0A89520E0AE01435E5F4F67
:10C9D00062E0C80134E0880F991F3A95E1F70E94A0
:10C9E000C25F8D8D9E8D8E159F0521F08C01E8CF45
:10C9F0000FEF1FEF84E00030180788F58F819885CE
:10CA00008F8F98A3CE0101960E94E65F0115110554
:10CA100029F48F8D98A18D839E830DC021E0AE01F6
:10CA2000415E5F4F62E0C80104E0880F991F0A95DC
:10CA3000E1F70E94C25FA89521E0AE014D5F5F4F14
:10CA400062E0C70114E0880F991F1A95E1F70E9470
:10CA5000C25FEB82FC82CE0101960E94EE5FA0963F
:10CA60000FB6F894DEBF0FBECDBFDF91CF911F91FF
:10CA70000F91FF90EF900895EF92FF920F931F9305
:10CA8000CF93DF93CDB7DEB728970FB6F894DEBF0C
:10CA90000FBECDBF7B018C01FA018091F005909112
:10CAA000F105892B91F1E982FA820B831C831F82A5
:10CAB0001886022F112700FF09C04F83588740E0D6
:10CAC00050E0BA01CF010E947C61FC0101FF05C06A
:10CAD0008F81988590688F839887ED83FE83EF2BF5
:10CAE000A1F021E0AE014F5F5F4F68E08091F0055B
:10CAF0009091F1050E94C25F8091F0059091F1053F
:10CB000008969093F1058093F00528960FB6F89457
:10CB1000DEBF0FBECDBFDF91CF911F910F91FF9070
:10CB2000EF900895CF92DF92EF92FF921F93CF93F1
:10CB3000DF93CDB7DEB728970FB6F894DEBF0FBEF0
:10CB4000CDBF10E0C12C30E4D32E8091C90A181754
:10CB500098F5812F9927FC0123E0EE0FFF1F2A95FE
:10CB6000E1F7E80FF91FE80FF91FE75BF74F808146
:10CB7000918189839A83828193818B839C83848131
:10CB800095818D839E838085282F33272F83388737
:10CB9000868187FD03C031602F83388721E0AE0195
:10CBA0004F5F5F4F68E0C6010E94C25F1F5F88E071
:10CBB00090E0C80ED91EC9CF0E942C552FEF3FEF31
:10CBC00029833A83FC01858596858B839C8321E0AC
:10CBD000AE014F5F5F4F68E0C6010E94C25F88E010
:10CBE00090E0C80ED91E0E94412AFC01D092F105A6
:10CBF000C092F005848995892089892B41F020FF16
:10CC000002C023E001C021E04489558907C020FF0C
:10CC100002C022E001C020E04081518160E070E06C
:10CC200080E090E00E943C6510E040E050E06BE066
:10CC3000812F0E94E8571F5F1034B8F310E00E9464
:10CC4000FE578823E1F31F5F1630C8F310E0212F51
:10CC50004FEF5FEF6FEF7FEF8FEF9FEF0E943C652D
:10CC6000C090F005D090F1051092F1051092F005FA
:10CC70008CE8E82E8BE0F82E1FE121E0A70168E0A8
:10CC8000C6010E94C25F1150E8E0F0E0EE0EFF1E08
:10CC9000CE0EDF1E17FFF1CF28960FB6F894DEBF39
:10CCA0000FBECDBFDF91CF911F91FF90EF90DF902E
:10CCB000CF9008957F928F929F92AF92BF92CF9222
:10CCC000DF92EF92FF920F931F93CF93DF93CDB735
:10CCD000DEB76C970FB6F894DEBF0FBECDBF0E94D3
:10CCE000840E782E80E00E94450E40E050E060E027
:10CCF000CA010E94E62A86E08E010F5E1F4FF801EE
:10CD000011928A95E9F7FF24A80167E08F2D0E9410
:10CD1000E85784E190E00E94FA16F3942FE32F1570
:10CD200098F70E94012619821A82A12C00E4B02EE5
:10CD300020E0AE014F5F5F4F68E0C5010E94C25F17
:10CD400089819A81EFEF8F3F9E07E1F00E941C27B7
:10CD50008C01892BB9F08F818F70682FF801808149
:10CD600091810E94B7278B819C81F80182839383F4
:10CD70008D819E81848395838F819885892F9927C2
:10CD800080FD168288E090E0A80EB91E89819A8104
:10CD90008F5F9F4F69F619861A861B861C86B9E03D
:10CDA0008B2E912C8C0E9D1E20E0A40168E0C50105
:10CDB0000E94C25F89859A85AB85BC858050904072
:10CDC000A040B14008F0AAC08D859E85009709F467
:10CDD000A5C028E28030920708F0A0C0FF242F856C
:10CDE000388937FF02C0A2E0FA2E8C0121153105E7
:10CDF00089F089011F7740E050E0BA01C8010E9424
:10CE00007C612D853E852817390719F481E0F82AC1
:10CE100001C08901F4012081318142815381CF2CED
:10CE2000DD242115310541055105D1F50E94412A26
:10CE30007C01C0FE08C04696AC0160E070E0C8010D
:10CE40000E947C618C01C8010E9449268C010097D8
:10CE5000E1F0FC01448155816681808191810E94CD
:10CE6000E62A60E070E0F80180850E94472BF80117
:10CE7000828193810E944926009739F0FC016481E8
:10CE80007581808191810E94302BC1FE04C0F70121
:10CE900080898160808BF70180898260808B3EC0B1
:10CEA000802F8F778F8B000F012F001F110B119593
:10CEB000802F8F77888FF40180818F77898FE7E0CB
:10CEC0005695479537952795EA95D1F7822F8F7715
:10CED0008A8F77E056954795379527957A95D1F7BC
:10CEE000822F8F778B8F67E05695479537952795DB
:10CEF0006A95D1F7822F877053E0CC0CDD1C5A95D0
:10CF0000E1F78C298C8FAE01495E5F4F6CE08FEFAB
:10CF10000E94E8570E94FE578823E1F388E090E0E2
:10CF2000A80EB91E89859A85AB85BC858050904036
:10CF3000A040B14008F433CF0CE81BE04FE1F42EE1
:10CF400020E0A80168E0C5010E94C25FFA94085F72
:10CF50001F4F88E090E0A80EB91EF7FEF1CF83E0E6
:10CF60000E94450E84E690E00E94FA168B819C8117
:10CF70000E94DF6A872D0E94450E6C960FB6F894CA
:10CF8000DEBF0FBECDBFDF91CF911F910F91FF90FC
:10CF9000EF90DF90CF90BF90AF909F908F907F9059
:10CFA00008952FEF3FEFE2EFF5E08FE1208331832B
:10CFB0003796815087FFFACF0895AC01FC0123E03A
:10CFC000F695E7952A95E1F7E457F44F8081992784
:10CFD0009A012770307002C0959587952A95E2F7DF
:10CFE000440F551F382F317080FF02C04F5F5F4FD5
:10CFF00020E0E2EFF5E0808191818417950759F4F4
:10D00000868180FF0CC0332319F082E590E00895FB
:10D0100087E490E008952F5F3796203260F3332342
:10D0200019F082E790E0089587E690E0089508956A
:10D030001F93CF93DF93EC01162F892B09F4A2C025
:10D04000662319F08E8180FD9DC0112309F481C0F3
:10D050008091D2069091D306A091D406B091D506C6
:10D060008896A11DB11DBC01CD010E94C314882367
:10D0700009F488C04881598190E0E2EFF5E0BA01F7
:10D08000B3E076956795BA95E1F7208131818FEF0E
:10D090002F3F380779F02417350761F0868180FF2C
:10D0A00009C0A3E036952795AA95E1F7261737071B
:10D0B00009F468C09F5F3796903238F361E0888149
:10D0C00099810E94C71D8091330790913407A091E8
:10D0D0003507B09136078A839B83AC83BD838093E9
:10D0E000D2069093D306A093D406B093D5068E8132
:10D0F00081608E8383FF06C088819981969587958C
:10D100000E94DE6B48815981CA0164E0969587953B
:10D110006A95E1F7682F9A01369527952770307048
:10D1200081E090E002C0880F991F2A95E2F7982FBE
:10D13000772740FF06C0FB01E457F44F8081892B1D
:10D1400006C0FB01E457F44F9095808189238083CA
:10D150003EC08E8182608E83992780FF13C082FF3C
:10D1600011C08091D2069091D306A091D406B091BF
:10D17000D5068896A11DB11DBC01CD010E94C31426
:10D18000882319F480E090E024C0612F8881998180
:10D190000E94C71D8091330790913407A0913507F5
:10D1A000B09136078093D2069093D306A093D4060D
:10D1B000B093D5068E8183FF06C0888199819695AC
:10D1C00087950E94DE6B8FEF9FEF8883998381E0C4
:10D1D00090E0DF91CF911F910895DF92EF92FF923F
:10D1E0000F931F93CF93DF93CDB7DEB726970FB67C
:10D1F000F894DEBF0FBECDBF8C01D62E805F9F405E
:10D2000018F080E090E06FC020E0E2EFF5E0808170
:10D2100091818017910731F12F5F37962032B8F353
:10D22000DD2089F41CC00083118380913307909125
:10D230003407A0913507B091360782839383A48386
:10D24000B58316820FC020E0E2EFF5E08081918186
:10D250008F5F9F4F41F32F5F37962032B8F3EE2454
:10D26000FF2403C07F01309721F4C701DD20D9F5E9
:10D2700038C0442319F08681886086830E942C552B
:10D28000FC01DD2061F0980136952795858596850E
:10D290008217930720F4258736870E94B3546D2D9B
:10D2A000C7010E941868802F8F778983000F012F94
:10D2B000001F110B1195802F8F778A83000F012F8C
:10D2C000001F110B1195802F8F778B8380E0D11079
:10D2D00081E08C83AE014F5F5F4F63E28FEF0E946E
:10D2E000E85781E090E026960FB6F894DEBF0FBEB7
:10D2F000CDBFDF91CF911F910F91FF90EF90DF9005
:10D3000008956F927F928F929F92AF92BF92CF9229
:10D31000DF92EF92FF920F931F93CF93DF930E94C0
:10D320002C558C01FC0183859927AA27BB27BC01BA
:10D33000CD0122E330E040E050E00E947B716B01C0
:10D340007C01F80184859927AA27BB27BC01CD0160
:10D3500024E630E040E050E00E947B713B014C014C
:10D36000AA24BB24C2EFD5E00FE1888199818F5FA9
:10D370009F4F51F18E81992780FF14C082FD24C0F8
:10D380008A819B81AC81BD818C0D9D1DAE1DBF1D11
:10D39000BC01CD010E94C3148823B1F08E8184604A
:10D3A0008E8312C0A114B10471F0F5012281338182
:10D3B000448155818A819B81AC81BD81821793070D
:10D3C000A407B50708F45E010150279607FFCDCFEB
:10D3D0008091D2069091D306A091D406B091D50643
:10D3E0008896A11DB11DBC01CD010E94C3148823E4
:10D3F00099F08091330790913407A0913507B0914F
:10D4000036078897A109B1098093D2069093D30675
:10D41000A093D406B093D50600E0C2EFD5E0888192
:10D4200099818F5F9F4FE1F08E81992780FF18C00F
:10D4300082FF16C081FD0EC08A819B81AC81BD81B7
:10D44000860D971DA81DB91DBC01CD010E94C314F6
:10D45000882331F060E0CE010E941868882359F4D7
:10D460000F5F27960032D8F2A114B10421F061E0D9
:10D47000C5010E941868DF91CF911F910F91FF9015
:10D48000EF90DF90CF90BF90AF909F908F907F9064
:10D490006F900895CF93DF93EC018FE0C03FD807E2
:10D4A00018F08FEF9FEF23C0D695C79583E0CD3F4F
:10D4B000D807C0F4D695C795D695C795CE0153E049
:10D4C000969587955A95E1F78452904F0E943B6C50
:10D4D0009927C770D07002C095958795CA95E2F7D5
:10D4E00080FF03C083E090E002C081E090E0DF9124
:10D4F000CF9108951F93CF93DF93039711F41FEFFC
:10D5000001C010E0CCEDDFE0A895612FCE010E94B4
:10D51000546C21968FE0CC3FD807B4F3DF91CF91C4
:10D520001F910895EF92FF920F931F93CF93DF9374
:10D53000EC018B018FE0C03FD807D0F56330710557
:10D5400019F061307105A1F5D695C79583E0CD3FFF
:10D55000D80770F5D695C795D695C7957E01E3E0B7
:10D56000F694E794EA95E1F7C7018452904F0E9440
:10D570003B6C682F9E01277030700330110549F411
:10D5800081E090E002C0880F991F2A95E2F7682B8E
:10D5900009C081E090E002C0880F991F2A95E2F748
:10D5A00080956823A895C7018452904F0E94546CBF
:10D5B000DF91CF911F910F91FF90EF9008959F926F
:10D5C000AF92BF92CF92DF92EF92FF920F931F9391
:10D5D000CF93DF937C0188EFE81687E0F80608F028
:10D5E00076C00E942C555C01FC01E586F6860E94FF
:10D5F000B354CC24DD249924092D1127E016F1061B
:10D6000008F450C0C801C3E096958795CA95E1F724
:10D61000482F98012770307081E090E002C0880F99
:10D62000991F2A95E2F7982FE801CC0FDD1FE42F10
:10D63000FF27E457F44F8081892309F0219640E0C9
:10D6400061E0CE010E94ED6840E0642FCE010E94AF
:10D65000ED6860E081E00E94A1180894E11CF11CD3
:10D66000FF92EF920894E108F1080894C11CD11CC4
:10D67000DF92CF9288E10E941A549F938F9382E0A9
:10D680008F930E947F1A84E690E00E94FA168DB76D
:10D690009EB707960FB6F8949EBF0FBE8DBF0C5F66
:10D6A0001F4FACCFF501838599270E94FA169394FA
:10D6B000F3E0F91508F0A0CF84E690E00E94FA1696
:10D6C00002C00E94880E0E94B71F8823D1F3DF9109
:10D6D000CF911F910F91FF90EF90DF90CF90BF906F
:10D6E000AF909F900895EF92FF920F931F93CF9367
:10D6F000DF938091D606682F77271092D606ECE844
:10D70000FCE08191882311F0706805C08DE0EB3852
:10D71000F807B9F3B4F340E050E08091C90A9927C3
:10D72000481759079CF4DC019A01F901E40FF51F31
:10D73000E75BF74F878180FF02C0706407C04F5FCF
:10D740005F4F275F3F4F4A175B077CF340E050E095
:10D750008091CA0A9927880F991F4817590704F51D
:10D760007C01ECE0FBE00CEC1AE0CCE4DBE099910E
:10D77000D8018D918D01981759F48081282F332776
:10D78000892F99278095909528233923232B11F0F1
:10D79000706206C04F5F5F4F31964E155F053CF3D8
:10D7A000CB01DF91CF911F910F91FF90EF900895E2
:10D7B0009091D606982B9093D60608959C0187E009
:10D7C000283F3807A0F4F90183E0F695E7958A959C
:10D7D000E1F7E457F34F2770307081E090E002C02A
:10D7E000880F991F2A95E2F72081282B208308951E
:10D7F000089528E28030920740F40E944926FC01F7
:10D80000892B19F087818160878308950895CF93CC
:10D81000DF931092D60680E091E0ECE8FCE01192F4
:10D820000197E9F7CCECDAE0ACE4BBE0ECE0FBE03C
:10D830008091CA0A9927880F991F009741F09C018F
:10D840008D919191892B899321503040C9F7E9E45A
:10D85000F8E08091C90A9927009751F09C018781CF
:10D860008E7F8783215030403A9621153105B9F7D4
:10D87000DF91CF910895E199FECF9FBB8EBBE09AD7
:10D8800099278DB308954115510569F0DC01E1999F
:10D89000FECF7FBB6EBBE09A6F5F7F4F0DB20D92E4
:10D8A00041505040B1F70895E199FECF9FBB8EBB28
:10D8B0006DBB0FB6F894E29AE19A0FBE0895411538
:10D8C000510589F0DC018FB7E199FECF7FBB6EBBBC
:10D8D0000D900DBAF894E29AE19A8FBF6F5F7F4F77
:10D8E0004150504089F70895DC0101C06D934150CB
:10D8F0005040E0F708950F931F93CF93DF93CDB778
:10D90000DEB72C970FB6F894DEBF0FBECDBF0B89E4
:10D910001C89ED89FE893EE03C8309831A834FEF21
:10D920005FE74D835E83AE01495E5F4FBF01CE016D
:10D9300001960E94366E2F813885020F131FD80181
:10D940001C922C960FB6F894DEBF0FBECDBFDF91B0
:10D95000CF911F910F910895FB01DC018D910190F2
:10D96000801911F40020D1F7990B0895FB01DC0117
:10D9700001900D920020E1F70895FB01DC01415078
:10D98000504030F08D910190801919F40020B9F7C2
:10D99000881B990B0895FB01DC014150504030F089
:10D9A0008D910590801919F40020B9F7881B990B07
:10D9B00008952F923F924F925F926F927F929F9223
:10D9C000AF92BF92CF92DF92EF92FF920F931F938D
:10D9D000CF93DF93CDB7DEB76E970FB6F894DEBF67
:10D9E0000FBECDBF898B9A8B6B8B7C8B4D8B5E8BE7
:10D9F0003C011F8A188EF30191903F01892D9927D0
:10DA00000E94F571892BB9F70DE2901609F4FFC059
:10DA10001BE2911609F4F7C02D893E8921153105C5
:10DA200009F4DAC02031310509F4D6C0ED89FE8948
:10DA3000EF2B41F430E3931609F4C9C04AE050E0FB
:10DA40004D8B5E8B8D899E89AA2797FDA095BA2F55
:10DA5000898F9A8FAB8FBC8F8F89988D892B09F412
:10DA6000B1C060E070E080E090E8298D3A8D4B8D88
:10DA70005C8D0E94267229873A874B875C876D8769
:10DA80007E878F87988B58E0DE011196FE013996CC
:10DA900001900D925A95E1F7CC24DD247601AA2459
:10DAA000BB2429803A804B805C802D813E812D8F64
:10DAB0003E8F092D1127C8010E94E971892BC9F1F8
:10DAC000C8010E94EE71892B09F46BC070ED970EAE
:10DAD000892D99276D897E898617970754F5B7FC9C
:10DAE00024C02C143D044E045F04F8F0C214D30487
:10DAF000E404F504A9F021E0A22EB12CC701B6017F
:10DB0000298D3A8D4B8D5C8D0E947B716B017C0160
:10DB1000C90CD11CE11CF11CD3019D903D01C9CF62
:10DB2000AD8CBE8CA816B90634F73FEFA32EB32EEA
:10DB3000F3CFB7FE29C0EF89F88DEF2BE1F0C12CB0
:10DB4000D12CE12C90E8F92E02E210E010938D0D1B
:10DB500000938C0D8B899C89892B09F460C0AB28BC
:10DB600039F0C3010197AB89BC898D939C9357C051
:10DB700089899A89F8CF8FEFC82E8FEFD82E8FEF33
:10DB8000E82E8FE7F82EE0CFAF89B88DAB2B11F3DD
:10DB9000F094E094D094C094C11CD11CE11CF11C01
:10DBA000D9CFC8010E94CF71892B19F2C8010E94F8
:10DBB000CD71892B21F0802F8753982E89CF802F0C
:10DBC0008755FBCF6FEF7FEF8FEF9FE74ECF08E0DA
:10DBD00010E00D8B1E8B36CF40E3941609F026CF54
:10DBE000F3018081883719F0883509F01FCFD30100
:10DBF00011969C9082E090E0680E791E60E170E0E2
:10DC00006D8B7E8B13CFD3019D903D0105CF21E01D
:10DC100030E02F8B388FF30191903F01FDCEC7018B
:10DC2000B6016E960FB6F894DEBF0FBECDBFDF9182
:10DC3000CF911F910F91FF90EF90DF90CF90BF9009
:10DC4000AF909F907F906F905F904F903F902F90FC
:10DC50000895DC015C91552341F05F7D51341CF047
:10DC60005B350CF45C931196F5CF08952F923F929B
:10DC70004F925F926F927F928F929F92AF92BF92DC
:10DC8000CF92DF92EF92FF920F931F93CF93DF9388
:10DC9000CDB7DEB762970FB6F894DEBF0FBECDBF2B
:10DCA000AA24BB2465014C016D877E874F87588B62
:10DCB00044245524FC0146825782838181FD5BC246
:10DCC0008FEF9FEF6FC240FE44C2862D80538A3093
:10DCD000E0F4F0E36F1641F42A89222329F4772037
:10DCE00019F480E091E08BC08AE09A89989F902D8A
:10DCF0001124892F860D80538A8B882314F4EFE733
:10DD0000EA8B43FC38C27A8836C243FE05C0FA89E2
:10DD1000FF2311F421E02A8B862D992787FD90950A
:10DD20008836910554F5853691050CF06BC0883521
:10DD3000910509F4D3C089359105B4F48B3291056E
:10DD400009F442C08C32910544F48032910509F403
:10DD50003FC0839709F442C0F2C18D329105D9F1D9
:10DD60008E9709F440C0EBC18336910509F454C085
:10DD70008436910509F478C0E2C18037910509F431
:10DD8000A5C08137910584F48C369105B1F18D36AB
:10DD900091052CF48936910509F466C0D0C18F36FF
:10DDA000910509F490C0CBC18537910509F498C05D
:10DDB0008637910524F483379105B9F1C0C18837BE
:10DDC000910509F48BC0BBC180E190E0482A592A33
:10DDD000E0E2F0E005C080E890E011C0E0E4F0E0AF
:10DDE0004E2A5F2AC8C188E090E0482A592AEFEFFE
:10DDF000FEEF4E225F221A8ABEC184E090E0482ADC
:10DE0000592AB9C10F2EFFE3AF2EF02D7A940F2EB1
:10DE1000F3E66F2EF02D3AC1EF85F889CF01029617
:10DE20008F87988BA0807A9431C1EF85F889CF01D4
:10DE300002968F87988BA080B18043FE0BC0EA8941
:10DE40008E2F992787FD9095BC01C5010E947071A6
:10DE5000898B07C0F50101900020E9F73197EA1995
:10DE6000E98BF9897F1A12C142FE0BC0EF85F88950
:10DE7000CF0104968F87988B208131814281538115
:10DE80000DC0EF85F889CF0102968F87988B80812E
:10DE900091819C01442737FD4095542F59016A0117
:10DEA000552364F4E2E0F0E04E2A5F2AD094C09457
:10DEB000B094A094A11CB11CC11CD11C8FEB9FEF8E
:10DEC000482259222BC098E0998B0AC0E0E4F0E088
:10DED0004E2A5F2A0F2EF8E76F2EF02DF0E1F98B16
:10DEE00042FE0BC0EF85F889CF0104968F87988B8F
:10DEF00020813181428153810BC0EF85F889CF01A8
:10DF000002968F87988B808191819C0144275527A9
:10DF100059016A01EFECFFEF4E225F221E010894C7
:10DF2000211C311CF989EF2EFF2400271127C6017F
:10DF3000B501A80197010E940472DC01CB01F10137
:10DF400080838A301CF0860D815203C0F1018081EC
:10DF5000805DF10181931F01C601B501A801970100
:10DF60000E94047259016A012115310541055105CC
:10DF7000F1F6CE010196A22CA81AC201827390700C
:10DF8000892B09F07A9446FE0FC0872D992787FDCB
:10DF90009095F989F03131F40F2EFEEF7F2EF02DA0
:10DFA000780E02C0782E7A9443FE12C08A89282FF8
:10DFB000332727FD30958A2D9927821793072CF058
:10DFC000E7EFFFEF4E225F2203C0FA89FA19FA8BBE
:10DFD00043FE03C02A89721A01C07A18C2018078F0
:10DFE0009170892B69F4872D7A9418164CF4B4013A
:10DFF00080E290E00E943D71872D7A941816BCF360
:10E0000041FE04C0B4018DE290E00BC044FE04C0A8
:10E01000B4018BE290E005C045FE05C0B40180E28A
:10E0200090E00E943D7146FE0FC0B40180E390E095
:10E030000E943D718989803139F4862D992787FDA9
:10E040009095B4010E943D7150FE0DC0872D7A94C9
:10E0500018164CF4B40180E390E00E943D71872DC6
:10E060007A941816BCF343FE11C08A89982F9150F8
:10E070009A8B18165CF4B40180E390E00E943D7125
:10E080008A89E82FE150EA8B1816ACF3842D80784A
:10E0900069F4872D7A9418164CF4B40180E290E06C
:10E0A0000E943D71872D7A941816BCF3F3E66F1623
:10E0B00041F48A2D992787FD9095B4010E943D7106
:10E0C0002DC023E76216B1F489898150898B8F3F77
:10E0D00029F1F5018081992787FD90950894A11C6D
:10E0E000B11CB4010E943D7199899150998B9F3F59
:10E0F00081F714C0CE0101962816390679F08E01F9
:10E100000F5F1F4FF10182911F01992787FD9095A5
:10E11000B4010E943D7120163106A1F7842D80784C
:10E12000A9F0872D7A9418168CF4B40180E290E05F
:10E130000E943D71872D7A941816BCF307C0862D76
:10E14000992787FD9095B4010E943D714424552480
:10E1500012C0F5E26F1641F44424552443941A8A00
:10E160007A882AE0298B07C0862D992787FD90950C
:10E17000B4010E943D71F401838183FF08C0ED85E5
:10E18000FE85CF0101968D879E87649005C0ED8541
:10E19000FE856190ED87FE87662009F094CDF4013D
:10E1A0008681978162960FB6F894DEBF0FBECDBF11
:10E1B000DF91CF911F910F91FF90EF90DF90CF9063
:10E1C000BF90AF909F908F907F906F905F904F9097
:10E1D0003F902F9008950F931F93CF93DF93CDB768
:10E1E000DEB72C970FB6F894DEBF0FBECDBF8C0103
:10E1F00036E03C8389839A832FEF3FE72D833E836C
:10E20000CE0101960E94366EAF81B885A00FB11F76
:10E210001C922C960FB6F894DEBF0FBECDBFDF91D7
:10E22000CF911F910F9108950F931F93CF93DF9379
:10E23000CDB7DEB72C970FB6F894DEBF0FBECDBFBB
:10E240008C013EE03C8389839A832FEF3FE72D8347
:10E250003E83CE0101960E94366EAF81B885A00F35
:10E26000B11F1C922C960FB6F894DEBF0FBECDBF27
:10E27000DF91CF911F910F9108950F931F93CF932B
:10E28000DF938C01EB018B81992781FF22C082FFF4
:10E2900014C02E813F814C815D81241735073CF4E9
:10E2A000A881B9810D93A883B9832E813F812F5F07
:10E2B0003F4F2E833F83C8010EC0E885F985802F2C
:10E2C0000995892B31F4EE81FF813196EE83FF832E
:10E2D000F2CF8FEF9FEFDF91CF911F910F910895B4
:10E2E000FC016150704001900110D8F78095909525
:10E2F0008E0F9F1F0895629FD001739FF001829F30
:10E30000E00DF11D649FE00DF11D929FF00D839FC4
:10E31000F00D749FF00D659FF00D9927729FB00D61
:10E32000E11DF91F639FB00DE11DF91FBD01CF0174
:10E3300011240895991B79E004C0991F961708F0DD
:10E34000961B881F7A95C9F78095089597FB092E2B
:10E3500007260AD077FD04D00CD006D000201AF48E
:10E36000709561957F4F0895F6F7909581959F4F31
:10E370000895AA1BBB1B51E107C0AA1FBB1FA6170C
:10E38000B70710F0A61BB70B881F991F5A95A9F75E
:10E3900080959095BC01CD01089585FD17C08062E0
:10E3A0009923A1F4813694F08B3784F4089599234E
:10E3B00069F4803269F0893059F08B3039F408956E
:10E3C0008F93EDDF8F9109F0806208959927882758
:10E3D00008959923D9F78095807808959923B1F706
:10E3E0008033A4F38A3394F70895992379F7803220
:10E3F00079F38A3069F38C3059F38D3049F38930E1
:10E4000039F38B3019F70895A1E21A2EAA1BBB1B12
:10E41000FD010DC0AA1FBB1FEE1FFF1FA217B307F0
:10E42000E407F50720F0A21BB30BE40BF50B661F06
:10E43000771F881F991F1A9469F7609570958095CA
:10E4400090959B01AC01BD01CF01089597FB092E6A
:10E4500005260ED057FD04D0D7DF0AD0001C38F4B3
:10E4600050954095309521953F4F4F4F5F4F089500
:10E47000F6F790958095709561957F4F8F4F9F4FE0
:02E480000895FD
:10E482005A7A41003F004800484C00485400484630
:10E49200002E0053544F50002100474F0048414C7A
:10E4A20054004C004C4300460046580054005900AA
:10E4B20056004D5400535200535300534500404000
:10E4C200004200534F004C4F4344554D50004C4FB7
:10E4D20043414444004C4F43434C45415200545243
:10E4E2004B44554D500054524B4144440054524BFE
:10E4F200434C4541520000019E3D0401773606011E
:10E502007736080162360B0169360E017036110149
:10E51200B6361301B6361801CB361A01CB361D01B9
:10E52200E0362201023724018C382701BD38290147
:10E53200063A2C015C3B2E018B3630010C3C320139
:10E54200323C35017D3C3801AC3C3B01123D3E0181
:10E55200335741013F3D4301703D4601C63D4E01E7
:10E56200513E5501DF3E5E01EB3E66015B3F6D01B0
:10E572008C3F0000000080058131810586318403D3
:10E582008B318503BA318804E43189040B328C0360
:10E5920036328D034F3290036D329403DC32950292
:10E5A200153398023133990154339C0259339D0338
:10E5B2007C33A001A333A2010034A4031734A501C4
:10E5C2003B34A6014434A7014A34C4015034C60284
:10E5D200C040C703B640C8015334C9019034CA01D0
:10E5E200D234CB016B35000000004D4D31006D6D12
:10E5F20031004D4D32006D6D32004443430064637F
:10E6020063002C20000000010000FF00020000FF58
:10E612000000B74DFF00030000FF0000CA4EFF00DC
:10E6220000B346FF00008E43FF0000D443FF010009
:10E632008A45FF0100E643FF0100B344FF01006287
:10E6420046FF0200BD49FF02002C49FF0200414A79
:10E65200FF0200A04AFF0200D049FF0200E349FF87
:10E662000200EB48FF03040000FF0300664E1303A1
:10E672000500001A0300754DFF030600001A03008F
:10E68200AD4BFF0300B24BFF04000A50FF040064CD
:10E6920050FF0500B74BFF0500AE4FFF0600D04B01
:10E6A200FF0600214CFF06006D4DFF0600714DFF75
:0EE6B2002534642D2534643A2000253464009C
:00000001FF
